:1080000000000120BD490200D5130200D513020073
:10801000D5130200D5130200D513020000000000A2
:10802000000000000000000000000000D513020066
:10803000D513020000000000D5130200D1B70100E3
:10804000D5130200D5130200D5130200D513020088
:10805000D5130200D5130200D5130200D513020078
:10806000D5130200D5130200D5130200D513020068
:10807000D5130200D5130200D5130200D513020058
:10808000D5130200D5130200D5130200D513020048
:10809000D5130200D5130200D5130200D513020038
:1080A000D5130200D5130200D5130200D513020028
:1080B000D5130200D5130200D5130200D513020018
:1080C000D5130200D5130200D5130200D513020008
:1080D000D5130200D5130200D5130200D5130200F8
:1080E000D5130200D5130200D5130200D5130200E8
:1080F000D5130200D9CA0100D5130200D51302001E
:10810000D51302006DCF0100D5130200D513020074
:10811000D5130200B5C80100D5130200D513020023
:10812000D5130200D5130200D5130200D5130200A7
:10813000D5130200D5130200D51302001DE601007D
:10814000DDDB0100D5130200D5130200D5130200B8
:10815000D5130200D5130200D5130200D513020077
:10816000D51302006D260200D5130200D5130200BC
:10817000D5130200D5130200D5130200D513020057
:10818000D5130200D5130200D5130200D513020047
:10819000D5130200D5130200D5130200D513020037
:1081A00069DB0100D5130200D5130200D5130200CC
:0C81B000D5130200D5130200D513020005
:10840000FFFFFFFFFFFFFFFFFFFFFFFF7EF9FFFF03
:1084200010B5054C237833B9044B13B10448AFF3AE
:1084300000800123237010BD0010FF1F000000000A
:10844000647202000C4B43B10C480D4910B5AFF3F8
:1084500000800C48036823B910BD0A48036833B98B
:108460007047094B002BF7D0BDE810401847064B6A
:10847000002BF5D0184700BF000000006472020016
:108480000410FF1FFC0EFF1F0000000010B515F0C8
:10849000D5FB064B00221A70054B1B689847054B0D
:1084A0009B69BDE810405B69184700BFB809FF1F12
:1084B000A400FF1F704C0200431E2DE9F047154633
:1084C000072B00F24F82DFE813F008000E000E00C9
:1084D00051006C00BC000301B301FFF7D7FF47F662
:1084E000A8532B603FE0764B764C022816BFA1467E
:1084F00099461C46744BDF68A9F10409043C4FF00F
:10850000FF364FF000084FF0010A3B68D9F804002D
:108510001B6998473B686068DB6898473B68606800
:108520005B6998473B68D9F804001B6A984718B9FB
:108530000AFA08F326EA03063B6854F8040F9B691D
:1085400098473B6859F8040F1B6A984718B10AFA14
:1085500008F326EA030608F10108B8F1110FD4D197
:10856000C6F310062E600020BDE8F08729600329BD
:108570001DD8DFE801F0020B0F13534BDB691B68BA
:108580001B889AB2322353431B14AAE74E4BDB6974
:108590005B68F5E74C4BDB699B68F1E74B4B1B696C
:1085A0009FE7012929601CD004D302292FD0022083
:1085B000BDE8F087444BDC68606823686430DB68A2
:1085C0009847606823688430DB6898472368606850
:1085D0005B6964309847236860685B6984309847BA
:1085E000C1E7394BDC6860682368C430DB689847B2
:1085F00060682368A430DB68984760682368C430EB
:108600005B699847236860685B69A430E7E72E4B95
:10861000DC686068236800F5A270DB6898476068D2
:10862000236800F5B270DB6898476068236800F53E
:10863000A2705B699847236860685B6900F5B27057
:10864000CDE70129296025D019D30229AFD11E4BCE
:10865000DC686068236800F5A270DB689847606892
:10866000236800F5B270DB6898476068236800F5FE
:10867000A2705B699847236860689B69DEE7124BCC
:10868000DC68606823688430DB689847236860682A
:108690001B699EE70C4BDC6860682368C430DB68AC
:1086A000984760682368A430DB689847606823684F
:1086B000C4305B699847236860689B69A5E700BF81
:1086C0004832FF1F3031FF1F704C0200B809FF1FF6
:1086D0002960002956D001297FF469AF7B4BDC6803
:1086E0006068236800F2C460DB68984760682368AC
:1086F00000F2C4609B6998476068236800F2E460F8
:10870000DB6898476068236800F2E4609B699847DB
:108710006068236800F20470DB689847606823682B
:1087200000F204709B6998476068236800F2247027
:10873000DB6898476068236800F224709B6998475B
:108740006068236800F24470DB68984760682368BB
:1087500000F244709B6998476068236800F2647077
:10876000DB6898476068236800F264709B699847EB
:108770006068236800F28470DB689847236860684B
:108780009B6952E0514BDD6868682B6800F2C46059
:10879000DB68984768682B6800F2C4605B6998479B
:1087A00068682B6800F2E460DB68984768682B68AB
:1087B00000F2E4605B69984768682B6800F2047017
:1087C000DB68984768682B6800F204705B6998471B
:1087D00068682B6800F22470DB68984768682B682B
:1087E00000F224705B69984768682B6800F2447057
:1087F000DB68984768682B6800F244705B699847AB
:1088000068682B6800F26470DB68984768682B68BA
:1088100000F264705B69984768682B6800F28470A6
:10882000DB6898472B6868685B6900F28470D6E65D
:10883000296000294CD001297FF4B9AE234BDC68B4
:108840006068236800F28450DB689847606823689A
:1088500000F284509B6998476068236800F2A45036
:10886000DB6898476068236800F2A4509B699847CA
:108870006068236800F2C450DB689847606823682A
:1088800000F2C4509B6998476068236800F2E45086
:10889000DB6898476068236800F2E4509B6998475A
:1088A0006068236800F20460DB68984760682368AA
:1088B00000F204609B6998476068236800F22460B6
:1088C000DB689847236860689B6948E0704C020049
:1088D000264BDD6868682B6800F28450DB68984797
:1088E00068682B6800F284505B69984768682B6859
:1088F00000F2A450DB68984768682B6800F2A45027
:108900005B69984768682B6800F2C450DB68984739
:1089100068682B6800F2C4505B69984768682B68E8
:1089200000F2E450DB68984768682B6800F2E45076
:108930005B69984768682B6800F20460DB689847B9
:1089400068682B6800F204605B69984768682B6868
:1089500000F22460DB6898472B6868685B6900F266
:1089600024603CE60420BDE8F08700BF704C0200A4
:1089700038B5064C2368C31AB3F5FA7F054604D30D
:10898000034B9B699B699847256038BD1C10FF1FEE
:10899000704C02003A4B3B4ADB685B6803F592710E
:1089A000116003F14401516003F18401916003F10E
:1089B000C401D16003F58271116103F5B271516197
:1089C00003F5D271916103F5F271D16103F509717B
:1089D000116203F51971516203F52971916203F572
:1089E0003971D16203F54971116303F5597151630E
:1089F00003F56971916303F57971D16303F2244141
:108A00001164214A191D116003F12401516003F121
:108A10006401916003F1A401D16003F1E4011161EB
:108A200003F5A271516103F5C271916103F5E27121
:108A3000D16103F50171116203F51171516203F502
:108A40002171916203F53171D16203F541711163B6
:108A500003F55171516303F56171916303F5717110
:108A600003F204431364094BD16301221A70084BCB
:108A7000084A1A65084A9A65084A5A65704700BF4D
:108A8000704C02003031FF1F4832FF1FB809FF1F32
:108A90007431FF1FB98400008D84000071890000CB
:108AA00070470220704702207047704770470220CD
:108AB00070470220704702207047012070477047BE
:108AC00070474369114A124910B5C3F80422C3F82C
:108AD0000822104B8365104B836183620363C3617B
:108AE0000E4B43640E4B83640E4B0F4A0F4C416296
:108AF00043630F49C36303640E4B4265C1628463E1
:108B00000465C164C265036610BD00BFBB8A000076
:108B1000A38A0000A18A0000A78A0000AB8A000097
:108B2000AD8A0000B38A0000C18A0000B78A000045
:108B3000AF8A0000BF8A0000704700BF0748084A9C
:108B4000C2670023137053704FF0FF3280F8783003
:108B500043670267C3666830FFF7B3BF7431FF1F16
:108B60002C10FF1F0648074A426100231370537000
:108B70004FF0FF320374C36082604360FFF7A1BF10
:108B80007431FF1F4412FF1F10B50023064C184616
:108B90001A5D590002F0030201338A40072B40EAB4
:108BA0000200F5D110BD00BF5C14FF1F0449002373
:108BB0005A5C02F00302C2540133072BF8D170470C
:108BC0005C14FF1F074B1A7802705A7842709A782B
:108BD0008270DA78C2701A7902715A7942719B797F
:108BE000837170475C14FF1FF8B5094B094F0A4D9C
:108BF000DE680024E15D33686A6CDB6952F82400AA
:108C000001F0030101349847072CF3D1F8BD00BFF0
:108C1000704C02005C14FF1F0800FF1F054A002370
:108C200000F0030199540133072B4FEA9000F7D16C
:108C3000DAE700BF5C14FF1F014B586AEEE700BF84
:108C40000800FF1F04490023C25C02F003025A54CB
:108C50000133072BF8D1C7E75C14FF1F074B0278DD
:108C60001A7042785A7082789A70C278DA700279F3
:108C70001A7142795A7182799A71B5E75C14FF1FB3
:108C8000074B1A68821AB2F57A7F04D39A685A6041
:108C900000229A6018609A6801329A60704700BF9B
:108CA0009014FF1F0020704701207047014B0022E5
:108CB0005A6070477431FF1F10B50C4613F01CFA50
:108CC000206010BD13F044BA022804BF0B4B93F888
:108CD000D00030B90A4BDB681B689B69094A1068F1
:108CE0001847012809D1054B93F8D030012B04D146
:108CF000034BDB681B685B69F0E770477431FF1F4B
:108D0000704C02009032FF1F10B50020FFF7DCFF0F
:108D1000044B054ADB6810681B68BDE810409B687F
:108D2000184700BF704C02009032FF1F4B2938B526
:108D30000446154600F0F38200F28E803B2900F0D5
:108D40000D8245D82E2900F0A4811CD82A2900F0D4
:108D5000448109D8282900F00C8100F224812729B8
:108D600000F0F9800424FDE02C2900F0668140F237
:108D70004A81002840F07B81112013F0BDF9C0F337
:108D800080702860EEE0332900F0BF8110D83029D0
:108D900000F0A881C0F094813129E3D1002C40F08B
:108DA000AA810021132013F032FA00242860D9E0B0
:108DB000392900F0BB8100F2C2813429D2D10028C8
:108DC00040F0AB810146012013F021FA2860C9E090
:108DD000432900F0438220D83F2900F0FF810ED8BC
:108DE0003D2900F0DF8140F2CB81002840F0EC818A
:108DF0000146072013F00BFA00B22860B2E04129C7
:108E000000F00E8240F2FB81002840F01D820146F6
:108E10000B2013F0FCF92860A4E0472900F05B82E6
:108E20000ED8452900F03C8240F22982002840F00B
:108E3000488201460F2013F0EAF900B2286091E061
:108E4000492900F06382A9D8002840F056821120F9
:108E500013F052F9286085E05B2900F0EC8240D8DD
:108E6000532900F08A821ED84F2900F06B820DD85A
:108E70004D2900F05D8240F23581002874D1014611
:108E8000212013F0C4F900B228606BE0512900F0F2
:108E90006B8240F26082002866D10146252013F0E3
:108EA000B6F928605EE0572900F08F820CD855296A
:108EB00000F0738240F26982002840F07D82312008
:108EC00013F01AF928604DE0592900F09C8240F215
:108ED0008B82002840F0A682352013F00DF928601F
:108EE00040E0632900F0E58219D85F2900F0C982CB
:108EF0000AD85D2900F0BD8240F2AC82A0BB3920C7
:108F000013F0FAF828602DE0612900F0CA8240F2DF
:108F1000C08248BB3D2013F0EFF8286022E06729AB
:108F200000F0DF820AD8652900F0D38240F2C982BE
:108F3000D0B9772013F0E0F8286013E0692900F039
:108F4000E082C0F0D682FF297FF40CAF60B9B84B45
:108F50005B68136006E038B90146142013F057F936
:108F600000B22860204638BD012C14BF0024042420
:108F7000F8E730B9112013F0BFF8C0F302402860C1
:108F8000F0E7012840F0C582112013F0B5F82B68F6
:108F90001B0403F4E02320F4E0211943112013F013
:108FA000D7F80024DEE730B9112013F0A5F8C0F39C
:108FB000C4402860D6E7012840F0AD82112013F0AC
:108FC0009BF82B68DB0403F4780320F47801194341
:108FD000112013F0BDF80024C4E728B9112013F0C4
:108FE0008BF880B22860BDE7012840F096821120FE
:108FF00013F082F82988000C00040143112013F0BB
:10900000A7F80024AEE730B9112013F075F8C0F3CB
:1090100002602860A6E7012840F08182112013F049
:109020006BF82B681B0603F0E06320F0E061194346
:10903000112013F08DF8002494E730B9112013F0BB
:109040005BF8C0F3C26028608CE7012840F06982B9
:10905000112013F051F82B68DB0603F0605320F069
:1090600060511943112013F073F800247AE70128A6
:1090700040F05982112013F03FF82B689B0703F052
:10908000804320F080411943112013F061F800243F
:1090900068E728B9112013F02FF8C00F286061E7A6
:1090A000012840F04282112013F026F8296820F0B0
:1090B000004040EAC171112013F04AF8002451E742
:1090C00030B90146122013F0A2F800B2286049E737
:1090D000012C40F02C822A880021122013F0C8F8BD
:1090E00000243FE7002C7FF43FAF152013F004F875
:1090F0000024286036E7012C40F01B822A880021DA
:10910000132013F0B5F800242CE700287FF42CAFCF
:10911000014613F07CF8286024E7012840F00B8218
:109120001288002113F0A4F800241BE700287FF424
:109130001BAF0021022013F06AF8286012E720B963
:10914000032012F0D9FF28600CE7012840F0F581D8
:109150001168032012F0FCFF002403E730B9014638
:10916000042013F054F800B22860FBE6012840F018
:10917000E68112880021042013F07AF80024F1E639
:1091800030B90146052013F042F800B22860E9E644
:10919000012840F0D68112880021052013F068F8DC
:1091A0000024DFE630B90021062013F030F800B2C9
:1091B0002860D7E6012840F0C681128800210620E9
:1091C00013F056F80024CDE6012840F0BE81128845
:1091D0000021072013F04CF80024C3E628B901460B
:1091E000082013F014F82860BCE6012840F0AF8195
:1091F00012880021082013F03BF80024B2E628B9B9
:109200000146092013F003F82860ABE6012840F07E
:10921000A08112880021092013F02AF80024A1E679
:1092200040B900210A2012F0F2FF28609AE600BF40
:109230009014FF1F012840F08E81128800210A201F
:1092400013F016F800248DE6012840F0868112887C
:1092500000210B2013F00CF8002483E628B9014606
:109260000C2012F0D4FF28607CE6012840F07781C2
:10927000128800210C2012F0FBFF002472E628B9AE
:1092800001460D2012F0C3FF28606BE6012840F074
:109290006881128800210D2012F0EAFF002461E6A7
:1092A00028B900210E2012F0B2FF28605AE60128EA
:1092B00040F05981128800210E2012F0D9FF0024BD
:1092C00050E6012840F05181128800210F2012F051
:1092D000CFFF002446E630B90146102012F097FF78
:1092E00000B228603EE6012840F04181128800214A
:1092F000102012F0BDFF002434E6012840F039812F
:109300001168112012F024FF00242BE600287FF4BE
:10931000DFAE0021122012F07AFF286022E600283A
:109320007FF422AE0146142012F071FF286019E686
:1093300000287FF419AE0021202012F068FF00B24F
:1093400028600FE600287FF40FAE0146222012F0BD
:109350005EFF286006E600287FF406AE0146232063
:1093600012F055FF2860FDE500287FF4FDAD0021D7
:10937000242012F04CFF2860F4E500287FF4F4ADBF
:10938000262012F0B9FE2860ECE500287FF4ECAD51
:10939000272012F0B1FE2860E4E520B9302012F059
:1093A000ABFE2860DEE5012840F0E5801168302042
:1093B00012F0CEFE0024D5E5012840F0DE801168D1
:1093C000312012F0C5FE0024CCE520B9322012F085
:1093D00093FE2860C6E5012840F0D1801168322054
:1093E00012F0B6FE0024BDE520B9332012F084FE51
:1093F0002860B7E5012840F0C4801168332012F0DE
:10940000A7FE0024AEE520B9342012F075FE2860D6
:10941000A8E5012840F0B7801168342012F098FECA
:1094200000249FE5012840F0B0801168352012F03B
:109430008FFE002496E520B9362012F05DFE2860EC
:1094400090E5012840F0A3801168362012F080FEDC
:10945000002487E520B9372012F04EFE286081E510
:10946000012840F096801168372012F071FE002428
:1094700078E500287FF478AD382012F03DFE2860B2
:1094800070E500287FF470AD3A2012F035FE2860B8
:1094900068E500287FF468AD3B2012F02DFE2860BF
:1094A00060E500287FF460AD3C2012F025FE2860C6
:1094B00058E500287FF458AD3E2012F01DFE2860CC
:1094C00050E500287FF450AD3F2012F015FE2860D3
:1094D00048E500287FF448AD762012F00DFE2860A4
:1094E00040E500287FF440AD7C2012F005FE2860A6
:1094F00038E500287FF438AD7D2012F0FDFD2860AE
:1095000030E500287FF430AD7E2012F0F5FD2860B4
:1095100028E5002426E5002424E5002422E5002493
:1095200020E500241EE500241CE500241AE50024A3
:1095300018E5002416E5002414E5002412E50024B3
:1095400010E500240EE500240CE500240AE50024C3
:1095500008E5002406E5002404E5002402E50024D3
:1095600000E50024FEE40024FCE40024FAE40024E6
:10957000F8E40024F6E40024F4E40024F2E40024F7
:10958000F0E40024EEE40024ECE40024EAE4002407
:10959000E8E40024E6E40B4619B901461846FFF753
:1095A000C5BB082070470120704707B5019239B943
:1095B000014601AA0120FFF7B9FB03B05DF804FBE7
:1095C0000820FAE7084612F097BD0846114612F047
:1095D000BFBD12F01CBE12F04BBE38B51B4B1C4D6C
:1095E000DC686068236864302860DB68984723681B
:1095F00028685B699847174B17495A690A601749E9
:10960000C2F804121649C2F8081201200021517054
:109610001070144A9A63144A5A63144A9A64144A9A
:109620005A64144A5A65144A1A65144A1A66144A46
:10963000DA65144A9A653222DA6018744FF48C7233
:109640009A60BDE83840FFF73FBB00BF704C020096
:109650009032FF1F7431FF1F8C32FF1FA79500004F
:10966000A98C000097950000AB950000C58C000008
:10967000B98C0000818C0000A58C0000C98C000012
:10968000AD8C0000098D0000014B0022DA667047A6
:109690007431FF1F70B50B4E0B4D33682A460146DF
:1096A0000446002015F0B1FC002015F09FF8336847
:1096B0002A462146012015F0A8FC0120BDE8704093
:1096C00015F094B81435FF1F9432FF1F012808B518
:1096D00003D815F07FF8002008BD082008BD012838
:1096E00008B503D815F06AF8002008BD082008BDA9
:1096F0000021F4E74942F2E7F1E7024B186815F060
:1097000094BC00BF1435FF1F38B5002015F04CF98C
:1097100008B1002038BD012015F046F905460028A3
:10972000F7D10A4B0A4C186815F076FC15F082F94F
:109730002B46A2682168284615F0CCF82B46E26833
:109740006168012015F0C6F8012038BD1435FF1FEF
:10975000A814FF1F022804BF0B4B93F8D00030B9A8
:109760000A4BDB681B685B69094A106918470128C6
:1097700009D1054B93F8D030012B04D1034BDB68A2
:109780001B689B69F0E770477431FF1F704C020043
:10979000A814FF1F70B50020FFF7DCFF0A4B0B4C2D
:1097A000DD6820692B689B6898472B68206A9B6856
:1097B00098472B68606A9B68984715F089F9044BB5
:1097C000BDE870405B681847704C0200A814FF1F8A
:1097D0006809FF1F012838B504460D4605D820B991
:1097E00015F0E2F82860204638BD082038BD022870
:1097F00010B5144610D0032815D0012817D10D4BF1
:109800000D4ADB68106A1B681B6A9847003018BF56
:1098100001202060002010BD064B074ADB68506A1B
:109820001B681B6AF1E7084615F034F8F1E70420DD
:1098300010BD00BF704C0200A814FF1F012838B5EE
:1098400004460D4608D815F095F82B68C118296014
:109850002046BDE8384039E7082038BD2DE9F843F7
:10986000184C9DF820609DF82450984623680F46B8
:109870009B68002147F080009146984723680021AB
:109880009B6848469847236800219B684046984754
:10989000236800219B6830469847236828469B68C8
:1098A00001219847084B1B6848EA092807F07F0701
:1098B00046EA082603EB870745EA06257D60BDE8F2
:1098C000F88300BF1835FF1F1435FF1F07B5D3B24B
:1098D0000193C2F307230093C2F30743120EFFF76D
:1098E000BDFF03B05DF804FB0A4601460020FFF708
:1098F000EDBF38B5234B01F07F04234493F80032C9
:10990000DB0705D4204B1B6803EB8404606838BD7B
:109910001E4D2B6800219B68204698472B6800212C
:109920009B68084698472B6800219B680846984723
:109930002B6800219B68084698472B6801219B688B
:10994000002098472B6800219B68204698472B6889
:1099500000219B68084698472B68002104029B68F9
:10996000084698472B68002104439B68084698479F
:109970002B68240204439B6801210020984724029D
:10998000204338BD9432FF1F1435FF1F1835FF1FC9
:1099900010B50C4601460020FFF7ABFF206010BD5C
:1099A000A42A2DE9F04104460D461E4600F0C1816F
:1099B00049D8062A00F0E38017D8022A00F0B780C1
:1099C00007D8002A00F09680012A00F0A480042421
:1099D00099E0042A00F0BD8040F2B580002840F0F4
:1099E000C780084614F0FCFF88E01D2A00F01D81A6
:1099F00014D8082A00F00081C0F0E1801C2AE6D1CA
:109A0000002840F00081090141F06C0101F0FC01E7
:109A10002846FFF76EFFC0F380406FE0A22A00F0F7
:109A20004C8100F268818C2AD1D1002840F003815A
:109A3000090141F06C0101F0FC012846FFF759FFD4
:109A4000C0F303605AE0AC2A00F0878229D8A82A24
:109A500000F0188212D8A62A00F0D98140F287813E
:109A6000002840F0FE81090141F06C0101F0FC0189
:109A70002846FFF73EFF00F00F003FE0AA2A00F063
:109A80003C8240F21C82002840F05582090141F0DE
:109A90006D0101F0FD012846FFF72BFFC0F34110D7
:109AA0002CE0B42A00F0BC8214D8AE2A00F08182E7
:109AB000C0F06182B32A8AD1002840F09F82090158
:109AC00041F06C0101F0FC012846FFF712FFC0F3E2
:109AD000404013E0B82A00F0B882CE2A00F0D382CA
:109AE000B52A7FF474AF002840F0A782084614F02E
:109AF00093FF03E020B9084614F048FF306002E00D
:109B0000012803D000242046BDE8F08119682846CA
:109B100014F060FEF6E718B9084614F02BFFEDE7E5
:109B20000128EFD11968284614F0FEFEEAE718B9BB
:109B3000084614F047FFE1E70128E3D119682846F9
:109B400014F03CFEDEE7002871D1084614F02CFF2B
:109B5000D4E718B9084614F051FFCFE70128D1D156
:109B600019680029B8BF4942284614F0EBFEC9E73E
:109B70000128C7D11968284614F0DBFFC2E750B9A5
:109B80002021A94041F01001C9B22846FFF7B1FEDB
:109B9000C0F30420B2E70128B4D120248C4044F063
:109BA0001004E4B221462846FFF7A3FE33681B02E7
:109BB00003F4F85320F4F8521A43214623E150B934
:109BC0002021A94041F01001C9B22846FFF791FEBB
:109BD00000F01F0092E7012894D120248C4044F02B
:109BE0001004E4B221462846FFF783FE336820F0D4
:109BF0001F0203F01F03DFE7C8B9084614F04AFE4E
:109C0000C0F300107AE701287FF47CAF0C0144F028
:109C10006C04E4B221462846FFF76BFE33689B04D0
:109C200003F4802320F48022C6E700288ED0012C84
:109C30003FF4CDAE66E701287FF464AF1B68102BBC
:109C400023D00DDC022B1CD004DC012B16D04FF0EE
:109C5000FF3314E0042B16D0082BF8D105230EE0B7
:109C6000402B14D003DC202BF1D1032307E0802B01
:109C70000FD0B3F5807FEAD1002300E008233360E2
:109C800008E00723FBE70623F9E70423F7E70223AD
:109C9000F5E73060336801333FF434AF2C0144F012
:109CA0006C04E4B221462846FFF723FE33681B0606
:109CB00003F0706320F070627EE750B9090141F053
:109CC0006C0101F0FC012846FFF713FEC0F3C13020
:109CD00014E701287FF416AF0C0144F06C04E4B2E1
:109CE00021462846FFF705FE3368DB0303F4C03343
:109CF00020F4C03260E750B9090141F06C0101F075
:109D0000FC012846FFF7F5FDC0F38030F6E6012898
:109D10007FF4F8AE0C0144F06C04E4B2214628460E
:109D2000FFF7E7FD33689B0303F4804320F4804290
:109D300042E750B9090141F06C0101F0FC012846ED
:109D4000FFF7D7FDC0F30030D8E601287FF4DAAE84
:109D50000C0144F06C04E4B221462846FFF7C9FD2B
:109D600033681B0303F4805320F4805224E70F016F
:109D700047F06C07FFB239462846FFF7BAFD804628
:109D8000A4B918F4804F3946284604D0FFF7B1FD36
:109D9000C0F3C310B2E6FFF7ACFD18F4006FC0F3D8
:109DA000021018BF40F008003060ABE6012C7FF4D1
:109DB000A9AE18F480483946284608D0FFF799FD27
:109DC0003368DB0103F4F06320F4F06247E0FFF74F
:109DD00090FD3268120120F0700002F07002024320
:109DE00039462846FFF772FD39462846FFF781FDC0
:109DF000336813F0080F20F4006218BF4FF40068B6
:109E000042EA080239462846FFF760FD7AE60F016C
:109E100047F06C07FFB239462846FFF76AFD74B970
:109E200010F480483946284604D0FFF762FDC0F39D
:109E3000021063E6FFF75DFDC0F3C310B4E7012C29
:109E40007FF460AE10F4804F39462846B6D0FFF755
:109E500050FD33681B0103F0700320F070021A43B9
:109E6000D0E701287FF44EAE0C0144F06C04E4B25C
:109E700021462846FFF73DFD336820F00F0203F02E
:109E80000F0399E650B9090141F06D0101F0FD01A0
:109E90002846FFF72EFDC0F3C0302FE601287FF4DF
:109EA00031AE0C0144F06D04E4B221462846FFF7C0
:109EB00020FD3368DB039BB220F400427CE650B9FE
:109EC000090141F06D0101F0FD012846FFF711FD88
:109ED000C0F3413012E601287FF414AE0C0144F0C7
:109EE0006D04E4B221462846FFF703FD33685B03A7
:109EF00003F4C04320F4C0425EE650B9090141F0CA
:109F00006D0101F0FD012846FFF7F3FCC0F30320CB
:109F1000F4E501287FF4F6AD0C0144F06D04E4B2E1
:109F200021462846FFF7E5FC33681B0203F4706303
:109F300020F4706240E601287FF4E4AD0C0144F0A7
:109F40006D04E4B221462846FFF7D3FC33685B0179
:109F500003F0600320F060022EE628B9090141F009
:109F60006D0101F0FD0183E501287FF4CBAD0C010B
:109F700044F06D047BE750B9090141F06D0101F037
:109F8000FD012846FFF7B5FCC0F30060B6E50128E7
:109F90007FF4B8AD0C0144F06D04E4B221462846CC
:109FA000FFF7A7FC33681B0603F0807320F0807274
:109FB00002E688B9090141F06D0101F0FD01284672
:109FC000FFF797FC001400F07F0310F0400018BF6B
:109FD0006FF07F00184391E501287FF493AD0C01E9
:109FE00044F06D04E4B221462846FFF782FC336852
:109FF0001B0403F4FE0320F4FE02DDE501287FF4D8
:10A0000081AD0C0144F06C04E4B221462846FFF710
:10A0100070FC33685B0403F4003320F40032CBE5BA
:10A0200000287FF404AE090141F06F01C9B228464F
:10A03000FFF75FFCC0F3044060E501287FF462ADE8
:10A040001968284614F088FC5CE550B9090141F014
:10A050006C0101F0FC012846FFF74BFCC0F34030D7
:10A060004CE501287FF44EAD0C0144F06C04E4B2E1
:10A0700021462846FFF73DFC33685B0303F4005399
:10A0800020F4005298E500287FF4D1AD090141F099
:10A090006F01C9B22846FFF72CFCC0F309002DE57B
:10A0A00007B50129019207D8024601AB0120FFF74D
:10A0B00077FC03B05DF804FB0820FAE7012913469A
:10A0C00002D8024600206BE40820704770B54E4E5F
:10A0D0004E484F4C14F066FFF5686B6803F164025C
:10A0E000226103F1E402626203F58272226203F5E7
:10A0F000A272A26003F5B27203F59270626003F57A
:10A10000C27203F50173A3622B68E260DB68206012
:10A1100098472B68A068DB6898472B686068DB6805
:10A1200098472B68E068DB6898472B682069DB68F4
:10A1300098472B68A06ADB68364D98473369364AE2
:10A1400003F110011160A26A5A61344B344A1A605B
:10A1500014F070FC0023A2682168184614F0BAFBC2
:10A16000E26861680023012014F0B4FB2D4B2E49F6
:10A17000DA6FC2F804122D49C2F808120024012136
:10A18000117054702A4AC3F888202A4AC3F88420E0
:10A19000294AC3F88020294AC3F88C20284AC3F8EA
:10A1A000A020284AC3F89C20274AC3F89020274AB9
:10A1B000C3F89420264AC3F8B020264AC3F8AC203E
:10A1C000254AC3F8BC20254AC3F8B820244AC3F85E
:10A1D000B420244AC3F8C820234AC3F8C42032223A
:10A1E0005A674FF48F7202201A67204A83F878006A
:10A1F000C3F8C020FFF7AEFA2B689847AB6820463B
:10A20000BDE87040184700BF704C02009432FF1F39
:10A21000A814FF1F6809FF1F1835FF1F1435FF1F03
:10A220002C10FF1F7431FF1F09970000FB960000E0
:10A23000DF960000F9960000F5960000F196000008
:10A24000BDA00000A1A00000CD9600003D98000038
:10A25000E99800009199000095960000EF970000A2
:10A26000D59700005597000089960000959700004B
:10A27000014B0846DB6B18470800FF1F034B10B566
:10A280001B6C0C469847206010BD00BF0800FF1FE4
:10A2900007B5034B68461B6B984703B05DF804FB9A
:10A2A0000800FF1F70B50020FFF7F2FF1E4B1F4C88
:10A2B000DD68206B2B689B6898472B68E06A9B6879
:10A2C00098472B68E0689B6898472B68A0689B6854
:10A2D00098472B6860689B6898472B6820689B6844
:10A2E00098472B68A0699B6898472B68E0699B6832
:10A2F00098472B68A06A9B6898472B6860699B68A1
:10A3000098472B68206A9B6898472B68606A9B680F
:10A3100098472B6820699B68984714F0D9FB044B39
:10A32000BDE870405B681847704C0200E014FF1FE6
:10A330006809FF1F002014F059BA38B515460446C5
:10A3400028B9084614F0A6FA2860204638BD042033
:10A3500038BD10B5044618B914F03CFA204610BDBB
:10A36000082010BD10B5044618B914F027FA20468D
:10A3700010BD082010BD0021F4E74942F2E7F1E7E3
:10A38000062873B505460C465DD8022903D9012875
:10A390005BD10F2959DC2E4E6846336B9847334604
:10A3A000052D06D8DFE805F0030B4346494C8DF830
:10A3B00000406846DB6A9847002002B070BD082C58
:10A3C000F7D8DFE804F0050C11161B20252A2F0012
:10A3D000F2788DF80120327B8DF80220E9E732799E
:10A3E0008DF80120727BF7E772798DF80120B27B3E
:10A3F000F2E7B2798DF80120F27BEDE7F2798DF882
:10A400000120327CE8E7727A8DF80120B27CE3E724
:10A41000B27A8DF80120F27CDEE7327A8DF80120E5
:10A42000727CD9E7F27A8DF80120327DD4E78DF87D
:10A430000340BEE78DF80440BBE78DF80540B8E760
:10A440008DF80640B5E70420B7E71020B5E700BF58
:10A450000800FF1F73B5404D04462B6B68460E463F
:10A4600098472B46062C1DD8DFE804F0700464677B
:10A470006A6D70009DF80120E978914208D19DF83D
:10A480000200297B884203D10020306002B070BDF9
:10A490001979914208D19DF80200597B884203D175
:10A4A000012333600020F1E75979914206D19DF8EC
:10A4B0000200997B884201D10223F2E79979914207
:10A4C00006D19DF80200D97B884201D10323E8E739
:10A4D000D979914206D19DF80200197C884201D1B8
:10A4E0000423DEE7597A914206D19DF80200997C57
:10A4F000884201D10523D4E7997A914206D19DF88B
:10A500000200D97C884201D10623CAE7197A914218
:10A5100006D19DF80200597C884201D10723C0E78B
:10A52000D97A914215D19DF802201B7D9A4210D113
:10A530000823B6E79DF80330B3E79DF80430B0E791
:10A540009DF80530ADE79DF80630AAE79DF800308C
:10A55000A7E710209AE700BF0800FF1F38B50C4698
:10A56000054640B914F006FA2368C1182160284650
:10A57000BDE83840EDE6082038BD30B585B0054669
:10A5800001920C46002961D10B2812D8062846D228
:10A59000022837D004D848B301282CD004242EE058
:10A5A000042834D00528F9D11146204614F0C1FA08
:10A5B00025E013280ED80E2846D20C2836D00D28B8
:10A5C000ECD142F210739A42E8D8214B90B29B68CA
:10A5D000984714E08C28E1D101A90120FFF73AFF48
:10A5E0001C4B04469B6B02A8984708E0114614F0E8
:10A5F000F1F82C4603E01146204614F095F9204668
:10A6000005B030BD1146204614F0D8F8F7E782EACD
:10A61000E271A1EBE271204614F094F9EFE70638FD
:10A620001146C0B2FFF7ACFE0446E8E715460A4AF9
:10A630000A4BD26812681DB15269D86A9047DEE7AA
:10A640009269D86A9047D4E70E38E9E70824D6E73C
:10A650006809FF1F0800FF1F704C0200E014FF1F75
:10A6600010B51446002947D1132847D8DFE800F079
:10A670000A1014181C202424242424242C373E3EA1
:10A680003E3E3E3E002014F081F92060002010BDC7
:10A69000002014F06FF9F8E7002014F093F9F4E7C4
:10A6A000002014F081F9F0E7002014F0A7F9ECE79E
:10A6B000002014F095F9E8E708281FD1002014F0D5
:10A6C000E9F8C0F30010E0E70D4B0E4ADB68D06AF2
:10A6D0001B681B6A9847003018BF0120D5E7084B5C
:10A6E000084ADB68106B1B681B6AF3E70E381146DB
:10A6F000C0B2FFF7AFFEC9E7082010BD042010BDAF
:10A70000704C0200E014FF1F6B4B2DE9F041DE6836
:10A710006A4C70686A4F00F5E273236300F5D273E8
:10A72000E36200F52173E36000F52973A36000F58F
:10A730001973636000F50173236000F55973A36119
:10A7400000F55173E36100F16403A36200F5A273A5
:10A75000636100F56973236200F5717363623368A6
:10A7600000F59270DB682061984733686069DB68A8
:10A7700098473368206BDB6898473368E06ADB688A
:10A7800098473368206A1B6998473368606A1B6979
:10A7900098477B6CE2681A60A2685A6062689A60A7
:10A7A0002268DA60A2691A61E2695A61A26A9A6152
:10A7B00000257A6C33685059DB6898477A6C3368A7
:10A7C00050599B69043598471C2DF2D13D4DEB6FD4
:10A7D0004FF0000883F8008014F02CF943466269BA
:10A7E0002169404614F076F844F62061404614F0A2
:10A7F000A9F846F2A811404614F09BF9324BC5F86F
:10A800008830324BC5F88430314BC5F88030314B3D
:10A81000C5F88C30304BC5F8A030304BC5F89C30B3
:10A820002F4BC5F890302F4BC5F894302E4BC5F800
:10A83000B0302E4BC5F8AC302D4BC5F8B8302D4B91
:10A84000C5F8BC302C4BC5F8C830012385F87830EA
:10A8500002202A4BC5F8C030FFF71AFD404614F01D
:10A86000A3F810B1264B9B789BB1BB6A984714F0B4
:10A87000E1F8002318466269216914F02BF844F6C8
:10A880002061002014F05EF846F2A811002014F0B8
:10A8900050F93368206BDB689847206B194C042310
:10A8A000437533681B68984723689847A36800205E
:10A8B000BDE8F041184700BF704C0200E014FF1FD4
:10A8C0000800FF1F7431FF1F65A300007FA3000075
:10A8D0007BA3000077A3000061A600007BA5000019
:10A8E00053A300005DA5000071A200007DA200003E
:10A8F0003BA3000035A3000091A20000A5A2000028
:10A90000B809FF1F6809FF1F1B4B70B5DD681B4CA2
:10A910002B68A0685B6998472B6820689B689847FC
:10A920002B6860689B6898472B68206A9B689847EB
:10A930002B68606A9B6898472B68E0689B6898471B
:10A940002B6820699B6898472B6860699B689847CB
:10A950002B68A0699B6898472B68E0699B689847BB
:10A960002B68A0689B68984714F0B2F8044BBDE8C8
:10A9700070405B68184700BF704C02002015FF1F35
:10A980006809FF1F10B51446042804D8DFE800F05A
:10A99000052321343F00042010BD146844F62063D1
:10A9A0009C4239D81D4B1E4ADB68106A1B6842F274
:10A9B00010718C42DB6994BF00210121984742F25B
:10A9C0001173B4FBF3F003FB1040164B80B29B688D
:10A9D0009847002010BD114B1468DB6858681B684D
:10A9E0002CB1DB69002100F5F2709847F1E79B6814
:10A9F00000F5F2709847ECE7084B1168DB68084AED
:10AA00001B681069DB69003118BF0121EDE70846BA
:10AA100013F040FF2060DCE7102010BD704C0200F6
:10AA20002015FF1F6809FF1F10B5044618B913F061
:10AA3000D1FE204610BD082010BD10B5044618B93F
:10AA400013F0BCFE204610BD082010BD0021F4E725
:10AA50004942F2E7F1E7024B186814F031BB00BF3E
:10AA60009C37FF1F08B5002013F09EFF10B1084B64
:10AA7000987860B1074B186814F019FB13F0DAFFEF
:10AA800005490023184606C913F024FF012008BD1C
:10AA9000B809FF1F9C37FF1F2015FF1F022804BFA6
:10AAA0000B4B93F8D00030B90A4BDB681B685B692D
:10AAB000094A90681847012809D1054B93F8D0300E
:10AAC000012B04D1034BDB681B689B69F0E77047DF
:10AAD0007431FF1F704C02002015FF1F38B50D4662
:10AAE000044620B913F060FF2860204638BD0820D6
:10AAF00038BD38B50C46054640B913F03BFF236816
:10AB0000C11821602846BDE838408DE7082038BDCF
:10AB10002DE9F0471C4D9DF820709DF82460994662
:10AB200055F82030044688469B68002148F0800094
:10AB30009246984755F8243000219B685046984724
:10AB400055F8243000219B684846984755F8243032
:10AB500000219B683846984755F8243030469B685A
:10AB600001219847094B53F8243049EA0A2908F093
:10AB70007F0847EA092703EB880846EA0726C8F852
:10AB80000460BDE8F08700BFA037FF1F9C37FF1FA0
:10AB900007B5D3B20193C2F307230093C2F307436F
:10ABA000120EFFF7B5FF03B05DF804FB0A4601463D
:10ABB0000020FFF7EDBF70B52B4A4FF4207301F072
:10ABC0007F0403FB00232344054693F80032DB0790
:10ABD00006D4264B53F8203003EB8404606870BD24
:10ABE000234E56F8203000219B682046984756F89F
:10ABF000253000219B680846984756F825300021EB
:10AC00009B680846984756F8253000219B680846FF
:10AC1000984756F8253001219B680020984756F840
:10AC2000253000219B682046984756F825300021A2
:10AC30009B680846984756F82530002104029B6817
:10AC40000846984756F82530002104439B6808467B
:10AC5000984756F82530240204439B6801210020C0
:10AC600098472402204370BD1C35FF1F9C37FF1FEF
:10AC7000A037FF1F0F4B104A1B6810B5014600207C
:10AC800014F00EFA002013F0B1FD002013F002FEC4
:10AC900010F008040DD182060BD56F212046FFF776
:10ACA0008AFFC30105D520460221BDE8104013F0FC
:10ACB000C9BD10BD9C37FF1F1C35FF1F10B50C46CA
:10ACC00001460020FFF777FF206010BDA62AF8B5E7
:10ACD00004460D461E4600F0B18200F28180172A1C
:10ACE00000F0768130D8042A00F029810CD8012A9E
:10ACF00000F00681C0F0F480022A00F00D81032AE2
:10AD000000F016810424F0E0072A00F045810ED8F7
:10AD1000052A00F02381062AF4D1002840F02A8178
:10AD200010212846FFF747FFC0F30420DCE0082A83
:10AD300000F04681152AE5D10028E3D0012840F033
:10AD4000D8801A68112123E11D2A00F0A8811CD89F
:10AD50001A2A00F0668109D8182AD3D1002840F0B9
:10AD60005A8133212846FFF726FFBDE01B2A00F059
:10AD700070811C2AC6D1002840F0818101462846F6
:10AD8000FFF719FFC0F34000AEE0A32A00F0E68110
:10AD90000ED88C2A00F08A81A22AB3D1002840F074
:10ADA000CF816C212846FFF706FFC0F3C1309BE03E
:10ADB000A42A00F0E981A52AA4D1002840F00A8243
:10ADC0006C212846FFF7F7FE10F4804F4FF06C011E
:10ADD000284600F0EF81FFF7EEFEC0F3C31083E0DA
:10ADE000B52A00F01D833CD8AB2A00F0B28214D8FB
:10ADF000A82A00F07182C0F05A82A92A00F0858248
:10AE0000AA2A7FF47FAF002840F095826D21284662
:10AE1000FFF7D1FEC0F3032066E0AE2A00F0CD823A
:10AE20000FD8AC2A00F0AB82AD2A7FF46BAF0028BC
:10AE300040F0B5826D212846FFF7BDFEC0F30060EB
:10AE400052E0B32A00F0D682B42A7FF45BAF002828
:10AE500040F028816F212846FFF7ADFEC0F3044083
:10AE600042E0BB2A00F02F8316D8B82A00F0F78200
:10AE700007D8B62A7FF446AF002840F0DE821421BE
:10AE8000A8E0B92A00F0FB82BA2A7FF43BAF002881
:10AE900040F0078313219DE0C02A00F05F830FD8A4
:10AEA000BC2A00F03583BF2A7FF42CAF002840F085
:10AEB000438370212846FFF77EFEC0F3014013E074
:10AEC000CC2A00F05E83CE2A7FF41CAF002840F02D
:10AED000E9806F212846FFF76EFEC0F3090003E00A
:10AEE00028B9084613F052FD30602046F8BD01280D
:10AEF00001D00024F9E71968284613F06BFCF8E745
:10AF000018B9084613F036FDEEE70128F1D11968AB
:10AF1000284613F009FDECE718B9084613F052FD76
:10AF2000E2E70128E5D11968284613F047FCE0E77D
:10AF3000002840F0B780084613F036FDD4E718B972
:10AF4000084613F05BFDCFE70128D2D1196800292C
:10AF5000B8BF4942284613F0F5FCCAE718B90846BD
:10AF600013F03EFDC0E70128C3D11968284613F04D
:10AF7000E0FDBEE70128BCD110212846FFF71BFEEB
:10AF800033681B0203F4F85320F4F8521A431021DB
:10AF90002846FFF7FDFDACE730B910212846FFF742
:10AFA0000AFE00F01F009FE70128A2D110212846C9
:10AFB000FFF701FE336820F01F0203F01F03E5E7EF
:10AFC00000286FD1084613F065FCC0F300108BE732
:10AFD00078B915212846FFF7EEFDC34A002800F096
:10AFE0005E824FF0807393FBF0F09042A8BF104652
:10AFF000EBE001287FF47DAF1968BB4B49B14FF0FE
:10B00000807292FBF1F29A42A8BF1A463260152173
:10B01000BEE71A46FAE701287FF46BAF1A683321BE
:10B02000B6E730B96C212846FFF7C5FDC0F3804074
:10B030005AE701287FF45DAF6C212846FFF7BBFD7E
:10B0400033689B0403F4802320F480221A436C218C
:10B050009EE730B96C212846FFF7ADFDC0F3C04034
:10B0600042E701287FF445AF6C212846FFF7A3FD96
:10B070003368DB0403F4002320F40022E6E7012810
:10B080007FF437AF00212846FFF795FD33685B005A
:10B0900003F0020320F002021A43002178E700289F
:10B0A0003FF44AAF012C3FF42DAE22E750B96C219A
:10B0B0002846FFF780FD4FF48073C0F3036043FA26
:10B0C00000F011E701287FF414AF1B68102B23D088
:10B0D0000DDC022B1CD004DC012B16D04FF0FF330B
:10B0E00014E0042B16D0082BF8D105230EE0402BDA
:10B0F00014D003DC202BF1D1032307E0802B0FD0E9
:10B10000B3F5807FEAD1002300E00823336008E034
:10B110000723FBE70623F9E70423F7E70223F5E714
:10B1200030603368013300F042826C212846FFF71B
:10B1300042FD33681B0603F0706320F0706285E700
:10B1400001287FF4D6AE6C212846FFF734FD336822
:10B15000DB0303F4C03320F4C03277E730B96C214D
:10B160002846FFF728FDC0F38030BDE601287FF4B4
:10B17000C0AE6C212846FFF71EFD33689B0303F425
:10B18000804320F4804261E730B96C212846FFF704
:10B1900012FDC0F30030A7E601287FF4AAAE6C21AF
:10B1A0002846FFF708FD33681B0303F4805320F49F
:10B1B00080524BE7FFF7FFFC6C2107462846FFF75C
:10B1C000FAFC3A05C0F3021001D4306091E640F079
:10B1D000080089E601287FF48CAE6C212846FFF731
:10B1E000EAFC10F480444FF06C01284608D0FFF7C9
:10B1F000E2FC3368DB0103F4F06320F4F06225E73E
:10B20000FFF7D9FC6C212846FFF7D5FC336813F013
:10B21000080F20F4006218BF4FF400646C21284628
:10B220002243FFF7B5FC6C212846FFF7C4FC3368C6
:10B230001B0103F0700320F0700207E7E0B96C21F6
:10B240002846FFF7B8FC10F480474FF06C01284601
:10B2500004D0FFF7B0FCC0F3021045E6FFF7ABFCEB
:10B260006C2104462846FFF7A6FC2305C0F3C31053
:10B2700048BF40F00800A8E701287FF43AAE6C21EF
:10B280002846FFF798FC10F480444FF06C012846E4
:10B29000CBD1FFF790FC3368DB0103F4F06320F4BB
:10B2A000F0621A436C212846FFF772FC1DE630B9A4
:10B2B0006C212846FFF77FFC00F00F0014E6012800
:10B2C0007FF417AE6C212846FFF775FC336820F039
:10B2D0000F0203F00F03B9E640B96D212846FFF7CE
:10B2E0006AFCC0F3C030FFE5FFFF0F0001287FF4C8
:10B2F00000AE6D212846FFF75EFC3368DB039BB28E
:10B3000020F400421A436D2142E630B96D212846EF
:10B31000FFF751FCC0F34130E6E501287FF4E9ADC9
:10B320006D212846FFF747FC33685B0303F4C043F5
:10B3300020F4C042E6E701287FF4DBAD6D2128460A
:10B34000FFF739FC33681B0203F4706320F470626A
:10B35000D8E730B96D212846FFF72DFCC0F3411026
:10B36000C2E501287FF4C5AD6D212846FFF723FC17
:10B3700033685B0103F0600320F06002C2E708B9A4
:10B380006D2196E701287FF4B4AD6D212846FFF7C3
:10B3900012FC336820F00F0203F00F03B2E701281C
:10B3A0007FF4A7AD6D212846FFF705FC33681B0627
:10B3B00003F0807320F08072A4E768B96D212846FD
:10B3C000FFF7F9FB001400F07F0310F0400018BFF6
:10B3D0006FF07F00184387E501287FF48AAD6D2167
:10B3E0002846FFF7E8FB33681B0403F4FE0320F450
:10B3F000FE0287E730B96C212846FFF7DCFBC0F37B
:10B40000404071E501287FF474AD6C212846FFF7B8
:10B41000D2FB33685B0403F4003320F4003215E6FA
:10B4200018B9084613F0F8FA5EE501287FF461AD1B
:10B430001968284613F090FA5BE501287FF459ADAE
:10B4400019685C4B49B14FF0807292FBF1F29A425D
:10B45000A8BF1A46326014219AE51A46FAE730B9B5
:10B460006C212846FFF7A7FBC0F340303CE50128DC
:10B470007FF43FAD1A68520302F40052E7E530B999
:10B480006C212846FFF797FBC0F303502CE50128F9
:10B490007FF42FAD1A68120502F47002D7E510464A
:10B4A00093E601287FF425AD1968424B49B14FF06E
:10B4B000807292FBF1F29A42A8BF1A4632601321C1
:10B4C00066E51A46FAE730B970212846FFF773FBA4
:10B4D000C0F3072008E501287FF40BAD7021284652
:10B4E000FFF769FB3268120220F47F4092B20243F8
:10B4F00070212846FFF74CFB00212846FFF75BFB35
:10B500003368002B20F00402CCBF04230023C3E5E2
:10B5100028B970212846FFF74EFBC0B2E4E40128A9
:10B520007FF4E7AC70212846FFF745FB327820F026
:10B53000FF00024370212BE501287FF4DAAC1B6881
:10B54000032B34D870212846FFF735FB33681B04E2
:10B5500003F4403320F440321A43EBE708B970217A
:10B5600061E501287FF4C5AC70212846FFF723FB75
:10B570003368002B20F4802214BF4FF48023002373
:10B58000EAE730B970212846FFF715FBC0F30150F8
:10B59000AAE401287FF4ADAC70212846FFF70BFB2D
:10B5A00033681B0503F4401320F44012D4E7102441
:10B5B0009BE400BFFFFF0F0007B5019239B90246B7
:10B5C00001AB0120FFF782FB03B05DF804FB08200C
:10B5D000FAE710B413460446084619B9224610BCCF
:10B5E000FFF774BB082010BC70472DE9F041624D95
:10B5F0006248634C13F022FDEE68736803F1640245
:10B60000A26003F59272226003F5A272626003F5F4
:10B61000D272226203F5E272626203F55172E26055
:10B6200003F5597203F56970226103F5617203F540
:10B630007173E361336862611B69A0619847336885
:10B64000E0691B699847336860691B6998473368EC
:10B650002068DB68984733686068DB689847336820
:10B66000A068DB68984733682069DB6898473368CF
:10B67000E068DB6898473368606ADB68984733683E
:10B68000206ADB6898473368606A9B69984733682B
:10B69000206A9B699847336860699B69984733685B
:10B6A000E0689B6998472A69364B374D02F11001D3
:10B6B0001960736803F501735361344BEA6F1A60C4
:10B6C00013F0B8F9002394E80600184613F002F9C5
:10B6D000EB6F2F4AC3F804222E4AC3F80822002732
:10B6E00001221A705F702C4BC5F888302B4BC5F8BF
:10B6F00084302B4BC5F880302A4BC5F88C302A4B50
:10B70000C5F8A030294BC5F89C30294BC5F89030BE
:10B71000284BC5F89430284BC5F8B030274BC5F8F6
:10B72000AC30274BC5F8BC30264BC5F8B830264B9B
:10B73000C5F8B430254BC5F8C83032236B674FF4D9
:10B74000F0732B670220224B85F87820C5F8C030B3
:10B75000FFF7A4F93368606ADB689847606A1D4C9C
:10B760000423437533681B68984723689847A36888
:10B770003846BDE8F0411847704C02001C35FF1FE9
:10B780002015FF1FA037FF1F7431FF1F9C37FF1FBD
:10B7900065AA000057AA00003BAA000055AA0000B5
:10B7A00051AA00004DAA0000D3B50000B9B50000B1
:10B7B00029AA0000F3AA0000ADAB0000BDAC000058
:10B7C00075AC000085A90000DDAA00009DAA00005C
:10B7D00009A900006809FF1F014B0022DA667047C3
:10B7E0007431FF1FF7B505238DF8003060F07F033B
:10B7F0008DF802300B168DF803300B148DF80430E1
:10B800008DF806100B1206460D4600240122072172
:10B810006846104F8DF805308DF8014013F076FB27
:10B820003B688DF807009B6998473B681DF804004A
:10B830009B6801349847082CF7D102200FF0E8FFED
:10B84000054B1B6826F0800603EB8606756003B087
:10B85000F0BD00BFA837FF1FA437FF1FF0B5314B65
:10B8600000F07F06334485B093F80C32DB070D46B9
:10B8700006D42D4B1B6803EB860673682B604FE0E4
:10B880000523012203218DF80430284C8DF8066031
:10B89000002301A88DF8053013F038FB23688DF8DC
:10B8A00007009B699847236804211B690DEB010081
:10B8B00098470FF0A7FF07462368DB6998470728DA
:10B8C00029D9236808215B690DEB01009847012203
:10B8D000072102A89DF80F4013F018FB84421FD1E6
:10B8E0009DF80830052B1BD19DF80930FF2B17D18F
:10B8F0009DF80A30B34213D19DF80C309DF80B200F
:10B900001B0443EA02639DF80E2013439DF80D20AB
:10B9100043EA0223B2E738460FF084FF0A28CBD966
:10B9200005B0F0BDAC37FF1FA437FF1FA837FF1FBE
:10B9300008B5064B064A1B680146002013F002FCBE
:10B940000020BDE8084012F051BF00BFA437FF1F20
:10B95000AC37FF1F38B51546044628B9084612F023
:10B9600099FF2860204638BD042038BD10B5044634
:10B9700018B912F02FFF204610BD082010BD10B5D9
:10B98000044618B912F01AFF204610BD082010BD59
:10B990000021F4E74942F2E7F1E7024B186813F09F
:10B9A000E9BB00BFA437FF1F08B513F043F80649F1
:10B9B000002318468A68496812F08CFF034B186808
:10B9C000BDE8084013F0CDBB5415FF1FA437FF1F7F
:10B9D000022804BF0B4B93F8D00030B90A4BDB6848
:10B9E0001B685B69094A10681847012809D1054B93
:10B9F00093F8D030012B04D1034BDB681B689B69A3
:10BA0000F0E770477431FF1F704C02005415FF1FA0
:10BA100038B50020FFF7DCFF114B124CDD682068C1
:10BA20002B689B6898472B6860689B6898472B68D1
:10BA3000A0689B6898472B68E0689B6898472B68CC
:10BA400020699B6898472B6860699B6898472B68BA
:10BA5000A0699B689847BDE8384013F039B800BF2B
:10BA6000704C02005415FF1F38B50C46054640B90E
:10BA700012F080FF2368C11821602846BDE83840D5
:10BA800074E7082038BD08B519BB052823D8DFE8BE
:10BA900000F003090E22131B1146002012F09AFE3B
:10BAA000002008BD1146002012F03EFFF8E71146C5
:10BAB000002012F083FEF3E782EAE271A1EBE2716B
:10BAC000002012F03FFFEBE71146002013F031F8A1
:10BAD000E6E7082008BD042008BD10B5144601BBE8
:10BAE000052820D8DFE800F003090D111519002002
:10BAF00012F04CFF2060002010BD002012F03AFF31
:10BB0000F8E7002012F05EFFF4E7002012F04CFF8F
:10BB1000F0E7002012F072FFECE7002012F060FF67
:10BB2000E8E7082010BD042010BD5BE696E6012280
:10BB300070B511464A4E4B4C072013F089F94A481C
:10BB400013F0C8FAF5686B6803F59272626003F54A
:10BB5000A272A26003F1C402E26003F1E40203F105
:10BB60006400226103F18402A433A3612B68626143
:10BB7000DB68206098472B686068DB6898472B6813
:10BB8000A068DB6898472B68E068DB6898472B68FB
:10BB90002069DB6898472B6860691B6998472B68A8
:10BBA000A0691B699847F56A2B6898472F4B304965
:10BBB0001D60304BDA6F0A602F49C2F8041200256D
:10BBC00001262E4916705570C2F808122C4AC3F887
:10BBD00088202C4AC3F884202B4AC3F880202B4AA3
:10BBE000C3F88C202A4AC3F8A0202A4AC3F89C2014
:10BBF000294AC3F89020294AC3F89420284AC3F858
:10BC0000B020284AC3F8AC20274AC3F8B820274AF6
:10BC1000C3F8C820264AC3F8C42032225A674FF41A
:10BC2000C3721A67234AC3F8C020234A83F8786096
:10BC3000C3F8BC2012F0FEFE2B46A26861682846BD
:10BC400012F048FE28464FF4484112F07BFE284689
:10BC50004FF4484112F06DFF3046BDE87040B7E642
:10BC6000704C02005415FF1FAC37FF1FA837FF1F91
:10BC7000A437FF1F7431FF1FA9B900009BB9000052
:10BC80007FB9000099B9000095B9000091B9000092
:10BC9000DBBA000087BA00006DB9000069BA000085
:10BCA000E5B700005DB8000055B90000D1B900004B
:10BCB000D9B7000011BA000031B90000014B0022D1
:10BCC000DA6670477431FF1FF7B505238DF8003031
:10BCD00060F07F038DF802300B168DF803300B14E3
:10BCE0008DF804308DF806100B1206460D46002420
:10BCF000012207216846104F8DF805308DF801406C
:10BD000013F004F93B688DF807009B6998473B687E
:10BD10001DF804009B6801349847082CF7D10220D5
:10BD20000FF076FD054B1B6826F0800603EB8606B8
:10BD3000756003B0F0BD00BFC83CFF1FCC3CFF1FC7
:10BD4000F0B5314B00F07F06334485B093F80C32E8
:10BD5000DB070D4606D42D4B1B6803EB8606736884
:10BD60002B604FE00523012203218DF80430284C7D
:10BD70008DF80660002301A88DF8053013F0C6F891
:10BD800023688DF807009B699847236804211B6985
:10BD90000DEB010098470FF035FD07462368DB697E
:10BDA0009847072829D9236808215B690DEB010012
:10BDB00098470122072102A89DF80F4013F0A6F82A
:10BDC00084421FD19DF80830052B1BD19DF8093006
:10BDD000FF2B17D19DF80A30B34213D19DF80C30D8
:10BDE0009DF80B201B0443EA02639DF80E201343C9
:10BDF0009DF80D2043EA0223B2E738460FF012FD0A
:10BE00001428CBD905B0F0BD383AFF1FCC3CFF1F3A
:10BE1000C83CFF1F08B5064B064A1B6801460020B8
:10BE200013F0ECF90020BDE8084012F0DFBC00BFC1
:10BE3000CC3CFF1F383AFF1F38B51546044628B9D9
:10BE4000084612F027FD2860204638BD042038BD82
:10BE500010B5044618B912F0BDFC204610BD0820EC
:10BE600010BD10B5044618B912F0A8FC204610BD4C
:10BE7000082010BD0021F4E74942F2E7F1E7024B48
:10BE8000186813F0D3B900BFCC3CFF1F08B512F0FF
:10BE9000D1FD0649002318468A68496812F01AFD48
:10BEA000034B1868BDE8084013F0B7B97C15FF1FB5
:10BEB000CC3CFF1F022804BF0B4B93F8D00030B9D5
:10BEC0000A4BDB681B685B69094A10681847012840
:10BED00009D1054B93F8D030012B04D1034BDB681B
:10BEE0001B689B69F0E770477431FF1F704C0200BC
:10BEF0007C15FF1F70B5144E144C0020FFF7DAFFBD
:10BF0000F56820682B689B6898472B6860689B6879
:10BF100098472B68A0689B6898472B68E0689B68E7
:10BF200098472B6820699B6898472B6860699B68D5
:10BF300098472B68A0699B689847F36A5B689847A5
:10BF4000BDE8704012F0C4BD704C02007C15FF1FAC
:10BF500038B50C46054640B912F00CFD2368C118EF
:10BF600021602846BDE8384072E7082038BD08B592
:10BF700019BB052823D8DFE800F003090E22131BA4
:10BF80001146002012F026FC002008BD11460020BA
:10BF900012F0CAFCF8E71146002012F00FFCF3E79C
:10BFA00082EAE271A1EBE271002012F0CBFCEBE738
:10BFB0001146002012F0BDFDE6E7082008BD042070
:10BFC00008BD10B5144601BB052820D8DFE800F0F5
:10BFD00003090D111519002012F0D8FC2060002073
:10BFE00010BD002012F0C6FCF8E7002012F0EAFCB9
:10BFF000F4E7002012F0D8FCF0E7002012F0FEFC7D
:10C00000ECE7002012F0ECFCE8E7082010BD04206B
:10C0100010BD59E694E6012270B511464A4E4B4CCC
:10C02000072012F015FF4A4813F0AEF8F5686B6868
:10C0300003F59272626003F5A272A26003F1C4027A
:10C04000E26003F1E40203F16400226103F184027F
:10C05000A433A3612B686261DB68206098472B687A
:10C060006068DB6898472B68A068DB6898472B6896
:10C07000E068DB6898472B682069DB6898472B6885
:10C0800060691B6998472B68A0691B699847F56A26
:10C090002B6898472F4B30491D60304BDA6F0A6090
:10C0A0002F49C2F80412002501262E49167055703A
:10C0B000C2F808122C4AC3F888202C4AC3F88420FE
:10C0C0002B4AC3F880202B4AC3F88C202A4AC3F895
:10C0D000A0202A4AC3F89C20294AC3F89020294A64
:10C0E000C3F89420284AC3F8B020284AC3F8AC20EB
:10C0F000274AC3F8B820274AC3F8C820264AC3F8FD
:10C10000C42032225A674FF4C3721A67234AC3F815
:10C11000C020234A83F87860C3F8BC2012F08AFC60
:10C120002B46A2686168284612F0D4FB28464FF4DB
:10C13000484112F007FC28464FF4484112F0F9FC40
:10C140003046BDE87040B5E6704C02007C15FF1F1C
:10C15000383AFF1FC83CFF1FCC3CFF1F7431FF1F44
:10C160008DBE00007FBE000063BE00007DBE0000EB
:10C1700079BE000075BE0000C3BF00006FBF0000A5
:10C1800051BE000051BF0000C9BC000041BD00000D
:10C1900039BE0000B5BE0000BDBC0000F5BE000009
:10C1A00015BE0000012810B514460CD003D3022898
:10C1B00010D0042010BD1368094AB3FA83F35B0959
:10C1C0009372002010BD1368064AB3FA83F35B092B
:10C1D0001360F6E7084612F05DFB2060F1E700BF50
:10C1E000D03CFF1F6C00FF1F10B5044618B912F0B9
:10C1F000F1FA204610BD082010BD024B186813F05C
:10C20000B4B800BF1C3DFF1F022804BF0B4B93F8BE
:10C21000D00030B90A4BDB681B685B69094AD068FB
:10C220001847012809D1054B93F8D030012B04D1D0
:10C23000034BDB681B689B69F0E770477431FF1F95
:10C24000704C0200A415FF1F38B50020FFF7DCFF7B
:10C250000F4B104CDD68E0682B685B6998472B68D2
:10C2600020689B6898472B68A0689B6898472B6854
:10C27000E0689B6898472B6820699B6898472B6803
:10C2800060689B689847BDE8384012F021BC00BF49
:10C29000704C0200A415FF1F38B50D46044620B9A6
:10C2A00012F082FB2860204638BD082038BD38B522
:10C2B0000C46054640B912F05DFB2368C1182160A9
:10C2C0002846BDE838408FE7082038BD10B5044641
:10C2D00030B9044B5872187212F070FA204610BD33
:10C2E000082010BDD03CFF1F0021EFE74942EDE7D9
:10C2F000ECE738B5002012F057FB0546A8B90C4B07
:10C300000C48196813F014F80B4B012402201C6030
:10C31000FFF77AFF12F08EFB084928460B698A68FE
:10C32000496812F0D7FA204638BD002038BD00BF5A
:10C330001C3DFF1FD03CFF1F6C00FF1FA415FF1FFB
:10C340002DE9F843830C04460DD0C0F34243062B7D
:10C3500009D1294B5A7A20F01F04002A43D01B78B8
:10C3600003F01F031C43254F254E264D3B68D6F88E
:10C37000008095F818909B680021C4F30740984707
:10C380002A7E336808EB890803EB8203C8F80400AF
:10C390005A6812025A603B6800219B68C4F3072068
:10C3A00098472B7E326802EB8302012153681843C1
:10C3B0003B68000250609B68E0B298473268297E73
:10C3C00002EB81014B6818430011A30C4860106117
:10C3D0000BD0C4F34243072B02D1C4F301112976D9
:10C3E00043F0080302E0DB7ABAE7082302EB830399
:10C3F0005C60BDE8F88300BFD03CFF1F183DFF1F05
:10C400001C3DFF1FA415FF1F0346C1F31300820C40
:10C4100010B40C4C05D04214062A04BF01F01F01D1
:10C42000E172094A03F07703126843F0080302EB54
:10C4300083035860A37A13B910BCFFF781BF10BC07
:10C44000704700BFD03CFF1F1C3DFF1FDCE738B525
:10C4500004460F2000F014F80323B4FBF3F303EBBE
:10C460004303E41A2401054604F0300420F03000B0
:10C470002043FFF765FF2846BDE83840FFF760BF5F
:10C4800010B5084B9B7A04461BB9030701D4FFF78C
:10C49000DEFF054B1B6804F07F0403EB8404606837
:10C4A00010BD00BFD03CFF1F1C3DFF1FA82A38B5A0
:10C4B00004461D46084600F03E8260D81D2A00F062
:10C4C000EA8023D8042A00F0F1800CD8012A00F079
:10C4D000C880C0F0B880022A00F0D080032A00F0A3
:10C4E000DA800424B3E0062A00F0FD80C0F0EE807C
:10C4F000072A00F01181082AF3D1002C40F0D180E6
:10C5000012F0C8F9C0F300102860A0E0A32A00F0E0
:10C51000978120D8A02A00F04D810DD88C2AE0D137
:10C52000002C40F006810820FFF7AAFF00F00F0062
:10C53000C0F1080028608AE0A12A00F05581A22AF3
:10C54000CFD1002C40F06A810C20FFF799FFC0F397
:10C55000C13028607BE0A52A00F0A881C0F08C8162
:10C56000A62A00F0BD81A72ABBD1002C40F0D281C1
:10C570000C20FFF785FF00F00F00286067E0B22A6B
:10C5800000F0C88228D8AD2A00F0448210D8AA2A28
:10C5900000F00482C0F0E881AB2A00F01982AC2AD6
:10C5A0009FD1002C40F02E82B24B5B7B2B604EE083
:10C5B000AF2A00F06A82C0F04782B02A00F07E8283
:10C5C000B12A8ED1002C40F093820720FFF758FF4C
:10C5D000C0F3802028603AE0B72A00F0EE8211D83C
:10C5E000B42A00F0CB82C0F0AF82B52A00F0D0822E
:10C5F000B62A7FF476AF002C40F0D7829D4B1B69A2
:10C600002B6024E0CE2A00F01C830FD8B82A00F05B
:10C61000ED82B92A7FF465AF002C40F0018307203A
:10C62000FFF72EFFC0F30040286010E0D02A00F092
:10C630001D83D62A7FF455AF002C40F020838D4B0C
:10C640005B682B6003E024B912F0A0F92860204653
:10C6500038BD012C40F01A83196812F0BBF8002491
:10C66000F5E71CB912F086F92860F0E7012C40F0DC
:10C670000F83196812F058F90024E8E71CB912F08A
:10C68000A1F92860E3E7012C40F00483196812F057
:10C6900095F80024DBE724B912F086F9002428601D
:10C6A000D5E7012C14BF00240424D0E71CB912F0F4
:10C6B000A5F92860CBE7012C40F0EE82196800292B
:10C6C000B8BF494212F03EF90024C0E71CB912F08D
:10C6D00087F92860BBE7012C40F0E082196812F06E
:10C6E00028FA0024B3E71CB9624BDB7A2B60AEE773
:10C6F000012C40F0D5821A685E4B0E20DA72FFF7EB
:10C70000BFFE2B6820F01F0103F01F0319430E200A
:10C71000FFF77AFE00249AE71CB9564B1B782B6072
:10C7200095E7012C40F0BE821A68524B00241A7023
:10C730008DE7012C40F0B8821B68102B23D00DDC54
:10C74000022B1CD004DC012B16D04FF0FF3314E079
:10C75000042B16D0082BF8D105230EE0402B14D063
:10C7600003DC202BF1D1032307E0802B0FD0B3F59E
:10C77000807FEAD1002300E008232B6008E0072334
:10C78000FBE70623F9E70423F7E70223F5E72C602C
:10C790002B68013300F08A820820FFF771FE2B68B6
:10C7A00020F00F0103F00F0319430820FFF72CFEC0
:10C7B00000244CE734B90820FFF762FEC0F34020A4
:10C7C000286044E7012C40F073820820FFF758FEF0
:10C7D0002B685B0203F4007320F4007119430820F6
:10C7E000FFF712FE002432E734B90820FFF748FEB5
:10C7F000C0F3002028602AE7012C40F05B8208206B
:10C80000FFF73EFE2B681B0203F4807320F4807157
:10C8100019430820FFF7F8FD002418E7012C40F029
:10C820004B820C20FFF72CFE2B68DB0303F4C03394
:10C8300020F4C03119430C20FFF7E6FD002406E781
:10C8400034B90C20FFF71CFEC0F380302860FEE6F0
:10C85000012C40F033820C20FFF712FE2B689B0363
:10C8600003F4804320F4804119430C20FFF7CCFDF2
:10C870000024ECE6D03CFF1F34B90C20FFF700FE8B
:10C88000C0F3C1202860E2E6012C40F019820C20A0
:10C89000FFF7F6FD2B68DB0203F4C05320F4C05110
:10C8A00019430C20FFF7B0FD0024D0E634B90C206A
:10C8B000FFF7E6FDC0F3C3102860C8E6012C40F086
:10C8C00001820C20FFF7DCFD2B68DB0103F4F06331
:10C8D00020F4F06119430C20FFF796FD0024B6E622
:10C8E00034B90C20FFF7CCFDC0F302102860AEE68F
:10C8F000012C40F0E9810C20FFF7C2FD2B681B01E1
:10C9000003F0700320F0700119430C20FFF77CFD49
:10C9100000249CE6012C40F0D9810C20FFF7B0FDEB
:10C920002B6820F00F0103F00F0319430C20FFF7D1
:10C930006BFD00248BE634B90520FFF7A1FDC0F3A1
:10C94000C030286083E6012C40F0C2810D20FFF743
:10C9500097FD2B68DB039BB220F4004119430D20A7
:10C96000FFF752FD002472E634B90520FFF788FD79
:10C97000C0F3413028606AE6012C40F0AB810D2005
:10C98000FFF77EFD2B685B0303F4C04320F4C04136
:10C9900019430D20FFF738FD002458E634B905206F
:10C9A000FFF76EFDC0F30320286050E6012C40F035
:10C9B00093810D20FFF764FD2B681B0203F4706365
:10C9C00020F4706119430D20FFF71EFD00243EE6A0
:10C9D00034B90520FFF754FDC0F34110286036E656
:10C9E000012C40F07B810D20FFF74AFD2B685B0195
:10C9F00003F0600320F0600119430D20FFF704FDF0
:10CA0000002424E6012C40F06B811A68BD4B002401
:10CA10005A731CE634B90620FFF732FDC0F300401C
:10CA2000286014E6012C40F05D810E20FFF728FD00
:10CA30002B681B0403F4803320F4803119430E204B
:10CA4000FFF7E2FC002402E66CB90620FFF718FDB0
:10CA5000000A00F07F0310F0400018BF6FF07F0065
:10CA600018432860F3E5012C40F03E810E20FFF7CB
:10CA700007FD2B681B0203F4FE4320F4FE4119431B
:10CA80000E20FFF7C1FC0024E1E534B90720FFF7D1
:10CA9000F7FCC0F381302860D9E5012C40F02681F5
:10CAA0000F20FFF7EDFC2B689B039BB220F4404165
:10CAB00019430F20FFF7A8FC0024C8E534B907206C
:10CAC000FFF7DEFCC0F301302860C0E5012C40F028
:10CAD0000F810F20FFF7D4FC2B681B0303F4405396
:10CAE00020F4405119430F20FFF78EFC0024AEE5DF
:10CAF000012C40F0FF800F20FFF7C2FC2B689B0247
:10CB000003F4806320F4806119430F20FFF77CFC5D
:10CB100000249CE534B90720FFF7B2FCC0F30120E4
:10CB2000286094E5012C40F0E7800F20FFF7A8FC77
:10CB30002B681B0203F4407320F4407119430F204B
:10CB4000FFF762FC002482E534B90720FFF798FC68
:10CB5000C0F3801028607AE5012C40F0CF800F20D0
:10CB6000FFF78EFC2B689B0103F0400320F040018F
:10CB700019430F20FFF748FC002468E5002C7FF4E0
:10CB800090AD0220FFF77CFCC0F3842028605EE5B6
:10CB90001CB911F041FF286059E5012C40F0B0802C
:10CBA000196811F0D9FE002451E5012C40F0AE8047
:10CBB0001A68544B00241A6149E534B90720FFF77D
:10CBC0005FFCC0F3C010286041E5012C40F0A0805C
:10CBD0000F20FFF755FC2B68DB01DBB220F0800152
:10CBE00019430F20FFF710FC002430E534B904206E
:10CBF000FFF746FCC0F34030286028E5012C40F0E8
:10CC000089800C20FFF73CFC2B685B0303F4005386
:10CC100020F4005119430C20FFF7F6FB002416E521
:10CC2000012C79D10F20FFF72BFC2B681B0403F498
:10CC3000803320F4803119430F20FFF7E5FB0024F7
:10CC400005E5002C7FF42DAD2F4B1B6843B102206E
:10CC5000FFF716FC800A00F4787028600024F6E4E0
:10CC60000120FFF70DFCC0F38920F6E7002C7FF4CC
:10CC700018AD0320FFF704FCC0B22860E7E4012CE4
:10CC80004CD11A681F4B00245A60E0E40024DEE413
:10CC90000024DCE40024DAE40024D8E40024D6E410
:10CCA0000024D4E40024D2E40024D0E41024CEE410
:10CCB0000024CCE40024CAE40024C8E40024C6E430
:10CCC0000024C4E40024C2E40024C0E40024BEE440
:10CCD0000024BCE40024BAE40024B8E40024B6E450
:10CCE0000024B4E40024B2E40024B0E40024AEE460
:10CCF0000024ACE40024AAE40024A8E40024A6E470
:10CD00000024A4E4D03CFF1F6C00FF1F00249EE41D
:10CD100000249CE400249AE4002498E4002496E48F
:10CD200007B5019239B9024601AB0120FFF7BEFBFE
:10CD300003B05DF804FB0820FAE710B4134604467C
:10CD4000084619B9224610BCFFF7B0BB082010BC3A
:10CD5000704710B50C46FFF793FB206010BD70B50F
:10CD60001E4B1F4C1B6822460146002012F08BFA16
:10CD7000002011F03BFD237A1A4A43B3D36E43F0EF
:10CD80000103617A39B343F002030020D36611F046
:10CD90000BFE154D2269697E0028B8BF40429042C3
:10CDA00034BF00260126B14210D090424FF00D0052
:10CDB0002CBF647B247BFFF763FB04F00F0420F09F
:10CDC0000F0121430D20FFF71FFB6E7670BDD36E60
:10CDD00023F00103D5E723F00203D6E71C3DFF1F34
:10CDE000D03CFF1F7431FF1FA415FF1FC2F31300B7
:10CDF000830C10B40B4C05D04314062B04BF02F077
:10CE00001F02E272084B01F077011B6841F0080134
:10CE100003EB81014860A37A13B910BCFFF790BA05
:10CE200010BC7047D03CFF1F1C3DFF1F10B5084BC6
:10CE30009B7A0C4623B90B0702D40846FFF707FB81
:10CE4000044B196804F07F0401EB8404606810BD92
:10CE5000D03CFF1F1C3DFF1F2DE9F8438B0C0C46F7
:10CE60000DD0C1F34243062B09D1294B5A7A21F048
:10CE70001F04002A43D01B7803F01F031C43254FD7
:10CE8000254E264D3B68D6F8008095F81A909B6891
:10CE90000021C4F307409847AA7E336808EB89084D
:10CEA00003EB8203C8F804005A6812025A603B6818
:10CEB00000219B68C4F307209847AB7E326802EBE1
:10CEC00083020121536818433B68000250609B684D
:10CED000E0B298473268A97E02EB81014B681843A3
:10CEE0000011A30C486010610BD0C4F34243072B20
:10CEF00002D1C4F30111A97643F0080302E0DB7A02
:10CF0000BAE7082302EB83035C60BDE8F88300BF47
:10CF1000D03CFF1F183DFF1F1C3DFF1FA415FF1F26
:10CF20002DE9F041444E454BDFF86881444C012720
:10CF300030461F6012F084F9D8F80C506B6803F18A
:10CF40006402E26003F1840203F59270226103F54A
:10CF5000A27203F5017323602B68A260DB68606036
:10CF600098472B68A068DB6898472B68E068DB6807
:10CF700098472B6820691B6998472B682068DB68F5
:10CF80009847D8F810302F4A03F110011160226839
:10CF90005A61052333704FF47A73736011F04AFDC0
:10CFA0002369A2686168002011F094FC264B274990
:10CFB000DA6F0A602649C2F808122649C2F804123C
:10CFC000002151701170244AC3F88820234AC3F805
:10CFD0008420234AC3F88020224AC3F88C20224AA6
:10CFE000C3F8A020214AC3F89C20214AC3F890200E
:10CFF000204AC3F89420204AC3F8B0201F4AC3F83F
:10D00000AC201F4AC3F8BC201E4AC3F8B8201E4AF1
:10D01000C3F8B4201D4AC3F8C820322283F87870C0
:10D020005A6740F225121A670220194AC3F8C02035
:10D03000BDE8F041FFF7E8B8D03CFF1F6C00FF1FD0
:10D04000A415FF1F183DFF1F7431FF1F1C3DFF1F5C
:10D05000FBC10000F3C20000CDC20000F1C200001D
:10D06000EDC20000E9C200003BCD000021CD000070
:10D07000E9C10000AFC200004DC4000053CD000064
:10D080005FCD0000A5C1000099C2000009C20000E8
:10D0900049C20000704C0200014B00225A607047E8
:10D0A0007431FF1F0128F8B514462DD003D3FF2893
:10D0B0003BD00420F8BD136833F003023FD113F0D6
:10D0C000010F204D204E0FD0F3681B681B692869A3
:10D0D0009847246814F002040ED0F3681B681B699B
:10D0E000686998470020F8BDF76828693B68DB68E5
:10D0F00098473B689B69EAE7F66868693368DB68CC
:10D10000984733689B69EBE714680E4D0E4B24B1CA
:10D11000DB681B681B69E868E3E7DE68E86833687A
:10D12000DB68984733689B69F5E7084CE36FD3F8F1
:10D13000043298476369D3F804329847D2E7102045
:10D14000F8BD00BFCC15FF1F704C02007431FF1FEB
:10D1500070B5144E144CF56860682B689B6998474D
:10D160002B6860699B6898472B6820699B68984783
:10D170002B68E0689B6898472B68A0689B68984775
:10D180002B68A0699B6898472B6820689B68984724
:10D190002B6860689B6898473369BDE87040DB691D
:10D1A000184700BF704C0200CC15FF1F2DE9F84353
:10D1B000194C9DF820501E462368894607469B68F7
:10D1C000002140F0800090469847144B83F8E0021D
:10D1D000236800219B6848469847236800219B6884
:10D1E00040469847236800219B683046984723684B
:10D1F00028469B6801219847094B1B6848EA092883
:10D2000007F07F0746EA082603EB870745EA06256D
:10D210007D60BDE8F88300BF203DFF1F283DFF1F54
:10D22000243DFF1F07B5CBB20093C1F30742C1F302
:10D230000723090EFFF7BAFF03B05DF804FBFFF701
:10D24000F1BF10B50F4C104A2368D26819781268E4
:10D250000E4B39B9926958689047236801221A70B9
:10D26000012010BD58685269904704211020FFF733
:10D27000D9FF236800221A70054BDB6FD3F8043204
:10D280009847EDE7243DFF1F704C0200CC15FF1FAF
:10D290007431FF1F10B5064C0649226812F05AFA85
:10D2A00023681B7813B1BDE81040CAE710BD00BF6A
:10D2B000243DFF1F283DFF1F10B50C46002940F0FC
:10D2C0008C8012286BD021D8052859D008D8012885
:10D2D00041D03AD3022841D004283FD0042438E07A
:10D2E0000F2853D007D80E28F8D1002A14BF0221E6
:10D2F000012120202BE010284BD01128EED1930DD6
:10D300009B05002B6BD19100292035E0172858D0C0
:10D3100009D814284CD045D315284CD01628DDD177
:10D3200011462D2013E01A2851D006D818284BD0CA
:10D330001928D3D11146302009E01B284AD0D6281D
:10D34000CCD128491520514301E011463720FFF781
:10D3500069FF204610BD11462120F8E782EAE271FC
:10D36000214BA1EBE271994204DD204911EA22022E
:10D3700038BF1A4611022420FFF754FF0024E8E7C3
:10D38000940DA4055CBB91002820E0E71146252000
:10D39000DDE7940DA40514BB91002A20D7E71146C0
:10D3A0002720D4E7940DA405CCB991002B20CEE71B
:10D3B00011462620CBE7940DA40584B911462C20F4
:10D3C000C5E711462E20C2E711462F20BFE71146C0
:10D3D0003320BCE711463420B9E70824B9E710240C
:10D3E000B7E700BF0071020000127A0000EE85FF6F
:10D3F00070B5254E00F07F04331993F80C32DB072B
:10D4000005D4224B1B6803EB8404606870BD204D7B
:10D410002B6800219B68204698472B6800219B6859
:10D42000084698472B6800219B68084698472B6858
:10D4300000219B68084698472B6801219B680020C3
:10D4400098472B6800219B68204698472B6886F8F0
:10D45000E00200219B68084698472B6800210402DF
:10D460009B68084698472B68002104439B68084640
:10D4700098472B68240204439B68012100209847A9
:10D480002402204370BD00BF283DFF1F243DFF1F25
:10D49000203DFF1F10B50C46FFF7AAFF206010BD0E
:10D4A00038B50D46044668B92020FFF7A1FF40F0CB
:10D4B00004012020FFF7B6FE29463720FFF7B2FE11
:10D4C000204638BD082038BD38B50C460546212019
:10D4D000FFF78EFF2368C11821602846BDE8384059
:10D4E000DEE738B515460C4600296DD111285BD012
:10D4F0001ED8042845D008D801283ED039D30228A8
:10D500003FD003283BD0042440E00E2845D009D862
:10D5100005283DD00828F6D10F20FFF769FF00F05D
:10D52000010032E00F283DD01028ECD12A2030E055
:10D53000172841D00ED814283AD005D8122835D053
:10D540001328E0D12B2024E0152833D01628DAD177
:10D550002D200FE01A2833D005D818282ED01928EE
:10D56000D1D1302006E01B282CD0D628CBD11520D5
:10D5700000E03720FFF73CFF07E02120FAE72220F8
:10D58000F8E72420FFF734FF00122860204638BD5A
:10D590002820FFF72DFF8010F7E72020FFF728FF56
:10D5A0004000F2E72520E5E72920F2E72720E1E720
:10D5B0002620DFE72C20DDE72E20DBE72F20D9E730
:10D5C0003320D7E73420D5E70824DFE710B50C4631
:10D5D000C8B92020FFF70CFF20F004012020FFF73E
:10D5E00021FE84EAE472094BA2EBE4729A4204DD64
:10D5F000074A12EA240438BF1C4621022420FFF700
:10D6000011FE002010BD082010BD00BF00127A00DE
:10D6100000EE85FF0021D9E74942D7E7D6E770B58C
:10D620003F4E4048404C11F0ADFFF5686B6803F584
:10D630008272A26103F55172626103F5597222612F
:10D6400003F5617203F57970E26003F5697203F224
:10D65000044323602B68A260DB68606098472B68F6
:10D660006069DB6898472B682069DB6898472B68FE
:10D67000E068DB6898472B68A068DB6898472B68F0
:10D6800060685B6998472B6860695B6998472B689D
:10D6900020695B6998472B68E0685B6998472B684D
:10D6A000A0685B6998472B68A0691B6998472B683D
:10D6B00020681B691D4C98471D4B32691A606B68C6
:10D6C00003F5317353601B4B62691A6001212020FE
:10D6D000FFF7A8FD6369184AC3F8042200225A70B4
:10D6E00001221A70154B2362154BE361154BA361A0
:10D6F000154B6362154BA363154B6363154BA36214
:10D70000154BE362154BA364154B6364154B6365BE
:10D71000154B2365154BE3652274154BA36570BD4E
:10D72000704C0200283DFF1FCC15FF1F7431FF1FF6
:10D73000203DFF1F243DFF1F43D20000CDD5000038
:10D740001DD6000019D6000015D60000E3D4000055
:10D75000B9D20000A1D40000C9D400003FD200001B
:10D7600095D4000095D20000A5D0000099D000000B
:10D7700051D10000014B00225A6070477431FF1FE5
:10D780000128F8B514462DD003D3FF283BD0042040
:10D79000F8BD136833F003023FD113F0010F204DA1
:10D7A000204E0FD0F3681B681B69286998472468CE
:10D7B00014F002040ED0F3681B681B69686998476F
:10D7C0000020F8BDF76828693B68DB6898473B682C
:10D7D0009B69EAE7F66868693368DB6898473368ED
:10D7E0009B69EBE714680E4D0E4B24B1DB681B6898
:10D7F0001B69E868E3E7DE68E8683368DB68984738
:10D8000033689B69F5E7084CE36FD3F80432984717
:10D810006369D3F804329847D2E71020F8BD00BFFF
:10D82000F815FF1F704C02007431FF1F70B5164EC3
:10D83000164CF56860682B689B6998472B6860698F
:10D840009B6898472B6820699B6898472B68E0681D
:10D850009B6898472B68A0689B6898472B68E0698D
:10D860009B6898472B68A0699B6898472B6820683D
:10D870009B6898472B6860689B6898473369BDE848
:10D880007040DB69184700BF704C0200F815FF1F9D
:10D8900038B50A4B0A4CDD6860682B689B6998476D
:10D8A00001200DF0B5FF2B6860685B699847054B58
:10D8B000186811F0B1FF012038BD00BF704C0200A4
:10D8C000F815FF1F0C40FF1F38B50A4B0A4CDD68E6
:10D8D00060682B689B69984701200DF099FF2B68C1
:10D8E00060685B699847054B186811F08CFF012050
:10D8F00038BD00BF704C0200F815FF1F0C40FF1F21
:10D900002DE9F843194D9DF820909DF82440984644
:10D910002B680E469B68002146F08000174698470A
:10D92000134B83F8E0022B6800219B683846984728
:10D930002B6800219B68404698472B6800219B6814
:10D94000484698472B6801219B6820469847094B19
:10D950001B6806F07F0644EA092203EB860642EACA
:10D96000084242EA07627260BDE8F8831040FF1F78
:10D970001440FF1F0C40FF1F07B5D3B20193C2F341
:10D9800007230093C2F30743120EFFF7B9FF03B05A
:10D990005DF804FB70B5174C174A23681D780146E3
:10D9A000002011F0E5FF1DB323681A7802BB134C69
:10D9B00094F86830012B19D0032B0BBF00222822CA
:10D9C0000D230F2343F0884343F0401343EA4232D0
:10D9D00004210020FFF7D0FFE36F012D0CBFD3F827
:10D9E0000432D3F80832BDE8704018470B23E9E74A
:10D9F00070BD00BF0C40FF1F1440FF1F7431FF1F9C
:10DA00000A4601460020FFF7B7BF38B514460D4659
:10DA1000002940F08280122868D021D8052857D0EC
:10DA200008D801283FD038D302283ED004283CD063
:10DA3000042536E00F2851D007D80E28F8D1002A47
:10DA400014BF02220122202128E0102848D01128EA
:10DA5000EED1930D9B05002B61D19200292132E07C
:10DA6000172852D008D8142848D041D3152847D0B9
:10DA70001628DDD12D2111E01A284AD005D8182802
:10DA800045D01928D4D1302108E01B2843D0D6280E
:10DA9000CED1244A1521624300E037212846FFF702
:10DAA0006BFF284638BD2121F8E784EAE4721E4B5B
:10DAB000A2EBE4729A4204DD1C4A12EA240438BF45
:10DAC0001C46220224210020FFF756FF0025E8E72C
:10DAD000950DAD051DBB92002821DFE72521DDE76F
:10DAE000950DAD05DDB992002A21D7E72721D5E7AD
:10DAF000950DAD059DB992002B21CFE72621CDE7ED
:10DB0000950DAD055DB92C21C8E72E21C6E72F2163
:10DB1000C4E73321C2E73421C0E70825C1E7102557
:10DB2000BFE700BF0071020000127A0000EE85FF1F
:10DB300070B5254E01F07F04331993F80C32DB07E2
:10DB400005D4224B1B6803EB8404606870BD204D34
:10DB50002B6800219B68204698472B6800219B6812
:10DB6000084698472B6800219B68084698472B6811
:10DB700000219B68084698472B6801219B6800207C
:10DB800098472B6800219B68204698472B6886F8A9
:10DB9000E00200219B68084698472B680021040298
:10DBA0009B68084698472B68002104439B680846F9
:10DBB00098472B68240204439B6801210020984762
:10DBC0002402204370BD00BF1440FF1F0C40FF1F04
:10DBD0001040FF1F10B50C4601460020FFF7A8FFBC
:10DBE000206010BD38B50D46044678B92021FFF7F6
:10DBF0009FFF202140F004022046FFF7BDFE204693
:10DC00002A463721FFF7B8FE204638BD082038BD28
:10DC100038B50C4621210546FFF78AFF21680144EB
:10DC200021602846BDE83840DCE738B515460C468B
:10DC3000002976D1112864D01FD8042847D008D8ED
:10DC4000012840D03AD3022841D003283DD00424F3
:10DC500043E00E2849D00AD8052840D00828F6D13C
:10DC60000F212046FFF764FF00F0010034E00F2889
:10DC700045D01028EBD12A2132E0172849D00ED800
:10DC8000142842D005D812283DD01328DFD12B21EB
:10DC900026E015283BD01628D9D12D210FE01A28CF
:10DCA0003BD005D8182836D01928D0D1302106E02D
:10DCB0001B2834D0D628CAD1152100E037212046B0
:10DCC000FFF736FF08E02121F9E72221F7E72421B9
:10DCD0002046FFF72DFF00122860204638BD28217E
:10DCE0002046FFF725FF8010F6E720212046FFF7AA
:10DCF0001FFF00F00300831E58425841ECE7252126
:10DD0000DDE72921ECE72721D9E72621D7E72C21D8
:10DD1000D5E72E21D3E72F21D1E73321CFE73421D7
:10DD2000CDE70824D9E738B50C460546D8B92021F7
:10DD3000FFF7FEFE202120F004022846FFF71CFE1C
:10DD400084EAE472094BA2EBE4729A4204DD084AC9
:10DD500012EA240438BF1C46220224210020FFF7C7
:10DD60000BFE002038BD082038BD00BF00127A002D
:10DD700000EE85FF0021D6E74942D4E7D3E7F8B5A6
:10DD8000314C256A666A2A023302C6B243EA156339
:10DD90000027324394F82800666B3B43276B013021
:10DDA000350E360246EA1766C0B23F02C4E90823C0
:10DDB00084F8280066632763002943D0042804D927
:10DDC0001A466D210020FFF7D7FD226A6C21002042
:10DDD000FFF7D2FD01200DF01BFD226A6C2100200F
:10DDE000FFF7CAFD01200DF013FD00230022C4E956
:10DDF0000C2394F82830042B0AD96F210020FFF758
:10DE000097FED4E90C23002632430343C4E90C23D4
:10DE10006E210020FFF78CFED4E90C6794F82820CF
:10DE20000346C2F10802D20047EAE371304315F01D
:10DE3000E5FC00230022C4E90C01C4E90823002307
:10DE400084F828302846F8BDF815FF1F70B5464EF7
:10DE50004648474C11F090FCF5686B6803F1E4020A
:10DE6000E26103F58272A26103F55172626103F50A
:10DE70005972226103F5617203F57970E26003F56E
:10DE8000697203F2044323602B68A260DB68606060
:10DE900098472B686069DB6898472B682069DB68C6
:10DEA00098472B68E068DB6898472B68A068DB68B8
:10DEB00098472B6860685B6998472B6860695B6965
:10DEC00098472B6820695B6998472B68E0685B6915
:10DED00098472B68A0685B6998472B68E0691B69C5
:10DEE00098472B68A0691B6998472B6820681B69B5
:10DEF000204C9847204B32691A606B6803F53173E8
:10DF000053601E4B62691A60202101220020FFF736
:10DF100033FD6369002159701949C3F804120122C5
:10DF200018491A70C3F80812174B6366174B23621F
:10DF3000174BE361174BA361174B6362174BA36346
:10DF4000174B6363174BA362174BE362174BA36432
:10DF5000174B6364174B6365174B2365174BE365DA
:10DF60002274174BA36570BD704C02001440FF1F54
:10DF7000F815FF1F7431FF1F1040FF1F0C40FF1FDB
:10DF8000C9D8000091D800007FDD000027DD000027
:10DF90007DDD000079DD000075DD00002BDC000078
:10DFA0000BDA0000E5DB000011DC000001DA000004
:10DFB000D5DB000095D9000081D7000075D700009F
:10DFC0002DD80000014B00225A6070477431FF1FAA
:10DFD00070B5184E184CF56860682B689B699847B7
:10DFE0002B68A0699B6898472B6860699B68984775
:10DFF0002B6820699B6898472B68E0689B68984766
:10E000002B68A0689B6898472B68206A9B68984794
:10E010002B68E0699B6898472B6820689B68984745
:10E020002B6860689B6898473369BDE87040DB697E
:10E03000184700BF704C02004016FF1F0228F8B5B9
:10E04000144652D004D888B101283CD0042438E0CA
:10E0500003285CD0FF28F9D1314CE36FD3F80432A8
:10E0600098476369D3F80432984703E0136833F0A4
:10E07000030201D0002424E013F0010F294D2A4EA1
:10E080000ED0F3681B681B6968699847246814F010
:10E0900002040DD0F368A8691B681B699847E9E77B
:10E0A000F76868693B68DB6898473B689B69EBE702
:10E0B000F668A8693368DB6898473368A8699B6984
:10E0C00098472046F8BD1468164D174B24B1DB68FD
:10E0D00028691B681B69E1E7DE6828693368DB682B
:10E0E0009847336828699B69EAE714680D4D0E4B21
:10E0F00024B1DB68A8681B681B69CFE7DE68A868E5
:10E100003368DB6898473368A8689B69D8E70120C3
:10E1100011F0BCFC20600028ACD12024D1E700BF66
:10E120007431FF1F4016FF1F704C020038B50A4BB8
:10E130000A4CDD6860682B689B69984701200DF0E8
:10E1400067FB2B6860685B699847054B186811F09E
:10E1500072FC012038BD00BF704C02004016FF1F4A
:10E16000F842FF1F38B50A4B0A4CDD6860682B681F
:10E170009B69984701200DF04BFB2B6860685B6939
:10E180009847054B186811F04DFC012038BD00BFC1
:10E19000704C02004016FF1FF842FF1F2DE9F843A4
:10E1A000194D9DF8204099462B680F4606469B68FE
:10E1B000002140F0800090469847144B83F8E0021D
:10E1C0002B6800219B68384698472B6800219B6884
:10E1D000404698472B6800219B68484698472B6823
:10E1E00001219B6820469847094B1B6806F07F0673
:10E1F00044EA092103EB860641EA084141EA076146
:10E200007160BDE8F88300BFFC42FF1F0043FF1FA1
:10E21000F842FF1F07B5CBB20093C1F30742C1F329
:10E220000723090EFFF7BAFF03B05DF804FB70B5D2
:10E23000154C16492268157811F094FC15B3236823
:10E240001978F9B9124C94F86830012B18D0032BC7
:10E250000BBF002128210D230F2343F0884343F0F7
:10E26000401343EA41310420FFF7D4FFE36F012D4F
:10E270000CBFD3F80432D3F80832BDE87040184719
:10E280000B23EAE770BD00BFF842FF1F0043FF1FEA
:10E290007431FF1FFFF7BEBF70B5254E00F07F043D
:10E2A000331993F80C32DB0705D4224B1B6803EBC0
:10E2B0008404606870BD204D2B6800219B68204657
:10E2C00098472B6800219B68084698472B680021D7
:10E2D0009B68084698472B6800219B68084698472A
:10E2E0002B6801219B68002098472B6800219B68C0
:10E2F000204698472B6886F8E00200219B68084674
:10E3000098472B68002104029B68084698472B68B1
:10E31000002104439B68084698472B682402044365
:10E320009B680121002098472402204370BD00BF54
:10E330000043FF1FF842FF1FFC42FF1F10B50C46B1
:10E34000FFF7AAFF206010BD38B50D46044668B936
:10E350002020FFF7A1FF40F004012020FFF75AFF23
:10E3600029463720FFF756FF204638BD082038BD24
:10E3700038B50C4605462120FFF78EFF2368C118EB
:10E3800021602846BDE83840DEE76F2970B50446B5
:10E39000154600F00A827ED8122900F0828144D806
:10E3A000052900F0398125D8022900F0118107D80C
:10E3B000002900F0F580012900F002810424F8E032
:10E3C000032900F022810429F8D1002800F00181FE
:10E3D000012840F0ED801168B64B81EAE172A2EBB2
:10E3E000E1729A4240F30E81B34A33EA210128BF19
:10E3F000114607E10F2900F033810CD8082900F0FD
:10E400001E810E29DAD1002840F021812020FFF75B
:10E4100043FF4000C8E0102900F02A811129CDD126
:10E42000002840F033812920F8E0182900F07A8193
:10E4300017D8152900F0598109D8132900F0408117
:10E440001429BBD1002840F04A812620AAE01629D1
:10E4500000F059811729B1D1002840F05D812E20AC
:10E46000A0E01B2900F0768109D8192900F063810A
:10E470001A29A3D1002840F06781332092E06D294A
:10E4800000F0778100F27E816C2997D1002840F05E
:10E490006A81602086E07D2900F020823CD87529C1
:10E4A00000F0D2811ED8722900F0A7810CD8702903
:10E4B00000F08E81712981D1002C40F092810620DC
:10E4C000FFF7EAFEC0B288E0732900F0AA81742940
:10E4D0007FF474AF002840F0B181784B1B68D3F80B
:10E4E0007031A3E1782900F0E1810AD8762900F0A3
:10E4F000C38177297FF462AF002840F0D1815E208C
:10E5000050E0792900F0DB817C297FF457AF0028A7
:10E5100040F0DE815C2045E0882900F01A8220D896
:10E52000842900F0FF8111D87E2900F0E081812943
:10E530007FF444AF01283BD11668002E00F0EB8138
:10E5400011F0A4FA286098BB202432E0852900F05D
:10E55000EE8186297FF432AF002840F0F48152200A
:10E5600020E0C829A8D00DD8892900F007828A297F
:10E570007FF424AF002840F01782504B1B6893F8BB
:10E58000923153E1D42900F02382D62900F02B8266
:10E59000D1297FF413AF002840F01482502001E00D
:10E5A00020B93720FFF778FE286002E0012802D06A
:10E5B0000024204670BD11683720FFF72BFEF7E7D7
:10E5C00008B92120EEE70128F2D111682120F4E7F3
:10E5D00028B92420FFF760FE00122860E8E7012830
:10E5E000E6D11168334B81EAE172A2EBE1729A4203
:10E5F00008DDA3F574032F4AA3F5105332EA210175
:10E6000028BF194609022420D7E708B92220C9E704
:10E61000012C3FF4D3AECBE720B92820FFF73CFE16
:10E620008010C1E70128C3D111688C0DA405002C0E
:10E6300040F0E48189002820FFF7ECFDB9E70028CD
:10E64000E6D10F20FFF728FE00F00100ACE701281B
:10E65000AED11368002B0CBF012102212020ACE7B2
:10E6600008B925209EE70128A2D111682520A4E73A
:10E6700008B92A20D2E701289AD111688C0DA40587
:10E68000002C40F0BB8189002A20D5E701288FD1DA
:10E6900011688C0DA405002C40F0B0818900292060
:10E6A000CAE708B927207DE7012881D11168272012
:10E6B00083E700BF00127A0000EE85FFF842FF1FDB
:10E6C00008B92B20AAE701287FF472AF11688C0DDE
:10E6D000A405002C40F0928189002B20ACE7012892
:10E6E0007FF466AF1168262067E708B92C2059E748
:10E6F00001287FF45DAF11688B0D9B05002B40F066
:10E700007D812C2059E708B92D204BE701287FF4A3
:10E710004FAF11682D2050E701287FF449AF1168F1
:10E720002E204AE708B92F203CE701287FF440AFAC
:10E7300011682F2041E708B9302033E701287FF422
:10E7400037AF1168302038E701287FF431AF116806
:10E75000332032E708B9342024E701287FF428AFBA
:10E760001168342029E701287FF422AF1168602066
:10E7700023E708B9612015E701287FF419AF116874
:10E7800061201AE720B91C20FFF786FD00140BE773
:10E7900001287FF40DAF1C20FFF77EFD2968C0F330
:10E7A000080040EA01411C2007E720B91C20FFF7C0
:10E7B00073FDC0B2F8E601287FF4FAAE1C20FFF723
:10E7C0006BFD2B6800F47F01C3F308031943EAE7EC
:10E7D00008B95920E6E601287FF4EAAE116859200D
:10E7E000EBE6012C7FF4E4AE0620FFF755FD297817
:10E7F00020F0FF0001430620DFE628B90620FFF7DE
:10E800004BFDC0F30720CFE601287FF4D1AE0620F0
:10E81000FFF742FD2B681B0220F47F419BB2194396
:10E82000E9E728B9764B1B68D3F86C312B60C0E65A
:10E8300001287FF4BDAE11685A20BEE601287FF49E
:10E84000B7AE11685B20B8E630B96D4B1B68D3F8E2
:10E850007031C3F30E03E9E701287FF4A9AE684BDA
:10E8600011681B68D3F8703123F4FF4323F07F0352
:10E87000C1F30E011943E5E720B9614B1B6893F81A
:10E880007231D3E701287FF493AE5D4B1B68D3F858
:10E89000701113681B0421F47F0103F47F03E9E77F
:10E8A00001287FF485AE11685E2086E608B918203D
:10E8B00078E601287FF47CAE116818207DE608B95F
:10E8C00019206FE601287FF473AE1168192074E6F1
:10E8D00001287FF46DAE11685C206EE608B95F20F8
:10E8E00060E601287FF464AE11685F2065E628B910
:10E8F0000620FFF7D1FCC0F3074055E601287FF45E
:10E9000057AE0620FFF7C8FC2B681B0420F47F01DC
:10E9100003F47F0383E70720FFF7BEFC20F48001A8
:10E9200007204AE600287FF473AE65203AE6002807
:10E930007FF43EAE0720FFF7AFFCC0F38150431ECB
:10E940005842584130E601287FF432AE1168522017
:10E9500033E620B92A4B1B6893F8903166E701280B
:10E960007FF426AE264B11681B68D3F8903101F076
:10E970000F0123F0FF03194363201EE630B9204B3B
:10E980001B68D3F89031C3F303234FE701287FF4CA
:10E990000FAE1B4B1B68D3F8901113681B0221F4B8
:10E9A000706103F47063E6E701287FF401AE144B55
:10E9B0001B68D3F8901113681B0421F47F0103F442
:10E9C0007F03D8E701287FF4F3AD11685020F4E508
:10E9D00018B90B4B1B68DB6928E701287FF4E8AD09
:10E9E00011685320E9E508B91520DBE501287FF41B
:10E9F000DFAD1368034915205943DEE51024D8E53F
:10EA0000F842FF1F0071020007B5019239B90146B3
:10EA100001AA0120FFF7B9FC03B05DF804FB082050
:10EA2000FAE70B4611B901461846AEE408207047D4
:10EA300010B50C46C8B92020FFF72EFC20F00401C9
:10EA40002020FFF7E7FB84EAE472094BA2EBE472B3
:10EA50009A4204DD074A12EA240438BF1C46210208
:10EA60002420FFF7D7FB002010BD082010BD00BFF9
:10EA700000127A0000EE85FF0021D9E74942D7E76E
:10EA8000D6E7F8B52F4CA56AE66A2A023302C6B269
:10EA900043EA15630027324394F83000E66B3B43AA
:10EAA000A76B0130350E360246EA1766C0B23F0248
:10EAB000C4E90A2384F83000E663A76300293ED046
:10EAC000042803D919466D20FFF7A4FBA16A6C2026
:10EAD000FFF7A0FB01200CF09BFEA16A6C20FFF762
:10EAE00099FB01200CF094FE00230022C4E90E23C0
:10EAF00094F83030042B09D96F20FFF7CDFBD4E90F
:10EB00000E23002632430343C4E90E236E20FFF791
:10EB1000C3FBD4E90E6794F830200346C2F1080223
:10EB2000D20047EAE371304314F068FE002300226C
:10EB3000C4E90E01C4E90A23002384F830302846D2
:10EB4000F8BD00BF4016FF1F70B54B4E4B484C4CF4
:10EB500010F020FFF5686B6803F1E402226203F510
:10EB60008272E26103F55172A26103F5597262612A
:10EB700003F56172226103F5697203F57970E26051
:10EB800003F5717203F2044323602B68A260DB6813
:10EB9000606098472B68A069DB6898472B686069BC
:10EBA000DB6898472B682069DB6898472B68E0682A
:10EBB000DB6898472B68A068DB6898472B6860681B
:10EBC0005B6998472B68A0695B6998472B68606907
:10EBD0005B6998472B6820695B6998472B68E068F8
:10EBE0005B6998472B68A0685B6998472B68206A27
:10EBF0001B6998472B68E0691B6998472B68206858
:10EC00001B69204C9847204B32691A606B6803F5EA
:10EC1000317353601D4B62691A6001212020FFF798
:10EC2000F9FA6369002159701949C3F804120122E5
:10EC300018491A70C3F80812174B6366174B236202
:10EC4000174BE361174BA361174B6362174BA36329
:10EC5000174B6363174BA362174BE362174BA36415
:10EC6000174B6364174B6365174B2365174BE365BD
:10EC70002274174BA36570BD704C02000043FF1F48
:10EC80004016FF1F7431FF1FFC42FF1FF842FF1F99
:10EC900065E100002DE1000083EA000031EA000098
:10ECA00081EA00007DEA000079EA000023EA000022
:10ECB00009EA000049E3000071E3000095E200006A
:10ECC0003DE300002FE200003DE00000C5DF000052
:10ECD000D1DF0000014B00225A6070477431FF1FE2
:10ECE00070B5184E184CF56860682B689B6998479A
:10ECF0002B68A0699B6898472B6860699B68984758
:10ED00002B6820699B6898472B68E0689B68984748
:10ED10002B68A0689B6898472B68206A9B68984777
:10ED20002B68E0699B6898472B6820689B68984728
:10ED30002B6860689B6898473369BDE87040DB6961
:10ED4000184700BF704C02009016FF1F0228F8B54C
:10ED5000144652D004D888B101283CD0042438E0AD
:10ED600003285CD0FF28F9D1314CE36FD3F804328B
:10ED700098476369D3F80432984703E0136833F087
:10ED8000030201D0002424E013F0010F294D2A4E84
:10ED90000ED0F3681B681B6968699847246814F0F3
:10EDA00002040DD0F368A8691B681B699847E9E75E
:10EDB000F76868693B68DB6898473B689B69EBE7E5
:10EDC000F668A8693368DB6898473368A8699B6967
:10EDD00098472046F8BD1468164D174B24B1DB68E0
:10EDE00028691B681B69E1E7DE6828693368DB680E
:10EDF0009847336828699B69EAE714680D4D0E4B04
:10EE000024B1DB68A8681B681B69CFE7DE68A868C7
:10EE10003368DB6898473368A8689B69D8E70120A6
:10EE200010F02EFF20600028ACD12024D1E700BFD5
:10EE30007431FF1F9016FF1F704C020038B50A4B4B
:10EE40000A4CDD6860682B689B69984701200CF0CC
:10EE5000DFFC2B6860685B699847054B186810F009
:10EE6000E4FE012038BD00BF704C02009016FF1F69
:10EE7000CC48FF1F38B50A4B0A4CDD6860682B6828
:10EE80009B69984701200CF0C3FC2B6860685B69A4
:10EE90009847054B186810F0BFFE012038BD00BF31
:10EEA000704C02009016FF1FCC48FF1F2DE9F8435D
:10EEB000194D9DF8204099462B680F4606469B68E1
:10EEC000002140F0800090469847144B83F8E00200
:10EED0002B6800219B68384698472B6800219B6867
:10EEE000404698472B6800219B68484698472B6806
:10EEF00001219B6820469847094B1B6806F07F0656
:10EF000044EA092103EB860641EA084141EA076128
:10EF10007160BDE8F88300BFC848FF1FE445FF1FCC
:10EF2000CC48FF1F07B5CBB20093C1F30742C1F332
:10EF30000723090EFFF7BAFF03B05DF804FB70B5B5
:10EF4000154C16492268157810F006FF15B3236892
:10EF50001978F9B9124C94F86830012B18D0032BAA
:10EF60000BBF002128210D230F2343F0884343F0DA
:10EF7000401343EA41310420FFF7D4FFE36F012D32
:10EF80000CBFD3F80432D3F80832BDE870401847FC
:10EF90000B23EAE770BD00BFCC48FF1FE445FF1F0D
:10EFA0007431FF1FFFF7BEBF70B5254E00F07F0420
:10EFB000331993F80C32DB0705D4224B1B6803EBA3
:10EFC0008404606870BD204D2B6800219B6820463A
:10EFD00098472B6800219B68084698472B680021BA
:10EFE0009B68084698472B6800219B68084698470D
:10EFF0002B6801219B68002098472B6800219B68A3
:10F00000204698472B6886F8E00200219B68084656
:10F0100098472B68002104029B68084698472B6894
:10F02000002104439B68084698472B682402044348
:10F030009B680121002098472402204370BD00BF37
:10F04000E445FF1FCC48FF1FC848FF1F10B50C4602
:10F05000FFF7AAFF206010BD38B50D46044668B919
:10F060002020FFF7A1FF40F004012020FFF75AFF06
:10F0700029463720FFF756FF204638BD082038BD07
:10F0800038B50C4605462120FFF78EFF2368C118CE
:10F0900021602846BDE83840DEE76F2970B5044698
:10F0A000154600F00A827ED8122900F0828144D8E9
:10F0B000052900F0398125D8022900F0118107D8EF
:10F0C000002900F0F580012900F002810424F8E015
:10F0D000032900F022810429F8D1002800F00181E1
:10F0E000012840F0ED801168B64B81EAE172A2EB95
:10F0F000E1729A4240F30E81B34A33EA210128BFFC
:10F10000114607E10F2900F033810CD8082900F0DF
:10F110001E810E29DAD1002840F021812020FFF73E
:10F1200043FF4000C8E0102900F02A811129CDD109
:10F13000002840F033812920F8E0182900F07A8176
:10F1400017D8152900F0598109D8132900F04081FA
:10F150001429BBD1002840F04A812620AAE01629B4
:10F1600000F059811729B1D1002840F05D812E208F
:10F17000A0E01B2900F0768109D8192900F06381ED
:10F180001A29A3D1002840F06781332092E06D292D
:10F1900000F0778100F27E816C2997D1002840F041
:10F1A0006A81602086E07D2900F020823CD87529A4
:10F1B00000F0D2811ED8722900F0A7810CD87029E6
:10F1C00000F08E81712981D1002C40F092810620BF
:10F1D000FFF7EAFEC0B288E0732900F0AA81742923
:10F1E0007FF474AF002840F0B181784B1B68D3F8EE
:10F1F0007031A3E1782900F0E1810AD8762900F086
:10F20000C38177297FF462AF002840F0D1815E206E
:10F2100050E0792900F0DB817C297FF457AF00288A
:10F2200040F0DE815C2045E0882900F01A8220D879
:10F23000842900F0FF8111D87E2900F0E081812926
:10F240007FF444AF01283BD11668002E00F0EB811B
:10F2500010F016FD286098BB202432E0852900F0CC
:10F26000EE8186297FF432AF002840F0F4815220ED
:10F2700020E0C829A8D00DD8892900F007828A2962
:10F280007FF424AF002840F01782504B1B6893F89E
:10F29000923153E1D42900F02382D62900F02B8249
:10F2A000D1297FF413AF002840F01482502001E0F0
:10F2B00020B93720FFF778FE286002E0012802D04D
:10F2C0000024204670BD11683720FFF72BFEF7E7BA
:10F2D00008B92120EEE70128F2D111682120F4E7D6
:10F2E00028B92420FFF760FE00122860E8E7012813
:10F2F000E6D11168334B81EAE172A2EBE1729A42E6
:10F3000008DDA3F574032F4AA3F5105332EA210157
:10F3100028BF194609022420D7E708B92220C9E7E7
:10F32000012C3FF4D3AECBE720B92820FFF73CFEF9
:10F330008010C1E70128C3D111688C0DA405002CF1
:10F3400040F0E48189002820FFF7ECFDB9E70028B0
:10F35000E6D10F20FFF728FE00F00100ACE70128FE
:10F36000AED11368002B0CBF012102212020ACE795
:10F3700008B925209EE70128A2D111682520A4E71D
:10F3800008B92A20D2E701289AD111688C0DA4056A
:10F39000002C40F0BB8189002A20D5E701288FD1BD
:10F3A00011688C0DA405002C40F0B0818900292043
:10F3B000CAE708B927207DE7012881D111682720F5
:10F3C00083E700BF00127A0000EE85FFCC48FF1FE4
:10F3D00008B92B20AAE701287FF472AF11688C0DC1
:10F3E000A405002C40F0928189002B20ACE7012875
:10F3F0007FF466AF1168262067E708B92C2059E72B
:10F4000001287FF45DAF11688B0D9B05002B40F048
:10F410007D812C2059E708B92D204BE701287FF486
:10F420004FAF11682D2050E701287FF449AF1168D4
:10F430002E204AE708B92F203CE701287FF440AF8F
:10F4400011682F2041E708B9302033E701287FF405
:10F4500037AF1168302038E701287FF431AF1168E9
:10F46000332032E708B9342024E701287FF428AF9D
:10F470001168342029E701287FF422AF1168602049
:10F4800023E708B9612015E701287FF419AF116857
:10F4900061201AE720B91C20FFF786FD00140BE756
:10F4A00001287FF40DAF1C20FFF77EFD2968C0F313
:10F4B000080040EA01411C2007E720B91C20FFF7A3
:10F4C00073FDC0B2F8E601287FF4FAAE1C20FFF706
:10F4D0006BFD2B6800F47F01C3F308031943EAE7CF
:10F4E00008B95920E6E601287FF4EAAE11685920F0
:10F4F000EBE6012C7FF4E4AE0620FFF755FD2978FA
:10F5000020F0FF0001430620DFE628B90620FFF7C0
:10F510004BFDC0F30720CFE601287FF4D1AE0620D3
:10F52000FFF742FD2B681B0220F47F419BB2194379
:10F53000E9E728B9764B1B68D3F86C312B60C0E63D
:10F5400001287FF4BDAE11685A20BEE601287FF481
:10F55000B7AE11685B20B8E630B96D4B1B68D3F8C5
:10F560007031C3F30E03E9E701287FF4A9AE684BBD
:10F5700011681B68D3F8703123F4FF4323F07F0335
:10F58000C1F30E011943E5E720B9614B1B6893F8FD
:10F590007231D3E701287FF493AE5D4B1B68D3F83B
:10F5A000701113681B0421F47F0103F47F03E9E762
:10F5B00001287FF485AE11685E2086E608B9182020
:10F5C00078E601287FF47CAE116818207DE608B942
:10F5D00019206FE601287FF473AE1168192074E6D4
:10F5E00001287FF46DAE11685C206EE608B95F20DB
:10F5F00060E601287FF464AE11685F2065E628B9F3
:10F600000620FFF7D1FCC0F3074055E601287FF440
:10F6100057AE0620FFF7C8FC2B681B0420F47F01BF
:10F6200003F47F0383E70720FFF7BEFC20F480018B
:10F6300007204AE600287FF473AE65203AE60028EA
:10F640007FF43EAE0720FFF7AFFCC0F38150431EAE
:10F650005842584130E601287FF432AE11685220FA
:10F6600033E620B92A4B1B6893F8903166E70128EE
:10F670007FF426AE264B11681B68D3F8903101F059
:10F680000F0123F0FF03194363201EE630B9204B1E
:10F690001B68D3F89031C3F303234FE701287FF4AD
:10F6A0000FAE1B4B1B68D3F8901113681B0221F49B
:10F6B000706103F47063E6E701287FF401AE144B38
:10F6C0001B68D3F8901113681B0421F47F0103F425
:10F6D0007F03D8E701287FF4F3AD11685020F4E5EB
:10F6E00018B90B4B1B68DB6928E701287FF4E8ADEC
:10F6F00011685320E9E508B91520DBE501287FF4FE
:10F70000DFAD1368034915205943DEE51024D8E521
:10F71000CC48FF1F0071020007B5019239B90146BC
:10F7200001AA0120FFF7B9FC03B05DF804FB082033
:10F73000FAE70B4611B901461846AEE408207047B7
:10F7400010B50C46C8B92020FFF72EFC20F00401AC
:10F750002020FFF7E7FB84EAE472094BA2EBE47296
:10F760009A4204DD074A12EA240438BF1C462102EB
:10F770002420FFF7D7FB002010BD082010BD00BFDC
:10F7800000127A0000EE85FF0021D9E74942D7E751
:10F79000D6E7F8B52D4CA56AE66A2A023302C6B24E
:10F7A00043EA15630027324394F83000E66B3B438D
:10F7B000A76B0130350E360246EA1766C0B23F022B
:10F7C000C4E90A2384F83000E663A76300293BD02C
:10F7D000042803D919466D20FFF7A4FBA16A6C2009
:10F7E000FFF7A0FB01200CF013F8A16A6C20FFF7D3
:10F7F00099FB00230022C4E90E2394F83030042B37
:10F8000009D96F20FFF7D0FBD4E90E23002632433D
:10F810000343C4E90E236E20FFF7C6FBD4E90E674D
:10F8200094F830200346C2F10802D20047EAE3719F
:10F83000304313F0E3FF00230022C4E90E01C4E9C2
:10F840000A23002384F830302846F8BD9016FF1FA5
:10F8500070B54B4E4B484C4C10F096F9F5686B6800
:10F8600003F1E402226203F58272E26103F5517250
:10F87000A26103F55972626103F56172226103F5B9
:10F88000697203F57970E26003F5717203F2044363
:10F8900023602B68A260DB68606098472B68A069D2
:10F8A000DB6898472B686069DB6898472B6820699C
:10F8B000DB6898472B68E068DB6898472B68A0688E
:10F8C000DB6898472B6860685B6998472B68A0697C
:10F8D0005B6998472B6860695B6998472B6820696A
:10F8E0005B6998472B68E0685B6998472B68A0685C
:10F8F0005B6998472B68206A1B6998472B68E06909
:10F900001B6998472B6820681B69204C9847204B3F
:10F9100032691A606B6803F5317353601D4B62697D
:10F920001A6001212020FFF7FDFA63690021597058
:10F930001949C3F80412012218491A70C3F80812B1
:10F94000174B6366174B2362174BE361174BA36199
:10F95000174B6362174BA363174B6363174BA36289
:10F96000174BE362174BA364174B6364174B636534
:10F97000174B2365174BE3652274174BA36570BDC6
:10F98000704C0200E445FF1F9016FF1F7431FF1FEB
:10F99000C848FF1FCC48FF1F75EE00003DEE000079
:10F9A00093F7000041F7000091F700008DF7000089
:10F9B00089F7000033F7000019F7000059F0000044
:10F9C00081F00000A5EF00004DF000003FEF0000C7
:10F9D0004DED0000D5EC0000E1EC00000020704788
:10F9E00001207047014B00225A6070477431FF1F9D
:10F9F00010B50C460CF080FB206010BD0CF0A8BBCD
:10FA000038B50D46044620B910F071FA286020463A
:10FA100038BD082038BDF0B589B004AC364D074676
:10FA200010220021204615F041F82B68FB1A092B03
:10FA300006D9AA682F60642353436B600023AB6030
:10FA4000AB680133AB602D4BA3F1080633F8081CFB
:10FA5000727A0291B11D0191B1880091002039465E
:10FA600010F05EFB0FF02CF920B100221146104679
:10FA70000FF0B2F90FF01EF998B10FF09BF90328BF
:10FA80000FD8DFE800F018100222002010F052FA20
:10FA90000490002010F055FA059094E80F000FF044
:10FAA00029F909B0F0BD002010F015FA04900020EB
:10FAB00010F01DFAF0E77189002010F0A4F97189A7
:10FAC0000490002010F0A9F9E6E7EB685BB1012B88
:10FAD000E3D164230493C82305934FF496730693EC
:10FAE0004FF4C87306E00A230493142305931E23DE
:10FAF000069328230793D0E7DC16FF1FD848FF1F83
:10FB000010B5044620B9096810F003FA204610BD6C
:10FB1000082010BD10B5044618B910F0EDF92046C4
:10FB200010BD082010BD10B5044618B910F0C6F974
:10FB3000204610BD082010BD0021F4E74942F2E73D
:10FB4000F1E7022804BF0C4B93F8D00030B90B4BFF
:10FB5000DB681B689B690A4A10681847012809D1AD
:10FB6000054B93F8D030012B04D1044BDB681B68A4
:10FB70005B69F0E7704700BF7431FF1F704C0200F3
:10FB80009032FF1F10B50020FFF7DBFF044B054A42
:10FB9000DB6810681B68BDE810409B69184700BF10
:10FBA000704C02009032FF1F043A38B504461D46DF
:10FBB0000846FB2A00F23E87DFE812F0FC003C0713
:10FBC0003C073C073C073C073C070C0112013C0783
:10FBD00016013C073C073C073C073C073C073C0739
:10FBE0003C073C073C073C073C073C073C073C07FD
:10FBF0003C073C073C073C073C073C073C073C07ED
:10FC00003C073C073C073C073C073C073C073C07DC
:10FC10003C073C073C073C071A012C013C073E010E
:10FC200050013C073C073C073C073C073C073C07AE
:10FC30003C073C073C073C073C073C073C073C07AC
:10FC40003C073C073C073C073C073C073C073C079C
:10FC50003C073C073C073C073C073C073C073C078C
:10FC60003C073C073C073C073C073C073C073C077C
:10FC70003C073C073C073C073C073C07620172011C
:10FC80007E018A019601A201AE01BA01C601D2012C
:10FC9000DE01EA01F601030210021D022A0234020B
:10FCA0003E023C07480252025C02660270027E027B
:10FCB0008C029A02A3023C073C073C07AC02B40248
:10FCC000BC02C602D0023C073C073C07D802E00257
:10FCD000E8023C073C073C073C073C073C073C0765
:10FCE000F202FC02060310033C073C073C073C07FA
:10FCF0003C073C071A0324032E03380342033C0746
:10FD00003C073C073C073C074C03560368037A0357
:10FD1000820390039A03A503AF03B603C303CF0383
:10FD2000DB03E703F303FF030B0417043C0723047F
:10FD30003004450451045E046A04760482048E048F
:10FD40009A04A804B604C404D204E004EE04FC043B
:10FD50000B051C052B053A05490558056705760571
:10FD600085059405A305B205C0053C073C073C0783
:10FD70003C073C073C073C073C073C073C073C076B
:10FD8000CE05DD05EC05FB050A0619062806370633
:10FD900046065406620670067E068C069A06A8067B
:10FDA000B606C306D006DD06EA06F8060A072107EE
:10FDB0002A0734072CB960200CF09EF928602046F1
:10FDC00038BD012C40F03986296860200CF0C0F95C
:10FDD0000024F4E7002C40F0338600242C60EEE78A
:10FDE000002CFAD00024EAE7002CF6D00024E6E745
:10FDF00034B9214608200CF00AFA00B22860DEE788
:10FE0000012C40F020862A88002108200CF030FACE
:10FE10000024D4E734B9214609200CF0F8F900B2E7
:10FE20002860CCE7012C40F011862A8800210920A7
:10FE30000CF01EFA0024C2E734B9012108200CF0AE
:10FE4000E6F900B22860BAE7012C40F002862146AC
:10FE50002A8808200CF00CFA0024B0E734B90121FC
:10FE600009200CF0D4F900B22860A8E7012C40F07A
:10FE7000F38521462A8809200CF0FAF900249EE730
:10FE80004CB9012103200CF063F9214602200CF04B
:10FE9000BEF9286093E7012C14BF002404248EE7E8
:10FEA000002CF8D1012103200CF052F9012102208D
:10FEB0000CF0ADF9286082E7002CECD10221032080
:10FEC0000CF046F9214602200CF0A1F9286076E7F3
:10FED000002CE0D1214603200CF03AF92146022003
:10FEE0000CF095F928606AE7002CD4D12146032054
:10FEF0000CF02EF9012102200CF089F928605EE750
:10FF0000002CC8D1032108460CF022F9214602201A
:10FF10000CF07DF9286052E7002CBCD104210320AD
:10FF20000CF016F9214602200CF071F9286046E722
:10FF3000002CB0D1042103200CF00AF90121022089
:10FF40000CF065F928603AE7002CA4D105210320C4
:10FF50000CF0FEF8214602200CF059F928602EE73B
:10FF6000002C98D1052103200CF0F2F80121022089
:10FF70000CF04DF9286022E7002C8CD106210320DB
:10FF80000CF0E6F8214602200CF041F9286016E753
:10FF9000002C80D1072103200CF0DAF82146022042
:10FFA0000CF035F928600AE7002C7FF474AF0721C4
:10FFB00003200CF0CDF8012102200CF028F9286074
:10FFC000FDE6002C7FF467AF082103200CF0C0F899
:10FFD000214602200CF01BF92860F0E6002C7FF48B
:10FFE0005AAF082103200CF0B3F8012102200CF0D5
:10FFF0000EF92860E3E6002C7FF44DAF09210320C1
:020000021000EC
:100000000CF0A6F8214602200CF001F92860D6E693
:10001000002C7FF440AF214612200CF0F8F800B21B
:100020002860CCE6002C7FF436AF012112200CF0C2
:10003000EEF800B22860C2E6002C7FF42CAF214617
:1000400013200CF0E4F800B22860B8E6002C7FF42E
:1000500022AF214615200CF0DAF800B22860AEE697
:10006000002C7FF418AF012115200CF0D0F800B25D
:100070002860A4E6002C7FF40EAF214616200CF079
:10008000C6F800B228609AE6002C7FF404AF012184
:1000900016200CF0BCF800B2286090E6002C7FF42B
:1000A000FAAE0A2103200CF053F8214602200CF08E
:1000B000AEF800B2286082E6002C7FF4ECAE0A2194
:1000C00003200CF045F8012102200CF0A0F800B24A
:1000D000286074E6002C7FF4DEAE0B2103200CF0C8
:1000E00037F8214602200CF092F800B2286066E64C
:1000F000002C7FF4D0AE214606200CF088F8286052
:100100005DE6002C7FF4C7AE012106200CF07FF8DD
:10011000286054E6002C7FF4BEAE41200BF0ECFFCB
:1001200028604CE6002C7FF4B6AE42200BF0E4FFD2
:10013000286044E6002C7FF4AEAE012146200CF08E
:1001400066F800B228603AE6002C7FF4A4AE21469F
:1001500046200CF05CF800B2286030E6002C7FF4FA
:100160009AAE47200BF0C8FF286028E6002C7FF4E9
:1001700092AE21200BF0C0FF286020E6002C7FF417
:100180008AAE22200BF0B8FF286018E6002C7FF41E
:1001900082AE214623200CF03AF800B228600EE629
:1001A000002C7FF478AE27200BF0A6FF20F07F40D4
:1001B000286004E6002C7FF46EAE28200BF09CFF34
:1001C00020F07F402860FAE5002C7FF464AE012126
:1001D0002A200CF01CF800B22860F0E5002C7FF417
:1001E0005AAE21462A200CF012F800B22860E6E54B
:1001F000002C7FF450AE214639200CF008F800B2F4
:100200002860DCE5002C7FF446AE012139200BF09C
:10021000FEFF00B22860D2E5002C7FF43CAE214600
:100220003D200BF0F4FF00B22860C8E5002C7FF4FD
:1002300032AE21463F200BF0EAFF00B22860BEE557
:10024000002C7FF428AE21463A200BF0E0FF00B2EC
:100250002860B4E5002C7FF41EAE214653200BF03D
:10026000D6FF00B22860AAE534B9012164200BF062
:10027000CEFF00B22860A2E5012C40F0F0832146B9
:100280002A8864200BF0F4FF002498E534B9214655
:1002900064200BF0BCFF00B2286090E5012C40F018
:1002A000E1832A88002164200BF0E2FF002486E528
:1002B000002C7FF4F0AD66200BF01EFF28607EE579
:1002C00024B968200BF018FF286078E5012C40F075
:1002D000CC8329680FF010FE002470E5002C7FF419
:1002E000DAAD012169200BF092FF00B2286066E5CB
:1002F000002C7FF4D0ADBE4B03EB011359890FF0F6
:100300008CFD28605BE5002C7FF4C5AD214669209B
:100310000BF07DFF00B2286051E5002C7FF4BBADEF
:100320000FF0E5FD28604AE51CB90FF00AFE2860D1
:1003300045E5012C40F09C8329680FF0FEFD002468
:100340003DE5002C7FF4A7AD21466D200BF000FFAA
:100350006C200BF0D1FE286031E5002C7FF49BADC2
:1003600001216D200BF0F4FE6C200BF0C5FE28601F
:1003700025E5002C7FF48FAD02216D200BF0E8FE07
:100380006C200BF0B9FE286019E5002C7FF483ADDA
:1003900003216D200BF0DCFE6C200BF0ADFE28601D
:1003A0000DE5002C7FF477AD04216D200BF0D0FE1D
:1003B0006C200BF0A1FE286001E5002C7FF46BADF2
:1003C00005216D200BF0C4FE6C200BF095FE28601B
:1003D000F5E4002C7FF45FAD06216D200BF0B8FE34
:1003E0006C200BF089FE2860E9E4002C7FF453AD0B
:1003F00007216D200BF0ACFE6C200BF07DFE286019
:10040000DDE41CB90FF0D8FC2860D8E4012C40F0E2
:10041000328329680FF0C2FC0024D0E43CB9744B4D
:1004200003EB011359890FF0EEFC2860C7E4012C9F
:1004300040F024836E4B2A6803EB01130024598992
:100440000FF0CFFCBBE4002C7FF425AD01216F2021
:100450000BF07EFE6E200BF04FFE2860AFE41CB95F
:100460000FF039FD2860AAE4012C40F00A832968C6
:100470000FF024FD0024A2E4002C7FF40CAD032136
:100480006F200BF065FE6E200BF036FE286096E4C0
:10049000002C7FF400AD04216F200BF059FE6E207C
:1004A0000BF02AFE28608AE4002C7FF4F4AC0521CE
:1004B0006F200BF04DFE6E200BF01EFE28607EE4D8
:1004C000002C7FF4E8AC06216F200BF041FE6E207B
:1004D0000BF012FE286072E4002C7FF4DCAC0721E4
:1004E0006F200BF035FE6E200BF006FE286066E4F0
:1004F000002C7FF4D0AC08216F200BF029FE2146A0
:100500006E200BF084FE00B2286058E4002C7FF4CB
:10051000C2AC08216F200BF01BFE01216E200BF0F6
:1005200076FE00B228604AE4002C7FF4B4AC0921C6
:100530006F200BF00DFE21466E200BF068FE00B21E
:1005400028603CE4002C7FF4A6AC0A216F200BF05D
:10055000FFFD21466E200BF05AFE00B228602EE40B
:10056000002C7FF498AC0A216F200BF0F1FD0121E3
:100570006E200BF04CFE00B2286020E4002C7FF4CB
:100580008AAC0B216F200BF0E3FD21466E200BF0AF
:100590003EFE00B2286012E4002C7FF47CAC0B21FC
:1005A0006F200BF0D5FD01216E200BF030FE00B264
:1005B000286004E4002C7FF46EAC0C216F200BF05B
:1005C000C7FD21466E200BF022FE00B22860FFF727
:1005D000F6BB002C7FF45FAC0C216F200BF0B8FD54
:1005E00001216E200BF013FE00B22860FFF7E7BB7D
:1005F000D048FF1F002C7FF44EAC0D216F200BF074
:10060000A7FD21466E200BF002FE00B22860FFF726
:10061000D6BB002C7FF43FAC0D216F200BF098FD72
:1006200001216E200BF0F3FD00B22860FFF7C7BB7D
:10063000002C7FF430AC0E216F200BF089FD214699
:100640006E200BF0E4FD00B22860FFF7B8BB002C71
:100650007FF421AC0E216F200BF07AFD01216E207A
:100660000BF0D5FD00B22860FFF7A9BB002C7FF48A
:1006700012AC0F216F200BF06BFD21466E200BF0AA
:10068000C6FD00B22860FFF79ABB002C7FF403ACD4
:100690000F216F200BF05CFD01216E200BF0B7FDE8
:1006A00000B22860FFF78BBB002C7FF4F4AB102165
:1006B0006F200BF04DFD21466E200BF0A8FD00B21F
:1006C0002860FFF77CBB002C7FF4E5AB11216F2085
:1006D0000BF03EFD21466E200BF099FD00B2286024
:1006E000FFF76DBB002C7FF4D6AB11216F200BF010
:1006F0002FFD01216E200BF08AFD00B22860FFF76C
:100700005EBB002C7FF4C7AB12216F200BF020FDE5
:1007100021466E200BF07BFD00B22860FFF74FBB37
:10072000002C7FF4B8AB13216F200BF011FD214694
:100730006E200BF06CFD2860FFF741BB002C7FF4AE
:10074000AAAB13216F200BF003FD01216E200BF0EB
:100750005EFD2860FFF733BB002C7FF49CABC0210B
:100760006F200BF0F5FC21466E200BF050FD00B21F
:100770002860FFF724BB002C7FF48DABC0216F20D5
:100780000BF0E6FC01216E200BF041FD00B2286069
:10079000FFF715BB002C7FF47EABC1216F200BF05F
:1007A000D7FC21466E200BF032FD00B22860FFF727
:1007B00006BB002C7FF46FABC1216F200BF0C8FC8F
:1007C00001216E200BF023FD00B22860FFF7F7BA7D
:1007D000002C7FF460ABC2216F200BF0B9FC2146E6
:1007E0006E200BF014FD00B22860FFF7E8BA002C71
:1007F0007FF451ABC2216F200BF0AAFC01216E20C7
:100800000BF005FD00B22860FFF7D9BA002C7FF489
:1008100042ABC3216F200BF09BFC21466E200BF0F6
:10082000F6FC00B22860FFF7CABA002C7FF433ABA5
:10083000C3216F200BF08CFC01216E200BF0E7FC34
:1008400000B22860FFF7BBBA002C7FF424ABC421B0
:100850006F200BF07DFC21466E200BF0D8FC286049
:10086000FFF7ADBA002C7FF416ABC4216F200BF05C
:100870006FFC01216E200BF0CAFC2860FFF79FBAC5
:10088000002C7FF408ABC5216F200BF061FC2146E2
:100890006E200BF0BCFC2860FFF791BA002C7FF4AF
:1008A000FAAAC5216F200BF053FC01216E200BF03A
:1008B000AEFC2860FFF783BA002C7FF4ECAAC621B7
:1008C0006F200BF045FC21466E200BF0A0FC286049
:1008D000FFF775BA002C7FF4DEAAC6216F200BF05B
:1008E00037FC01216E200BF092FC2860FFF767BAFD
:1008F000002C7FF4D0AAC7216F200BF029FC2146E1
:100900006E200BF084FC2860FFF759BA002C7FF4AE
:10091000C2AAC7216F200BF01BFC01216E200BF037
:1009200076FC2860FFF74BBA002C7FF4B4AAC821EC
:100930006F200BF00DFC6E200BF0DEFB2860FFF744
:100940003EBA002C7FF4A7AAC9216F200BF000FC4F
:100950006E200BF0D1FB2860FFF731BA002C7FF43A
:100960009AAACA216F200BF0F3FB6E200BF0C4FB98
:100970002860FFF724BA002C7FF48DAACB216F20CA
:100980000BF0E6FB6E200BF0B7FB2860FFF717BA01
:1009900024B9434BDB682B60FFF711BA012C73D1EC
:1009A0003F4B2A68DA600024FFF709BA34B93D49A1
:1009B00001EB001043892B60FFF701BA012C66D1CF
:1009C00038492B6801EB001000244381FFF7F7B989
:1009D00034B9344901EB0010437A2B60FFF7EFB9CB
:1009E000012C57D108012F4900F1080209300A44AF
:1009F000014428780FF09EFB0024FFF7E0B9002C9B
:100A00004BD1284901EB0010037A2B60FFF7D7B9CF
:100A1000002C7FF440AA234901EB0010C3882B600F
:100A2000FFF7CDB9002C7FF436AA1D4B5B682B6015
:100A3000FFF7C5B90424FFF7C2B90024FFF7BFB917
:100A40000024FFF7BCB90024FFF7B9B90024FFF771
:100A5000B6B90024FFF7B3B90024FFF7B0B90024FA
:100A6000FFF7ADB90024FFF7AAB90024FFF7A7B933
:100A70000024FFF7A4B90024FFF7A1B90024FFF771
:100A80009EB90024FFF79BB90024FFF798B9002412
:100A9000FFF795B90024FFF792B90024FFF78FB94B
:100AA000DC16FF1FD048FF1F10B41346044608464B
:100AB00019B9224610BCFFF777B8082010BC704760
:100AC0000120704707B5019239B9024601AB0120F8
:100AD000FFF76AF803B05DF804FB0820FAE7084660
:100AE0000BF00ABB084611460BF032BB0846114614
:100AF0000BF08DBB084611461A460BF0B9BB38B552
:100B0000274B284DDC686068236864302860DB6808
:100B10009847236828685B699847234B23495A699B
:100B20000A602349C2F804122249C2F808120021BF
:100B300011705170204A1A62204ADA61204A9A6183
:100B4000204A5A62204ADA64204A9A63204A5A6349
:100B5000204A9A62204ADA62204A9A64204A5A64F9
:100B6000204A5A65204A1A65204A1A66204ADA65E0
:100B7000204A9A653222DA60012040F28A229A6085
:100B800018741D4B4FF47A729A8041F270721A6099
:100B900059724FF480725A81BDE83840FEF7D1BFD8
:100BA000704C02009032FF1F7431FF1FE048FF1F9E
:100BB000C10A0100E1F9000027FB000041FB000031
:100BC0003DFB000039FB000001FA0000A90A01000A
:100BD000C50A010015FB000001FB0000FDF9000043
:100BE000F1F9000017FA0000DDF9000043FB0000F6
:100BF000E5F9000085FB0000D048FF1F002070478A
:100C000001207047014B00225A6070477431FF1F6A
:100C100010B50C460BF070FA206010BD0BF098BABE
:100C200038B50D46044620B90FF0D0FB28602046A9
:100C300038BD082038BD30B589B004AC0546102257
:100C40000021204613F032FF374B1A68AA1A092AEE
:100C500006D999681D6064224A435A6000229A604E
:100C60009A6801329A60314B33F8060C5A78029038
:100C7000981E019033F8041C0091002029460FF0C3
:100C8000BFFC0EF01DF820B10022114610460EF0F8
:100C9000A3F80EF00FF898B10EF08CF803280FD8D7
:100CA000DFE800F01810022E00200FF0B2FB0490D5
:100CB00000200FF0B5FB059094E80F000EF01AF835
:100CC00009B030BD00200FF07EFB049000200FF033
:100CD0007DFBF0E700216F200BF03AFA6E200BF05D
:100CE0000BFA0121049069200BF091FA00210546CE
:100CF00069200BF08CFA00B200FA85F50595DBE768
:100D000076200BF0F9F96423C0F30222C0F30250FD
:100D10005A434343A3F52F730593054B0693A3F55D
:100D2000FA6304920793C7E7F816FF1FD648FF1F20
:100D3000F0D8FFFF10B5044620B909680FF058FB42
:100D4000204610BD082010BD10B5044618B90FF09C
:100D500042FB204610BD082010BD10B5044618B94E
:100D60000FF024FB204610BD082010BD0021F4E741
:100D70004942F2E7F1E7022804BF0C4B93F8D00098
:100D800030B90B4BDB681B689B690A4A106818472F
:100D9000012809D1054B93F8D030012B04D1044B25
:100DA000DB681B685B69F0E7704700BF7431FF1FA9
:100DB000704C02009032FF1F10B50020FFF7DBFFE0
:100DC000044B054ADB6810681B68BDE810409B694E
:100DD000184700BF704C02009032FF1F043A38B52C
:100DE00004461D460846FB2A00F2D887DFE812F0C9
:100DF000FC00D607D607D607D607D607D6070C01BC
:100E00001201D6071601D607D607D607D607D6078A
:100E1000D607D607D607D607D607D607D607D607EA
:100E2000D607D607D607D607D607D607D607D607DA
:100E3000D607D607D607D607D607D607D607D607CA
:100E4000D607D607D607D607D607D6071A012B012D
:100E5000D6073C014E01D607D607D607D607D607D8
:100E6000D607D607D607D607D607D607D607D6079A
:100E7000D607D607D607D607D607D607D607D6078A
:100E8000D607D607D607D607D607D607D607D6077A
:100E9000D607D607D607D607D607D607D607D6076A
:100EA000D607D607D607D607D607D607D607D6075A
:100EB000600170017C01D607D607D607D607D60792
:100EC000D607D607D60788019401A001D607D60712
:100ED000AC01B501BE01D607C701D001D901D607C3
:100EE000E201EE01D607FB010402D607D607D607BA
:100EF0000D0215021D0227023102D607D607D607BA
:100F0000390241024902D607D607D607D607D607C7
:100F1000D607D60753025D02670271027B02920276
:100F2000A902C302DD02F70210031A0324032E03F1
:100F30003803D607D607D607D607D60742034C0391
:100F40005E037003780380038A039603A003A7035C
:100F5000B503C103CD03D903E503F103FD03090480
:100F6000D607150422043904450451045D046904BC
:100F7000750481048D049B04A904B704C504D3043B
:100F8000E104EF04FD040E051D052C053B054A0593
:100F900059056805770586059505A405B205D607A8
:100FA000C005D905F2050E062A0646066206D607D2
:100FB000D607D6076F067E068D069C06AB06BA06D8
:100FC000C906D806E706F506030711071F072D0710
:100FD0003B0749075707640771077E07D6078B074A
:100FE000A007B907C307CE072CB960200BF084F81F
:100FF0002860204638BD012C40F0D3862968602047
:101000000BF0A6F80024F4E7002C40F0CD86002475
:101010002C60EEE7002CFAD00024EAE7002CF6D092
:101020000024E6E72CB9214608200BF0F0F82860F0
:10103000DFE7012C40F0BB862A88002108200BF056
:1010400017F90024D5E72CB9214609200BF0DFF869
:101050002860CEE7012C40F0AD862A8800210920C7
:101060000BF006F90024C4E734B9012108200BF085
:10107000CEF800B22860BCE7012C40F09E862146E5
:101080002A8808200BF0F4F80024B2E734B90121D3
:1010900009200BF0BCF800B22860AAE7012C40F050
:1010A0008F8621462A8809200BF0E2F80024A0E769
:1010B0004CB9012103200BF04BF8214602200BF024
:1010C000A6F8286095E7012C14BF0024042490E7BB
:1010D000002CF8D1012103200BF03AF80121022065
:1010E0000BF095F8286084E7002CECD10221032056
:1010F0000BF02EF8214602200BF089F8286078E7E3
:10110000002CE0D1022103200BF022F80121022063
:101110000BF07DF828606CE7002CD4D10321084641
:101120000BF016F8012102200BF071F8286060E73F
:10113000002CC8D1032108460BF00AF821460220F2
:101140000BF065F8286054E7002CBCD12146122032
:101150000BF05DF800B228604BE7002CB3D1012101
:1011600012200BF054F800B2286042E7002CAAD1FC
:10117000214613200BF04BF800B2286039E7002C11
:10118000A1D1214615200BF042F800B2286030E7CB
:10119000002C98D1012115200BF039F800B22860FD
:1011A00027E7002C8FD1214616200BF030F800B233
:1011B00028601EE7002C86D1214603200AF0C8FFD4
:1011C000214602200BF023F8286012E7002C7FF460
:1011D0007AAF214603200AF0BBFF012102200BF069
:1011E00016F8286005E7002C7FF46DAF21460B2030
:1011F0000BF00DF82860FCE6002C7FF464AF0121B1
:101200000B200BF004F82860F3E6002C7FF45BAFB2
:1012100041200AF071FF2860EBE6002C7FF453AF09
:1012200042200AF069FF2860E3E6002C7FF44BAF10
:10123000012146200AF0EBFF00B22860D9E6002C1D
:101240007FF441AF214646200AF0E1FF00B228605A
:10125000CFE6002C7FF437AF47200AF04DFF28601F
:10126000C7E6002C7FF42FAF21200AF045FF28604D
:10127000BFE6002C7FF427AF22200AF03DFF286054
:10128000B7E6002C7FF41FAF214623200AF0BFFFF2
:1012900000B22860ADE6002C7FF415AF27200AF0DD
:1012A0002BFF20F07F402860A3E6002C7FF40BAFDB
:1012B00028200AF021FF20F07F40286099E6002CCA
:1012C0007FF401AF01212A200AF0A1FF00B22860BB
:1012D0008FE6002C7FF4F7AE21462A200AF097FF14
:1012E00000B2286085E644B9D4216F200AF030FFAF
:1012F0006E200AF001FF28607BE6012C40F0638538
:10130000D4216F200AF024FF29686E200AF020FF04
:1013100000246EE644B9D5216F200AF019FF6E2033
:101320000AF0EAFE286064E6012C40F04F85D521E2
:101330006F200AF00DFF29686E200AF009FF0024D3
:1013400057E654B9D6216F200AF002FF21466E20DD
:101350000AF05DFF00B228604BE6012C40F03985B1
:10136000D6216F200AF0F4FE2A8800216E200AF0B0
:101370007FFF00243DE654B9D6216F200AF0E8FE35
:1013800001216E200AF043FF00B2286031E6012CF3
:1013900040F02285D6216F200AF0DAFE21462A8805
:1013A0006E200AF065FF002423E654B9D7216F2090
:1013B0000AF0CEFE21466E200AF029FF00B2286016
:1013C00017E6012C40F00B85D7216F200AF0C0FEF4
:1013D0002A8800216E200AF04BFF002409E64CB950
:1013E000D7216F200AF0B4FE01216E200AF00FFF12
:1013F0002860FEE5012C40F0F584D7216F200AF02B
:10140000A7FE21462A886E200AF032FF0024F0E56C
:10141000002C7FF458AE214639200AF0F8FE00B2C5
:101420002860E6E5002C7FF44EAE012139200AF059
:10143000EEFE00B22860DCE5002C7FF444AE2146CD
:101440003D200AF0E4FE00B22860D2E5002C7FF4D3
:101450003AAE21463F200AF0DAFE00B22860C8E525
:10146000002C7FF430AE21463A200AF0D0FE00B2C4
:101470002860BEE5002C7FF426AE214653200AF0FA
:10148000C6FE00B22860B4E534B9012164200AF038
:10149000BEFE00B22860ACE5012C40F0A6842146D7
:1014A0002A8864200AF0E4FE0024A2E534B921462B
:1014B00064200AF0ACFE00B228609AE5012C40F0EE
:1014C00097842A88002164200AF0D2FE002490E547
:1014D000002C7FF4F8AD66200AF00EFE286088E547
:1014E000002C7FF4F0AD68200AF006FE286080E54D
:1014F000002C7FF4E8AD012169200AF088FE00B2DB
:10150000286076E5002C7FF4DEADBF4A0C2303FB98
:10151000012319890EF0F9FE28606AE5002C7FF49A
:10152000D2AD214669200AF072FE00B2286060E563
:10153000002C7FF4C8AD0EF049FF286059E51CB9B6
:101540000EF06EFF286054E5012C40F054842968A9
:101550006B200AF0FDFD00244BE5002C7FF4B3ADB9
:1015600021466D200AF0F4FD6C200AF0C5FD2860CC
:101570003FE5002C7FF4A7AD01216D200AF0E8FDC6
:101580006C200AF0B9FD286033E5002C7FF49BAD98
:1015900002216D200AF0DCFD6C200AF0ADFD286010
:1015A00027E5002C7FF48FAD03216D200AF0D0FDDC
:1015B0006C200AF0A1FD28601BE5002C7FF483ADB0
:1015C00004216D200AF0C4FD6C200AF095FD28600E
:1015D0000FE5002C7FF477AD05216D200AF0B8FDF2
:1015E0006C200AF089FD286003E5002C7FF46BADC8
:1015F00006216D200AF0ACFD6C200AF07DFD28600C
:10160000F7E4002C7FF45FAD07216D200AF0A0FD08
:101610006C200AF071FD2860EBE41CB90EF044FE6A
:101620002860E6E4012C40F0E98329680EF02EFEE4
:101630000024DEE444B9744A0C2303FB0123198916
:101640000EF059FE2860D4E4012C40F0DA836E4A93
:101650000C2303FB01232A6819890EF03AFE0024AB
:10166000C7E4002C7FF42FAD01216F200AF070FD3C
:101670006E200AF041FD2860BBE4002C7FF423AD0E
:1016800002216F200AF064FD6E200AF035FD28600B
:10169000AFE4002C7FF417AD03216F200AF058FD52
:1016A0006E200AF029FD2860A3E4002C7FF40BAD26
:1016B00004216F200AF04CFD6E200AF01DFD286009
:1016C00097E4002C7FF4FFAC05216F200AF040FD69
:1016D0006E200AF011FD28608BE4002C7FF4F3AC3F
:1016E00006216F200AF034FD6E200AF005FD286007
:1016F0007FE4002C7FF4E7AC07216F200AF028FD7F
:101700006E200AF0F9FC286073E4002C7FF4DBAC57
:1017100008216F200AF01CFD21466E200AF077FD9B
:1017200000B2286065E4002C7FF4CDAC08216F2066
:101730000AF00EFD01216E200AF069FD00B228605A
:1017400057E4002C7FF4BFAC09216F200AF000FDA4
:1017500021466E200AF05BFD00B2286049E4002CAF
:101760007FF4B1AC0A216F200AF0F2FC21466E2012
:101770000AF04DFD00B228603BE4002C7FF4A3ACDE
:101780000A216F200AF0E4FC01216E200AF03FFDDF
:1017900000B228602DE4002C7FF495AC0B216F2063
:1017A0000AF0D6FC21466E200AF031FD00B2286016
:1017B0001FE4002C7FF487AC0B216F200AF0C8FCDB
:1017C00001216E200AF023FD00B2286011E4002CF4
:1017D0007FF479AC0C216F200AF0BAFC21466E2010
:1017E0000AF015FD00B2286003E4002C7FF46BAC16
:1017F0000C216F200AF0ACFC01216E200AF007FDDD
:1018000000B22860FFF7F5BBD048FF1F002C7FF423
:101810005AAC0D216F200AF09BFC21466E200AF085
:10182000F6FC00B22860FFF7E4BB002C7FF44BAC61
:101830000D216F200AF08CFC01216E200AF0E7FCDC
:1018400000B22860FFF7D5BB002C7FF43CAC0E2122
:101850006F200AF07DFC21466E200AF0D8FC00B211
:101860002860FFF7C6BB002C7FF42DAC0E216F2043
:101870000AF06EFC01216E200AF0C9FC00B228605B
:10188000FFF7B7BB002C7FF41EAC0F216F200AF0CE
:101890005FFC21466E200AF0BAFC00B22860FFF718
:1018A000A8BB002C7FF40FAC0F216F200AF050FC76
:1018B00001216E200AF0ABFC00B22860FFF799BB53
:1018C000002C7FF400AC10216F200AF041FC21466F
:1018D0006E200AF09CFC00B22860FFF78ABB002C47
:1018E0007FF4F1AB11216F200AF032FC21466E200B
:1018F0000AF08DFC00B22860FFF77BBB002C7FF460
:10190000E2AB11216F200AF023FC01216E200AF0C6
:101910007EFC00B22860FFF76CBB002C7FF4D3ABD9
:1019200012216F200AF014FC21466E200AF06FFC91
:1019300000B22860FFF75DBB002C7FF4C4AB13211D
:101940006F200AF005FC21466E200AF060FC28603A
:10195000FFF74FBB002C7FF4B6AB13216F200AF0CA
:10196000F7FB01216E200AF052FC2860FFF741BB13
:101970004CB9D0216F200AF0EBFB6E200AF0BCFBC3
:101980002860FFF736BB012C40F03E82D0216F204B
:101990000AF0DEFB29686E200AF0DAFB0024FFF76C
:1019A00028BB4CB9D1216F200AF0D2FB6E200AF07F
:1019B000A3FB2860FFF71DBB012C40F02882D1213A
:1019C0006F200AF0C5FB29686E200AF0C1FB0024D5
:1019D000FFF70FBB5CB9D2216F200AF0B9FB21469B
:1019E0006E200AF014FC00B22860FFF702BB012C45
:1019F00040F01082D2216F200AF0AAFB2A88002131
:101A00006E200AF035FC0024FFF7F3BA5CB9D2214E
:101A10006F200AF09DFB01216E200AF0F8FB00B256
:101A20002860FFF7E6BA012C40F0F781D2216F2041
:101A30000AF08EFB21462A886E200AF019FC002449
:101A4000FFF7D7BA5CB9D3216F200AF081FB21469A
:101A50006E200AF0DCFB00B22860FFF7CABA012C46
:101A600040F0DE81D3216F200AF072FB2A8800212A
:101A70006E200AF0FDFB0024FFF7BBBA5CB9D3214E
:101A80006F200AF065FB01216E200AF0C0FB00B256
:101A90002860FFF7AEBA012C40F0C581D3216F203A
:101AA0000AF056FB21462A886E200AF0E1FB00244A
:101AB000FFF79FBA002C7FF406AB1D216F200AF0C0
:101AC00047FB6E200AF018FB2860FFF792BA002C43
:101AD0007FF4F9AAC0216F200AF03AFB21466E205C
:101AE0000AF095FB00B22860FFF783BA002C7FF460
:101AF000EAAAC0216F200AF02BFB01216E200AF018
:101B000086FB00B22860FFF774BA002C7FF4DBAAD2
:101B1000C1216F200AF01CFB21466E200AF077FBE2
:101B200000B22860FFF765BA002C7FF4CCAAC1216F
:101B30006F200AF00DFB01216E200AF068FB00B255
:101B40002860FFF756BA002C7FF4BDAAC2216F208F
:101B50000AF0FEFA21466E200AF059FB00B2286016
:101B6000FFF747BA002C7FF4AEAAC2216F200AF01B
:101B7000EFFA01216E200AF04AFB00B22860FFF75D
:101B800038BA002C7FF49FAAC3216F200AF0E0FA34
:101B900021466E200AF03BFB00B22860FFF729BA0D
:101BA000002C7FF490AAC3216F200AF0D1FA012102
:101BB0006E200AF02CFB00B22860FFF71ABA002C46
:101BC0007FF481AAC4216F200AF0C2FA21466E2058
:101BD0000AF01DFB2860FFF70CBA002C7FF473AAF3
:101BE000C4216F200AF0B4FA01216E200AF00FFB25
:101BF0002860FFF7FEB9002C7FF465AAC5216F208D
:101C00000AF0A6FA21466E200AF001FB2860FFF7D1
:101C1000F0B9002C7FF457AAC5216F200AF098FA7A
:101C200001216E200AF0F3FA2860FFF7E2B9002CD8
:101C30007FF449AAC6216F200AF08AFA21466E2055
:101C40000AF0E5FA2860FFF7D4B9002C7FF43BAA2C
:101C5000C6216F200AF07CFA01216E200AF0D7FA23
:101C60002860FFF7C6B9002C7FF42DAAC7216F208A
:101C70000AF06EFA21466E200AF0C9FA2860FFF7D2
:101C8000B8B9002C7FF41FAAC7216F200AF060FAB0
:101C900001216E200AF0BBFA2860FFF7AAB9002CD8
:101CA0007FF411AAC8216F200AF052FA6E200AF0C0
:101CB00023FA2860FFF79DB9002C7FF404AAC921FC
:101CC0006F200AF045FA6E200AF016FA2860FFF736
:101CD00090B9002C7FF4F7A9CA216F200AF038FAD6
:101CE0006E200AF009FA2860FFF783B9002C7FF410
:101CF000EAA9CB216F200AF02BFA6E200AF0FCF93A
:101D00002860FFF776B93CB94D4A0C2303FB01204C
:101D100003892B60FFF76DB9012C40F08780484A9A
:101D20000C2303FB01202B6803810024FFF761B91A
:101D30003CB9434A0C2303FB0120C3792B60FFF716
:101D400058B9012C75D101EB410080003C49821D3E
:101D500007300A44014428780EF05CFC0024FFF7A9
:101D600048B9002C68D1364A0C2303FB0120837943
:101D70002B60FFF73EB9002C7FF4A5A9304B0C2255
:101D800002FB013083882B60FFF733B9002C7FF40E
:101D90009AA92C4B5B682B60FFF72BB90424FFF743
:101DA00028B90024FFF725B90024FFF722B9002441
:101DB000FFF71FB90024FFF71CB90024FFF719B97A
:101DC0000024FFF716B90024FFF713B90024FFF72A
:101DD00010B90024FFF70DB90024FFF70AB9002459
:101DE000FFF707B90024FFF704B90024FFF701B992
:101DF0000024FFF7FEB80024FFF7FBB80024FFF72C
:101E0000F8B80024FFF7F5B80024FFF7F2B8002473
:101E1000FFF7EFB80024FFF7ECB80024FFF7E9B8AC
:101E20000024FFF7E6B80024FFF7E3B80024FFF72B
:101E3000E0B80024FFF7DDB80024FFF7DAB800BFF0
:101E4000D048FF1FF816FF1F10B41346044608467B
:101E500019B9224610BCFEF7C1BF082010BC70475C
:101E60000120704707B5019239B9024601AB012044
:101E7000FEF7B4FF03B05DF804FB0820FAE708465C
:101E80000AF03AB9084611460AF062B90846114606
:101E90000AF0BDB9084611461A460AF0E9B938B544
:101EA000274B284DDC686068236864302860DB6855
:101EB0009847236828685B699847234B23495A69E8
:101EC0000A602349C2F804122249C2F8081201200C
:101ED000002110705170204A1A62204ADA61204AAB
:101EE0009A61204A5A62204ADA64204A9A63204A58
:101EF0005A63204A9A62204ADA62204A9A64204A47
:101F00005A64204A5A65204A1A65204A1A66204AAD
:101F1000DA65204A9A653222DA6040F28A229A60B3
:101F200018741D4B4FF47A725A8041F270721A8005
:101F3000D9714FF480721A81BDE83840FEF71BBF9B
:101F4000704C02009032FF1F7431FF1FE448FF1FE6
:101F5000611E0100010C01005B0D0100750D010007
:101F6000710D01006D0D0100210C0100491E0100E1
:101F7000651E0100490D0100350D01001D0C010019
:101F8000110C0100370C0100FD0B0100770D010061
:101F9000050C0100B90D0100D048FF1F002070475B
:101FA00001207047014B00225A6070477431FF1FB7
:101FB00010B50C460AF0A0F8206010BD0AF0C8B8B1
:101FC00038B50D46044620B90EF084FC2860204642
:101FD00038BD082038BD30B589B004AC05461022A4
:101FE0000021204612F062FD374B1A68AA1A092A0E
:101FF00006D999681D6064224A435A6000229A609B
:102000009A6801329A60314B33F8060C5A78029084
:10201000981E019033F8041C0091002029460EF010
:1020200073FD0CF04DFE20B10022114610460CF05D
:10203000D3FE0CF03FFE98B10CF0BCFE03280FD885
:10204000DFE800F01810022E00200EF066FC04906D
:1020500000200EF069FC059094E80F000CF04AFE99
:1020600009B030BD00200EF032FC049000200EF0CC
:1020700031FCF0E700216F200AF06AF86E200AF0C8
:102080003BF80121049069200AF0C1F800210546BF
:1020900069200AF0BCF800B200FA85F50595DBE787
:1020A00076200AF029F86423C0F30222C0F302501C
:1020B0005A434343A3F52F730593054B0693A3F5AA
:1020C000FA6304920793C7E71017FF1FD648FF1F54
:1020D000F0D8FFFF10B5044620B909680EF00CFCDB
:1020E000204610BD082010BD10B5044618B90EF0EA
:1020F000F6FB204610BD082010BD10B5044618B9E7
:102100000EF0D8FB204610BD082010BD0021F4E7DA
:102110004942F2E7F1E7022804BF0C4B93F8D000E4
:1021200030B90B4BDB681B689B690A4A106818477B
:10213000012809D1054B93F8D030012B04D1044B71
:10214000DB681B685B69F0E7704700BF7431FF1FF5
:10215000704C02009032FF1F10B50020FFF7DBFF2C
:10216000044B054ADB6810681B68BDE810409B699A
:10217000184700BF704C02009032FF1F043A38B578
:1021800004461D460846FB2A00F2D887DFE812F015
:10219000FC00D607D607D607D607D607D6070C0108
:1021A0001201D6071601D607D607D607D607D607D7
:1021B000D607D607D607D607D607D607D607D60737
:1021C000D607D607D607D607D607D607D607D60727
:1021D000D607D607D607D607D607D607D607D60717
:1021E000D607D607D607D607D607D6071A012B017A
:1021F000D6073C014E01D607D607D607D607D60725
:10220000D607D607D607D607D607D607D607D607E6
:10221000D607D607D607D607D607D607D607D607D6
:10222000D607D607D607D607D607D607D607D607C6
:10223000D607D607D607D607D607D607D607D607B6
:10224000D607D607D607D607D607D607D607D607A6
:10225000600170017C01D607D607D607D607D607DE
:10226000D607D607D60788019401A001D607D6075E
:10227000AC01B501BE01D607C701D001D901D6070F
:10228000E201EE01D607FB010402D607D607D60706
:102290000D0215021D0227023102D607D607D60706
:1022A000390241024902D607D607D607D607D60714
:1022B000D607D60753025D02670271027B029202C3
:1022C000A902C302DD02F70210031A0324032E033E
:1022D0003803D607D607D607D607D60742034C03DE
:1022E0005E037003780380038A039603A003A703A9
:1022F000B503C103CD03D903E503F103FD030904CD
:10230000D607150422043904450451045D04690408
:10231000750481048D049B04A904B704C504D30487
:10232000E104EF04FD040E051D052C053B054A05DF
:1023300059056805770586059505A405B205D607F4
:10234000C005D905F2050E062A0646066206D6071E
:10235000D607D6076F067E068D069C06AB06BA0624
:10236000C906D806E706F506030711071F072D075C
:102370003B0749075707640771077E07D6078B0796
:10238000A007B907C307CE072CB9602009F0B4FE37
:102390002860204638BD012C40F0D3862968602093
:1023A00009F0D6FE0024F4E7002C40F0CD8600248E
:1023B0002C60EEE7002CFAD00024EAE7002CF6D0DF
:1023C0000024E6E72CB92146082009F020FF286008
:1023D000DFE7012C40F0BB862A880021082009F0A5
:1023E00047FF0024D5E72CB92146092009F00FFF4B
:1023F0002860CEE7012C40F0AD862A880021092014
:1024000009F036FF0024C4E734B90121082009F09F
:10241000FEFE00B22860BCE7012C40F09E862146FB
:102420002A88082009F024FF0024B2E734B90121EA
:10243000092009F0ECFE00B22860AAE7012C40F068
:102440008F8621462A88092009F012FF0024A0E780
:102450004CB90121032009F07BFE2146022009F03E
:10246000D6FE286095E7012C14BF0024042490E7D1
:10247000002CF8D10121032009F06AFE012102207D
:1024800009F0C5FE286084E7002CECD1022103206E
:1024900009F05EFE2146022009F0B9FE286078E7C7
:1024A000002CE0D10321084609F052FE214602200B
:1024B00009F0ADFE28606CE7002CD4D10421032084
:1024C00009F046FE0121022009F0A1FE286060E724
:1024D000002CC8D10421032009F03AFE2146022035
:1024E00009F095FE286054E7002CBCD1214612204B
:1024F00009F08DFE00B228604BE7002CB3D101211A
:10250000122009F084FE00B2286042E7002CAAD114
:102510002146132009F07BFE00B2286039E7002C29
:10252000A1D12146152009F072FE00B2286030E7E3
:10253000002C98D10121152009F069FE00B2286015
:1025400027E7002C8FD12146162009F060FE00B24B
:1025500028601EE7002C86D12146032009F0F8FDF3
:102560002146022009F053FE286012E7002C7FF478
:102570007AAF2146032009F0EBFD0121022009F08A
:1025800046FE286005E7002C7FF46DAF21460B2046
:1025900009F03DFE2860FCE6002C7FF464AF0121C9
:1025A0000B2009F034FE2860F3E6002C7FF45BAFCB
:1025B000412009F0A1FD2860EBE6002C7FF453AF29
:1025C000422009F099FD2860E3E6002C7FF44BAF30
:1025D0000121462009F01BFE00B22860D9E6002C3C
:1025E0007FF441AF2146462009F011FE00B2286079
:1025F000CFE6002C7FF437AF472009F07DFD28603F
:10260000C7E6002C7FF42FAF212009F075FD28606C
:10261000BFE6002C7FF427AF222009F06DFD286073
:10262000B7E6002C7FF41FAF2146232009F0EFFD11
:1026300000B22860ADE6002C7FF415AF272009F02A
:102640005BFD20F07F402860A3E6002C7FF40BAFF9
:10265000282009F051FD20F07F40286099E6002CE9
:102660007FF401AF01212A2009F0D1FD00B22860DA
:102670008FE6002C7FF4F7AE21462A2009F0C7FD33
:1026800000B2286085E644B9D4216F2009F060FDCE
:102690006E2009F031FD28607BE6012C40F0638557
:1026A000D4216F2009F054FD29686E2009F050FDF7
:1026B00000246EE644B9D5216F2009F049FD6E2053
:1026C00009F01AFD286064E6012C40F04F85D52101
:1026D0006F2009F03DFD29686E2009F039FD0024C6
:1026E00057E654B9D6216F2009F032FD21466E20FD
:1026F00009F08DFD00B228604BE6012C40F03985D1
:10270000D6216F2009F024FD2A8800216E2009F0CF
:10271000AFFD00243DE654B9D6216F2009F018FD25
:1027200001216E2009F073FD00B2286031E6012C12
:1027300040F02285D6216F2009F00AFD21462A8823
:102740006E2009F095FD002423E654B9D7216F20AF
:1027500009F0FEFC21466E2009F059FD00B2286008
:1027600017E6012C40F00B85D7216F2009F0F0FC13
:102770002A8800216E2009F07BFD002409E64CB96F
:10278000D7216F2009F0E4FC01216E2009F03FFD04
:102790002860FEE5012C40F0F584D7216F2009F078
:1027A000D7FC21462A886E2009F062FD0024F0E55E
:1027B000002C7FF458AE2146392009F028FD00B2E4
:1027C0002860E6E5002C7FF44EAE0121392009F0A7
:1027D0001EFD00B22860DCE5002C7FF444AE2146EB
:1027E0003D2009F014FD00B22860D2E5002C7FF4F2
:1027F0003AAE21463F2009F00AFD00B22860C8E544
:10280000002C7FF430AE21463A2009F000FD00B2E2
:102810002860BEE5002C7FF426AE2146532009F047
:10282000F6FC00B22860B4E534B90121642009F057
:10283000EEFC00B22860ACE5012C40F0A6842146F5
:102840002A88642009F014FD0024A2E534B9214649
:10285000642009F0DCFC00B228609AE5012C40F00D
:1028600097842A880021642009F002FD002490E565
:10287000002C7FF4F8AD662009F03EFC286088E566
:10288000002C7FF4F0AD682009F036FC286080E56C
:10289000002C7FF4E8AD0121692009F0B8FC00B2FA
:1028A000286076E5002C7FF4DEADBF4A0C2303FBE5
:1028B000012319890DF0ADFF28606AE5002C7FF433
:1028C000D2AD2146692009F0A2FC00B2286060E583
:1028D000002C7FF4C8AD0DF0FDFF286059E51CB950
:1028E0000EF022F8286054E5012C40F05484296849
:1028F0006B2009F02DFC00244BE5002C7FF4B3ADD8
:1029000021466D2009F024FC6C2009F0F5FB2860BD
:102910003FE5002C7FF4A7AD01216D2009F018FCE4
:102920006C2009F0E9FB286033E5002C7FF49BADB7
:1029300002216D2009F00CFC6C2009F0DDFB286001
:1029400027E5002C7FF48FAD03216D2009F000FCFA
:102950006C2009F0D1FB28601BE5002C7FF483ADCF
:1029600004216D2009F0F4FB6C2009F0C5FB286000
:102970000FE5002C7FF477AD05216D2009F0E8FB11
:102980006C2009F0B9FB286003E5002C7FF46BADE7
:1029900006216D2009F0DCFB6C2009F0ADFB2860FE
:1029A000F7E4002C7FF45FAD07216D2009F0D0FB28
:1029B0006C2009F0A1FB2860EBE41CB90DF0F8FED7
:1029C0002860E6E4012C40F0E98329680DF0E2FE7E
:1029D0000024DEE444B9744A0C2303FB0123198963
:1029E0000DF00DFF2860D4E4012C40F0DA836E4A2C
:1029F0000C2303FB01232A6819890DF0EEFE002445
:102A0000C7E4002C7FF42FAD01216F2009F0A0FB5B
:102A10006E2009F071FB2860BBE4002C7FF423AD2D
:102A200002216F2009F094FB6E2009F065FB2860FD
:102A3000AFE4002C7FF417AD03216F2009F088FB71
:102A40006E2009F059FB2860A3E4002C7FF40BAD45
:102A500004216F2009F07CFB6E2009F04DFB2860FB
:102A600097E4002C7FF4FFAC05216F2009F070FB88
:102A70006E2009F041FB28608BE4002C7FF4F3AC5E
:102A800006216F2009F064FB6E2009F035FB2860F9
:102A90007FE4002C7FF4E7AC07216F2009F058FB9E
:102AA0006E2009F029FB286073E4002C7FF4DBAC76
:102AB00008216F2009F04CFB21466E2009F0A7FB8E
:102AC00000B2286065E4002C7FF4CDAC08216F20B3
:102AD00009F03EFB01216E2009F099FB00B228604D
:102AE00057E4002C7FF4BFAC09216F2009F030FBC4
:102AF00021466E2009F08BFB00B2286049E4002CCF
:102B00007FF4B1AC0A216F2009F022FB21466E2030
:102B100009F07DFB00B228603BE4002C7FF4A3ACFD
:102B20000A216F2009F014FB01216E2009F06FFBD0
:102B300000B228602DE4002C7FF495AC0B216F20AF
:102B400009F006FB21466E2009F061FB00B2286007
:102B50001FE4002C7FF487AC0B216F2009F0F8FAFA
:102B600001216E2009F053FB00B2286011E4002C13
:102B70007FF479AC0C216F2009F0EAFA21466E202F
:102B800009F045FB00B2286003E4002C7FF46BAC35
:102B90000C216F2009F0DCFA01216E2009F037FBCF
:102BA00000B22860FFF7F5BBD048FF1F002C7FF470
:102BB0005AAC0D216F2009F0CBFA21466E2009F0A6
:102BC00026FB00B22860FFF7E4BB002C7FF44BAC7F
:102BD0000D216F2009F0BCFA01216E2009F017FBCE
:102BE00000B22860FFF7D5BB002C7FF43CAC0E216F
:102BF0006F2009F0ADFA21466E2009F008FB00B203
:102C00002860FFF7C6BB002C7FF42DAC0E216F208F
:102C100009F09EFA01216E2009F0F9FA00B228604D
:102C2000FFF7B7BB002C7FF41EAC0F216F2009F01B
:102C30008FFA21466E2009F0EAFA00B22860FFF709
:102C4000A8BB002C7FF40FAC0F216F2009F080FA95
:102C500001216E2009F0DBFA00B22860FFF799BB72
:102C6000002C7FF400AC10216F2009F071FA21468E
:102C70006E2009F0CCFA00B22860FFF78ABB002C66
:102C80007FF4F1AB11216F2009F062FA21466E202A
:102C900009F0BDFA00B22860FFF77BBB002C7FF47F
:102CA000E2AB11216F2009F053FA01216E2009F0E7
:102CB000AEFA00B22860FFF76CBB002C7FF4D3ABF8
:102CC00012216F2009F044FA21466E2009F09FFA84
:102CD00000B22860FFF75DBB002C7FF4C4AB13216A
:102CE0006F2009F035FA21466E2009F090FA28602D
:102CF000FFF74FBB002C7FF4B6AB13216F2009F018
:102D000027FA01216E2009F082FA2860FFF741BB03
:102D10004CB9D0216F2009F01BFA6E2009F0ECF9B4
:102D20002860FFF736BB012C40F03E82D0216F2097
:102D300009F00EFA29686E2009F00AFA0024FFF75C
:102D400028BB4CB9D1216F2009F002FA6E2009F09E
:102D5000D3F92860FFF71DBB012C40F02882D12158
:102D60006F2009F0F5F929686E2009F0F1F90024C7
:102D7000FFF70FBB5CB9D2216F2009F0E9F92146BA
:102D80006E2009F044FA00B22860FFF702BB012C64
:102D900040F01082D2216F2009F0DAF92A88002150
:102DA0006E2009F065FA0024FFF7F3BA5CB9D2216E
:102DB0006F2009F0CDF901216E2009F028FA00B248
:102DC0002860FFF7E6BA012C40F0F781D2216F208E
:102DD00009F0BEF921462A886E2009F049FA00243C
:102DE000FFF7D7BA5CB9D3216F2009F0B1F92146BA
:102DF0006E2009F00CFA00B22860FFF7CABA012C65
:102E000040F0DE81D3216F2009F0A2F92A88002149
:102E10006E2009F02DFA0024FFF7BBBA5CB9D3216C
:102E20006F2009F095F901216E2009F0F0F900B248
:102E30002860FFF7AEBA012C40F0C581D3216F2086
:102E400009F086F921462A886E2009F011FA00243B
:102E5000FFF79FBA002C7FF406AB1D216F2009F00D
:102E600077F96E2009F048F92860FFF792BA002C34
:102E70007FF4F9AAC0216F2009F06AF921466E207B
:102E800009F0C5F900B22860FFF783BA002C7FF47F
:102E9000EAAAC0216F2009F05BF901216E2009F038
:102EA000B6F900B22860FFF774BA002C7FF4DBAAF1
:102EB000C1216F2009F04CF921466E2009F0A7F9D5
:102EC00000B22860FFF765BA002C7FF4CCAAC121BC
:102ED0006F2009F03DF901216E2009F098F900B248
:102EE0002860FFF756BA002C7FF4BDAAC2216F20DC
:102EF00009F02EF921466E2009F089F900B2286008
:102F0000FFF747BA002C7FF4AEAAC2216F2009F068
:102F10001FF901216E2009F07AF900B22860FFF74D
:102F200038BA002C7FF49FAAC3216F2009F010F952
:102F300021466E2009F06BF900B22860FFF729BA2C
:102F4000002C7FF490AAC3216F2009F001F9012120
:102F50006E2009F05CF900B22860FFF71ABA002C65
:102F60007FF481AAC4216F2009F0F2F821466E2077
:102F700009F04DF92860FFF70CBA002C7FF473AA12
:102F8000C4216F2009F0E4F801216E2009F03FF917
:102F90002860FFF7FEB9002C7FF465AAC5216F20D9
:102FA00009F0D6F821466E2009F031F92860FFF7C4
:102FB000F0B9002C7FF457AAC5216F2009F0C8F89A
:102FC00001216E2009F023F92860FFF7E2B9002CF7
:102FD0007FF449AAC6216F2009F0BAF821466E2075
:102FE00009F015F92860FFF7D4B9002C7FF43BAA4B
:102FF000C6216F2009F0ACF801216E2009F007F915
:103000002860FFF7C6B9002C7FF42DAAC7216F20D6
:1030100009F09EF821466E2009F0F9F82860FFF7C4
:10302000B8B9002C7FF41FAAC7216F2009F090F8CF
:1030300001216E2009F0EBF82860FFF7AAB9002CF7
:103040007FF411AAC8216F2009F082F86E2009F0E0
:1030500053F82860FFF79DB9002C7FF404AAC9211A
:103060006F2009F075F86E2009F046F82860FFF728
:1030700090B9002C7FF4F7A9CA216F2009F068F8F5
:103080006E2009F039F82860FFF783B9002C7FF42F
:10309000EAA9CB216F2009F05BF86E2009F02CF82B
:1030A0002860FFF776B93CB94D4A0C2303FB012099
:1030B00003892B60FFF76DB9012C40F08780484AE7
:1030C0000C2303FB01202B6803810024FFF761B967
:1030D0003CB9434A0C2303FB0120C3792B60FFF763
:1030E00058B9012C75D101EB410080003C49821D8B
:1030F00007300A44014428780DF010FD0024FFF742
:1031000048B9002C68D1364A0C2303FB012083798F
:103110002B60FFF73EB9002C7FF4A5A9304B0C22A1
:1031200002FB013083882B60FFF733B9002C7FF45A
:103130009AA92C4B5B682B60FFF72BB90424FFF78F
:1031400028B90024FFF725B90024FFF722B900248D
:10315000FFF71FB90024FFF71CB90024FFF719B9C6
:103160000024FFF716B90024FFF713B90024FFF776
:1031700010B90024FFF70DB90024FFF70AB90024A5
:10318000FFF707B90024FFF704B90024FFF701B9DE
:103190000024FFF7FEB80024FFF7FBB80024FFF778
:1031A000F8B80024FFF7F5B80024FFF7F2B80024C0
:1031B000FFF7EFB80024FFF7ECB80024FFF7E9B8F9
:1031C0000024FFF7E6B80024FFF7E3B80024FFF778
:1031D000E0B80024FFF7DDB80024FFF7DAB800BF3D
:1031E000D048FF1F1017FF1F10B4134604460846AF
:1031F00019B9224610BCFEF7C1BF082010BC7047A9
:103200000120704707B5019239B9024601AB012090
:10321000FEF7B4FF03B05DF804FB0820FAE70846A8
:1032200008F06ABF0846114608F092BF08461146EA
:1032300008F0EDBF084611461A4609F019B838B52E
:10324000274B284DDC686068236864302860DB68A1
:103250009847236828685B699847234B23495A6934
:103260000A602349C2F804122249C2F80812012058
:10327000002110705170204A1A62204ADA61204AF7
:103280009A61204A5A62204ADA64204A9A63204AA4
:103290005A63204A9A62204ADA62204A9A64204A93
:1032A0005A64204A5A65204A1A65204A1A66204AFA
:1032B000DA65204A9A653222DA6040F28A229A6000
:1032C00018741D4B4FF47A725A8041F270721A8052
:1032D000D9714FF480721A81BDE83840FEF71BBFE8
:1032E000704C02009032FF1F7431FF1FE848FF1F2F
:1032F00001320100A11F0100FB2001001521010086
:10330000112101000D210100C11F0100E93101005F
:1033100005320100E9200100D5200100BD1F010098
:10332000B11F0100D71F01009D1F010017210100DF
:10333000A51F010059210100D048FF1F014B0022A9
:103340005A6070477431FF1F70B5084E084D3368DE
:1033500004462A46014600200DF04AFD33682A46FD
:1033600021460120BDE870400DF042BD884BFF1F93
:10337000EC48FF1F014B18680DF09BBD884BFF1FE9
:1033800001280CD8074B1A68202303FA00F040F0FC
:10339000020002EB800043680B60002070470820A9
:1033A000704700BF884BFF1F012810B5144611D08D
:1033B00003D302281AD0042010BD14680F4A104B02
:1033C000D268126824B15269D8689047002010BDB5
:1033D0009269F9E7094B0A4ADB6850681B681B6A67
:1033E0009847003018BF01202060EFE7034B044AE4
:1033F000DB6890681B681B6AF2E700BF704C020034
:103400002817FF1F022804BF0B4B93F8D00030B9D8
:103410000A4BDB681B685B69094A1068184701287A
:1034200009D1054B93F8D030012B04D1034BDB6855
:103430001B689B69F0E770477431FF1F704C0200F6
:103440002817FF1F70B50020FFF7DCFF104B114C51
:10345000DD6820682B689B6898472B6860689B68CC
:1034600098472B68A0689B6898472B68A0699B6861
:1034700098472B6820699B6898472B6860699B6810
:1034800098472B68E0689B68BDE87040184700BF0C
:10349000704C02002817FF1F2DE9F843184C9DF8C7
:1034A00020609DF82450984623680F469B680021B1
:1034B00047F0800091469847236800219B68484662
:1034C0009847236800219B6840469847236800215D
:1034D0009B6830469847236828469B680121984797
:1034E000084B1B6848EA092807F07F0746EA0826C8
:1034F00003EB870745EA06257D60BDE8F88300BF3A
:10350000844BFF1F884BFF1F07B5D3B20193C2F353
:1035100007230093C2F30743120EFFF7BDFF03B06A
:103520005DF804FB0A4601460020FFF7EDBF0128C5
:1035300073B505460C4624D8134E335C63B1134B68
:10354000202103EB8003814041F00701DA69C9B211
:10355000FFF7DAFF002373552026AE4046F00D0139
:103560002246C9B200242846FFF7CEFF2846019420
:10357000009423462246F1B2FFF78EFF204602B0A8
:1035800070BD0820FBE700BF7000FF1F2817FF1F5A
:10359000012873B505460E461CD82024844044F00B
:1035A000070186EAE672A2EBE672C9B2FFF7ACFF4A
:1035B000094A0123002E5355E1B2B8BF022300246B
:1035C00001932846009423462246FFF765FF2046D4
:1035D00002B070BD0820FBE77000FF1F0021D7E795
:1035E0004942D5E7D4E738B5234B01F07F042344A3
:1035F00093F81432DB0705D4204B1B6803EB8404DB
:10360000606838BD1E4D2B6800219B682046984796
:103610002B6800219B68084698472B6800219B680F
:10362000084698472B6800219B68084698472B68F6
:1036300001219B68002098472B6800219B68204649
:1036400098472B6800219B68084698472B68002103
:1036500004029B68084698472B68002104439B6836
:10366000084698472B68240204439B6801210020E8
:1036700098472402204338BDEC48FF1F884BFF1FAA
:10368000844BFF1F10B50C4601460020FFF7ABFF2F
:10369000206010BD38B50D462021814041F0010168
:1036A000C9B20446FFF79FFF2968014429602046FC
:1036B000BDE838403BE71C2A2DE9F84304460D4697
:1036C0001E4600F0B98300F2A6800C2A00F07A8230
:1036D0004AD8052A00F0FF8119D8022A00F0AA81F1
:1036E00007D8002A00F07081012A00F089810424A3
:1036F00074E1032A00F0BB81042AF8D1002840F0CD
:10370000CB81CB4800EB8100C369336066E1082AB6
:1037100000F0388213D8062A00F0F681072AE6D195
:10372000002840F017822021A94041F01001C9B2C1
:103730002846FFF758FF00F01F0030604EE10A2ACC
:1037400000F02E820B2AD2D1002840F0A181202146
:10375000A94041F01501C9B22846FFF744FFC04314
:1037600000F00100306039E1122A00F0C78227D84A
:103770000F2A00F0838211D80D2A00F04A820E2A07
:10378000B5D1002840F06C822021A94041F01401FD
:10379000C9B22846FFF727FF30601FE1102A00F06A
:1037A0008682112AA3D1002840F09A822021A940C4
:1037B00041F00801C9B22846FFF715FF30600DE15E
:1037C000152A00F0DF8211D8132A00F0B082142AE3
:1037D0008DD1002840F0C8822021A94041F00B0182
:1037E000C9B22846FFF7FFFE3060F7E0172A00F065
:1037F000FC82C0F0E082182A7FF479AF002840F004
:103800000D832021A94041F01301C9B22846FFF7DA
:10381000EAFE3060E2E0AC2A00F0258562D8A52AF5
:1038200000F0F68331D8A22A00F0908318D81D2A20
:1038300000F027838C2A7FF45AAF002840F02F83B2
:10384000090141F06C0101F0FC012846FFF7CBFEB5
:103850004FF48073C0F3036043FA00F03060BDE0C2
:10386000A32A00F09883A42A7FF441AF002840F0F7
:10387000B783090141F06C0101F0FC012846FFF714
:10388000B2FEC0F300303060A8E0A82A00F05F84E8
:1038900014D8A62A00F00484A72A7FF428AF0028B1
:1038A00040F03E84090141F06C0101F0FC01284622
:1038B000FFF799FE00F00F0030608FE0AA2A00F0B9
:1038C000928440F26884002840F0B484090141F0F9
:1038D0006D0101F0FD012846FFF785FEC0F34110A0
:1038E00030607BE0B62A00F066823ED8B32A00F052
:1038F00020851BD8AD2A00F0DC84AE2A7FF4F7AE19
:10390000002840F0FD84090141F06D0101F0FD0146
:103910002846FFF768FE001400F07F0310F0400017
:1039200018BF6FF07F001843306057E0B42A00F0F2
:103930002785B52A7FF4DBAE20278F407FB247F082
:1039400014085FFA88F841462846FFF74CFE002C21
:1039500040F02885410540F1228547F01101C9B2A8
:103960002846FFF740FE306038E0CE2A00F0788528
:1039700014D8B82A00F03485B92A7FF4B8AE0028EC
:1039800040F05585090141F06C0101F0FC01284629
:10399000FFF729FEC0F3035030601FE0D22A00F089
:1039A0007D85D32A00F09585D12A7FF4A0AE00282A
:1039B00040F065852021A94041F01901C9B228468F
:1039C000FFF711FE306009E058B92021A94041F00D
:1039D0000D01C9B22846FFF706FE30602046BDE85B
:1039E000F883012801D00024F8E72021A94041F004
:1039F0000D011A68C9B22846FFF786FD0024EDE7DD
:103A000048B92021A94041F00101C9B22846FFF779
:103A1000EAFD3060E2E70128E5D12021A94041F02C
:103A200001011A68C9B22846FFF76EFD0024D5E7E8
:103A30002817FF1F48B92021A94041F00701C9B24A
:103A40002846FFF7D0FD3060C8E70128CBD13268A7
:103A5000BC4B2021A940002A41F007015855B8BFAE
:103A60005242C9B22846FFF74FFD0024B6E778B9A5
:103A70002021A94041F00201C9B22846FFF7B3FD59
:103A800010F4000318BF4FF07F4318433060A5E7E0
:103A9000012CA8D10424A1E70128A4D13268AA4BA3
:103AA000202703EB8103002A07FA01F7B8BF52422F
:103AB000F9B22846DA61FFF796FD0446002892D154
:103AC000326847F00701002AB8BF5242C9B22846FF
:103AD000FFF71AFD82E748B92021A94041F006010D
:103AE000C9B22846FFF77FFD306077E701287FF4F1
:103AF0007AAF2021A94041F006011A68C9B22846D0
:103B0000FFF702FD002469E758B92021A94041F0E0
:103B10001001C9B22846FFF766FDC0F304203060EB
:103B20005CE701287FF45FAF20248C4044F0100450
:103B3000E4B221462846FFF756FD33681B0203F422
:103B4000F85320F4F85221461A432846FFF7DCFCCC
:103B5000002443E701287FF446AF20248C4044F042
:103B60001004E4B221462846FFF73DFD336820F0FB
:103B70001F0203F01F0321461A432846FFF7C4FC27
:103B800000242BE7002883D12021A94041F0150112
:103B9000C9B22846FFF727FDC0F3402030601DE77B
:103BA00000287FF475AF2021A94041F01501C9B26A
:103BB0002846FFF718FD10F0020F0CBF0123002369
:103BC00033600BE758B92021A94041F01401C9B274
:103BD0002846FFF708FDC0F340003060FEE60128EC
:103BE0007FF401AF20248C4044F01404E4B2214659
:103BF0002846FFF7F8FC3368002B20F0020214BFC0
:103C00000023022321461A432846FFF77DFC0024A7
:103C1000E4E658B92021A94041F01401C9B2284670
:103C2000FFF7E1FC00F001003060D7E601287FF4E7
:103C3000DAAE20248C4044F01404E4B22146284635
:103C4000FFF7D1FC326820F00100002A14BF0246C1
:103C500040F0010221462846FFF756FC0024BDE64D
:103C600001287FF4C0AE2021A94041F014011A6858
:103C7000C9B22846FFF748FC0024AFE648B9202126
:103C8000A94041F00401C9B22846FFF7ACFC3060FE
:103C9000A4E601287FF4A7AE2021A94041F0040149
:103CA0001A68C9B22846FFF72FFC002496E648B9E7
:103CB0002021A94041F00501C9B22846FFF793FC35
:103CC00030608BE601287FF48EAE2021A94041F0C0
:103CD00005011A68C9B22846FFF716FC00247DE6E4
:103CE00001287FF480AE2021A94041F008011A6824
:103CF000C9B22846FFF708FC00246FE648B9202126
:103D0000A94041F00A01C9B22846FFF76CFC3060B7
:103D100064E601287FF467AE2021A94041F00A0142
:103D20001A68C9B22846FFF7EFFB002456E668B9C7
:103D30002021A94041F00301C9B22846FFF753FCF6
:103D400030604BE67000FF1F2817FF1F01287FF42B
:103D50004AAE2021A94041F003011A68C9B22846A1
:103D6000FFF7D2FB002439E601287FF43CAE202186
:103D7000A94041F00B011A68C9B22846FFF7C4FBFD
:103D800000242BE648B92021A94041F00C01C9B21A
:103D90002846FFF728FC306020E601287FF423AE98
:103DA0002021A94041F00C011A68C9B22846FFF74A
:103DB000ABFB002412E654B92021A94041F01101C7
:103DC000C9B22846FFF70FFC0024306006E6012C3C
:103DD0007FF409AE2021A94041F011013268C9B237
:103DE0002846FFF791FB0024F8E548B92021A940B7
:103DF00041F01201C9B22846FFF7F5FB3060EDE54E
:103E000001287FF4F0AD2021A94041F012011A6889
:103E1000C9B22846FFF778FB0024DFE501287FF4CC
:103E2000E2AD2021A94041F013011A68C9B2284629
:103E3000FFF76AFB0024D1E558B9090141F06C0194
:103E400001F0FC012846FFF7CEFBC0F38040306054
:103E5000C4E501287FF4C7AD0C0144F06C04E4B262
:103E600021462846FFF7BFFB33689B0403F48023F9
:103E700020F4802221461A432846FFF745FB002400
:103E8000ACE500287FF404AEC94B20201B688840B5
:103E900040F0020003EB8000436833609EE5012898
:103EA0007FF4A1AD1B68102B23D00DDC022B1CD09E
:103EB00004DC012B16D04FF0FF3314E0042B16D096
:103EC000082BF8D105230EE0402B14D003DC202B67
:103ED000F1D1032307E0802B0FD0B3F5807FEAD127
:103EE000002300E00823336008E00723FBE70623F4
:103EF000F9E70423F7E70223F5E73060336801337D
:103F00003FF471AD2C0144F06C04E4B22146284624
:103F1000FFF769FB33681B0603F0706320F07062E3
:103F20001A4321462846FFF7EFFA21462846FFF7B5
:103F30005AFB33681B0603F0706320F07062214661
:103F40001A432846FFF7E0FA002447E558B909016B
:103F500041F06C0101F0FC012846FFF744FBC0F37F
:103F6000C13030603AE501287FF43DAD0C0144F0EA
:103F70006C04E4B221462846FFF735FB3368DB03C7
:103F800003F4C03320F4C03221461A432846FFF719
:103F9000BBFA002422E558B9090141F06C0101F097
:103FA000FC012846FFF71FFBC0F38030306015E5A9
:103FB00001287FF418AD0C0144F06C04E4B22146F2
:103FC0002846FFF710FB33689B0303F4804320F47B
:103FD000804221461A432846FFF796FA0024FDE462
:103FE00001287FF400AD0C0144F06C04E4B22146DA
:103FF0002846FFF7F8FA33681B0303F4805320F4D4
:10400000805221461A432846FFF77EFA0024E5E451
:104010000F0147F06C07FFB239462846FFF7E3FA75
:104020008046C4B918F480493946284605D0FFF7C0
:10403000DAFAC0F3C3103060D0E4FFF7D4FA18F412
:10404000006FC0F3021001D13060CCE440F00800F2
:1040500030604C46C2E4012C7FF4C5AC18F48044B7
:10406000394628460ED0FFF7BEFA3368DB0103F469
:10407000F06320F4F0621A4339462846FFF744FA09
:104080000024ABE4FFF7AFFA33681B0103F07003C1
:1040900020F070021A4339462846FFF735FA9DE4AE
:1040A0000F0147F06C07FFB239462846FFF79BFA2D
:1040B0008CB910F480443946284606D0FFF793FAAD
:1040C000C0F302103060002488E4FFF78CFAC0F3DC
:1040D000C310306082E4012C7FF485AC10F480447E
:1040E000394628460ED0FFF77EFA33681B0103F0ED
:1040F000700320F070021A4339462846FFF704FA8D
:1041000000246BE4FFF76FFA3368DB0103F4F0631C
:1041100020F4F0621A4339462846FFF7F5F95DE4CA
:1041200001287FF460AC0C0144F06C04E4B2214639
:104130002846FFF758FA336820F00F0203F00F0308
:1041400021461A432846FFF7DFF9002446E458B910
:10415000090141F06D0101F0FD012846FFF743FA26
:10416000C0F3C030306039E401287FF43CAC0C016E
:1041700044F06D04E4B221462846FFF734FA336870
:10418000DB039BB220F4004221461A432846FFF786
:10419000BBF9002422E468B9090141F06D0101F086
:1041A000FD012846FFF71FFAC0F34130306015E4E7
:1041B000884BFF1F01287FF416AC0C0144F06D04FE
:1041C000E4B221462846FFF70EFA33685B0303F496
:1041D000C04320F4C04221461A432846FFF794F911
:1041E0000024FFF7FBBB60B9090141F06D0101F04C
:1041F000FD012846FFF7F7F9C0F303203060FFF711
:10420000EDBB01287FF4EFAB0C0144F06D04E4B288
:1042100021462846FFF7E7F933681B0203F4706371
:1042200020F4706221461A432846FFF76DF90024F6
:10423000FFF7D4BB01287FF4D6AB0C0144F06D042A
:10424000E4B221462846FFF7CEF933685B0103F05C
:10425000600320F0600221461A432846FFF754F914
:104260000024FFF7BBBB60B9090141F06D0101F00B
:10427000FD012846FFF7B7F900F00F003060FFF7A7
:10428000ADBB01287FF4AFAB0C0144F06D04E4B288
:1042900021462846FFF7A7F9336820F00F0203F004
:1042A0000F0321461A432846FFF72EF90024FFF793
:1042B00095BB60B9090141F06D0101F0FD0128468F
:1042C000FFF791F9C0F300603060FFF787BB01286A
:1042D0007FF489AB0C0144F06D04E4B2214628461A
:1042E000FFF781F933681B0603F0807320F08072BA
:1042F00021461A432846FFF707F90024FFF76EBB53
:1043000001287FF470AB0C0144F06D04E4B2214647
:104310002846FFF768F933681B0403F4FE0320F412
:10432000FE0221461A432846FFF7EEF80024FFF765
:1043300055BB60B9090141F06C0101F0FC01284650
:10434000FFF751F9C0F340403060FFF747BB012849
:104350007FF449AB0C0144F06C04E4B221462846DA
:10436000FFF741F933685B0403F4003320F40032B3
:1043700021461A432846FFF7C7F80024FFF72EBB53
:1043800000287FF485AB090141F06F01C9B22846CE
:10439000FFF729F9C0F304403060FFF71FBB34601A
:1043A000FFF71CBB012C7FF41EAB47F011013268F4
:1043B000C9B22846FFF7A8F841462846FFF713F987
:1043C0003368002B20F480620CBF00234FF480631D
:1043D0001A4341462846FFF797F80024FFF7FEBA34
:1043E00060B9090141F06C0101F0FC012846FFF7BA
:1043F000FAF8C0F340303060FFF7F0BA01287FF4DC
:10440000F2AA0C0144F06C04E4B221462846FFF7FE
:10441000EAF833685B0303F4005320F400522146AA
:104420001A432846FFF770F80024FFF7D7BA01288F
:104430007FF4D9AA0C0144F06C04E4B2214628466A
:10444000FFF7D1F833681B0503F4700320F4700202
:1044500021461A432846FFF757F80024FFF7BEBA53
:1044600000287FF415AB090141F06F01C9B228465D
:10447000FFF7B9F8C0F309003060FFF7AFBA0128C1
:104480007FF4B1AA2021A94041F019011A68C9B2EC
:104490002846FFF739F80024FFF7A0BA50B92021C9
:1044A000A94041F01A01C9B22846FFF79CF83060D4
:1044B000FFF794BA01287FF496AA2021A94041F081
:1044C0001A011A68C9B22846FFF71EF80024FFF740
:1044D00085BAE8B979B101297FF480AA0146284656
:1044E000FFF781F800F06000A0F120035842584126
:1044F0003060FFF773BA0846FFF775F800F0180050
:10450000A0F110025042504130602C46FFF766BACD
:1045100001287FF468AA21B1012917D00024FFF7F0
:104520005DBA0846FFF75FF8336853B120F0080220
:1045300042F0100200210846FEF7E6FF0024FFF7D4
:104540004DBA20F0100242F00802F3E7002128469D
:10455000FFF749F8336853B120F0400242F02002DF
:1045600000210120FEF7D0FF0024FFF737BA20F02A
:10457000200242F04002F3E707B50129019207D873
:10458000024601AB0120FFF796F803B05DF804FB8B
:104590000820FAE70129134603D802460020FFF756
:1045A0008AB80820704708B522210020FFF71BF8C1
:1045B00050B942210120FFF716F828B9034B1868BB
:1045C000BDE808400CF06EBC002008BD884BFF1F02
:1045D00070B53D4E3D483E4C0CF0CCFBF5686B6829
:1045E00003F58272626003F59272A26003F5717244
:1045F000E26003F5797203F16400226103F2044280
:1046000003F22443A3612B686261DB682060984752
:104610002B68E068DB6898472B68E0689B699847DF
:104620002B6860681B6998472B68A0681B699847CE
:104630002B68A0691B6998472B6820691B699847FC
:104640002B6860691B699847224B32691A606B6856
:10465000214903F531735360204B5A690A602049A0
:10466000C2F804121F49C2F808120120002110707C
:1046700051701D4A1A621D4ADA611D4A9A611D4A2B
:104680005A621D4A9A631D4A5A631D4A9A621D4A1C
:10469000DA621D4A9A641D4A5A641D4A5A651D4AC7
:1046A0001A651D4ADA641D4A1A661D4ADA65022235
:1046B0001A743222DA60B6229A601A4A9A65BDE804
:1046C0007040FEF79FBE00BF704C0200EC48FF1F19
:1046D0002817FF1F844BFF1F884BFF1F7431FF1FDC
:1046E000A74501007533010091350100E535010052
:1046F000E1350100DD3501009545010079450100F6
:104700002F35010095360100253501008536010061
:1047100049330100A9330100813301000534010050
:104720003D3301004534010001289FBF034B53F87E
:1047300020300B60002088BF08207047944BFF1F7B
:10474000014B00225A6070477431FF1F70B5084E4C
:10475000084D336804462A46014600200CF0F0FB61
:1047600033682A4621460120BDE870400CF0E8BBC2
:104770008C4BFF1F944BFF1F014B18680CF02BBC98
:104780008C4BFF1F012810B5144603D002280ED011
:10479000042010BD094B0A4ADB6850681B681B6A7D
:1047A0009847003018BF01202060002010BD034B47
:1047B000034ADB6890681B681B6AF1E7704C0200D3
:1047C0005817FF1F022804BF0B4B93F8D00030B9D5
:1047D0000A4BDB681B685B69094A106818470128A7
:1047E00009D1054B93F8D030012B04D1034BDB6882
:1047F0001B689B69F0E770477431FF1F704C020023
:104800005817FF1F70B50020FFF7DCFF084B094C5D
:10481000DD6820682B689B6898472B6860689B68F8
:1048200098472B68A0689B68BDE87040184700BF98
:10483000704C02005817FF1F2DE9F843184C9DF8E3
:1048400020609DF82450984623680F469B680021FD
:1048500047F0800091469847236800219B684846AE
:104860009847236800219B684046984723680021A9
:104870009B6830469847236828469B6801219847E3
:10488000084B1B6848EA092807F07F0746EA082614
:1048900003EB870745EA06257D60BDE8F88300BF86
:1048A000904BFF1F8C4BFF1F07B5D3B20193C2F390
:1048B00007230093C2F30743120EFFF7BDFF03B0B7
:1048C0005DF804FB0A4601460020FFF7EDBF012812
:1048D000F7B505460F4628D8154C044494F8943291
:1048E00073B1144B202181401B6841F0070103EB99
:1048F0008103C9B25A68FFF7D7FF002384F89432C6
:104900002026AE4046F00D0100243A46C9B22846A2
:10491000FFF7CAFF28460194009423462246F1B2CD
:10492000FFF78AFF204603B0F0BD0820FBE700BF79
:10493000944BFF1F8C4BFF1F012873B505460C4697
:1049400021D82026864084EAE47246F00701A2EBD3
:10495000E472C9B2FFF7A8FF0C4B2B44002C4FF0B8
:10496000010283F894224FF00004ACBF13460223E7
:1049700001932846009423462246F1B2FFF75CFFDC
:10498000204602B070BD0820FBE700BF944BFF1F1C
:104990000021D1E74942CFE7CEE738B5234B01F0FC
:1049A0007F04234493F81432DB0705D4204B1B68A3
:1049B00003EB8404606838BD1E4D2B6800219B68A2
:1049C000204698472B6800219B68084698472B682B
:1049D00000219B68084698472B6800219B68084681
:1049E00098472B6801219B68002098472B6800217D
:1049F0009B68204698472B6800219B68084698478B
:104A00002B68002104029B68084698472B68002108
:104A100004439B68084698472B68240204439B681C
:104A20000121002098472402204338BD944BFF1FEA
:104A30008C4BFF1F904BFF1F10B50C46014600200A
:104A4000FFF7ABFF206010BD38B50D462021814037
:104A500041F00101C9B20446FFF79FFF29680144F4
:104A600029602046BDE8384031E71C2A2DE9F04195
:104A700004460D461E4600F0118300F294800C2A75
:104A800000F027824DD8052A00F0C7811ED8022ADF
:104A900000F0728107D8002A00F04A81012A00F054
:104AA0005E8104244EE1032A00F07F81042AF8D1BC
:104AB000002840F09381C74B20201B68884040F0BD
:104AC000070003EB8000436833603BE1082A00F0F5
:104AD000E38112D8062A00F0AD81072AE1D100282F
:104AE00040F0C8812021A94041F01001C9B22846F8
:104AF000FFF753FF00F01F0023E10A2A00F0D981DD
:104B00000B2ACED1002840F060812021A94041F03D
:104B10001501C9B22846FFF740FFC04300F001006D
:104B20000FE1122A00F05F821DD80F2A00F03782B1
:104B30000CD80D2A00F0FD810E2AB2D1002840F0D9
:104B400026822021A94041F01401F6E0102A00F04D
:104B50003482112AA5D1002840F03D822021A940AD
:104B600041F00801E9E0152A00F061820CD8132A0F
:104B700000F04782142A94D1002840F0508220216E
:104B8000A94041F00B01D8E0172A00F07182C0F073
:104B90005C82182A85D1002840F078822021A94023
:104BA00041F01301C9E0AB2A00F00D845ED8A52ABC
:104BB00000F02E832FD8A22A00F0DC8217D81D2AFD
:104BC00000F08A828C2A7FF46CAF002840F090823B
:104BD000090141F06C0101F0FC012846FFF7DDFE00
:104BE0004FF48073C0F3036043FA00F0A9E0A32AF6
:104BF00000F0DE82A42A7FF454AF002840F0F68251
:104C0000090141F06C0101F0FC012846FFF7C5FEE7
:104C1000C0F3003095E0A82A00F0888312D8A62AB5
:104C200000F03F83A72A7FF43CAF002840F06F8359
:104C3000090141F06C0101F0FC012846FFF7ADFECF
:104C400034607FE0A92A00F08E83AA2A7FF429AF7E
:104C5000002840F0A683090141F06D0101F0FD013B
:104C60002846FFF79AFEC0F303206AE0B52A00F059
:104C700039842AD8AE2A00F0F38313D8AC2A00F086
:104C8000C083AD2A7FF40DAF002840F0D78309011F
:104C900041F06D0101F0FD012846FFF77EFEC0F3F3
:104CA00000604EE0B32A00F0FF83B42A7FF4F9AE2F
:104CB000002840F08A80090141F06F01C9B22846FE
:104CC000FFF76BFEC0F304403BE0CE2A00F03C84CB
:104CD00013D8B62A00F0B981B82A7FF4E2AE0028D2
:104CE00040F02084090141F06C0101F0FC012846EC
:104CF000FFF753FEC0F3403023E0D12AFFF4D1AEDA
:104D0000D22A24D9D32A7FF4CCAE002840F03484B0
:104D1000002900F02784012914D101462846FFF715
:104D20003CFE00F06000A0F120035842584108E02A
:104D300058B92021A94041F00D01C9B22846FFF71A
:104D40002CFE30602046BDE8F081012801D000240F
:104D5000F8E72021A94041F00D01326820E020B998
:104D60002021A94041F00101E7E70128EFD12021EE
:104D7000A94041F00101F0E720B92021A94041F00C
:104D80000701DAE70128E2D1134B0B44202183F815
:104D900094023268A940002A41F00701B8BF52428C
:104DA000C9B22846FFF780FDD1E770B92021A9409C
:104DB00041F00201C9B22846FFF7EFFD10F40003ED
:104DC00018BF4FF07F431843BBE7012C3FF469AE97
:104DD000BDE700BF8C4BFF1F944BFF1F0128B6D1CE
:104DE000C14B32681B682021A94041F0070703EB43
:104DF0008703002AB8BF52425A60C9B22846FFF75B
:104E0000CCFD04460028A2D13268002AB8BF524225
:104E1000F9B22846FFF748FD94E720B92021A940C0
:104E200041F0060189E7012891D12021A94041F0F4
:104E3000060192E750B92021A94041F01001C9B202
:104E40002846FFF7AAFDC0F304207AE701287FF483
:104E50007EAF20248C4044F01004E4B22146284662
:104E6000FFF79BFD33681B0203F4F85320F4F8525C
:104E70001A4359E201287FF46AAF20248C4044F0A1
:104E80001004E4B221462846FFF787FD336820F07E
:104E90001F0203F01F03EBE7002896D12021A94051
:104EA00041F01501C9B22846FFF777FDC0F3402055
:104EB00047E7002889D12021A94041F01501C9B256
:104EC0002846FFF76AFD10F0020F0CBF01230023F4
:104ED000FAE550B92021A94041F01401C9B2284691
:104EE000FFF75BFDC0F340002BE701287FF42FAFF5
:104EF00020248C4044F01404E4B221462846FFF7F5
:104F00004CFD3368002B0CBF0023022320F002026B
:104F10001A4321462846FFF7C7FC21462846FFF7DB
:104F20003CFD3368022B20F0080214BF0023082345
:104F30009EE740B92021A94041F01401C9B228469A
:104F4000FFF72BFDEAE501287FF401AF20248C4018
:104F500044F01404E4B221462846FFF71EFD3268EF
:104F600020F00100002A0CBF024640F00102214659
:104F70002846FFF799FC21462846FFF70EFD3368C7
:104F8000022B20F0040214BF0023042370E7012841
:104F90007FF4DDAE2021A94041F01401DDE620B907
:104FA0002021A94041F00401C7E601287FF4CFAEDB
:104FB0002021A94041F00401CFE620B92021A940D9
:104FC00041F00501B9E601287FF4C1AE2021A940D6
:104FD00041F00501C1E601287FF4B9AE2021A940C6
:104FE00041F00801B9E620B92021A94041F00A01A9
:104FF000A3E601287FF4ABAE2021A94041F00A01CD
:10500000ABE620B92021A94041F0030195E6012833
:105010007FF49DAE2021A94041F003019DE60128C7
:105020007FF495AE2021A94041F00B0195E620B90F
:105030002021A94041F00C017FE601287FF487AED2
:105040002021A94041F00C0187E64CB92021A9405C
:1050500041F01101C9B22846FFF79FFC306076E6A7
:10506000012C7FF474AE2021A94041F0110174E6B7
:1050700020B92021A94041F012015EE601287FF409
:1050800066AE2021A94041F0120166E601287FF4B6
:105090005EAE2021A94041F013015EE650B909013E
:1050A00041F06C0101F0FC012846FFF776FCC0F3EB
:1050B000804046E601287FF44AAE0C0144F06C04BF
:1050C000E4B221462846FFF768FC33689B0403F4EA
:1050D000802320F48022CBE600287FF476AE034BB9
:1050E00053F82130F0E400BF8C4BFF1F944BFF1F9F
:1050F00001287FF42CAE1B68102B23D00DDC022B73
:105100001CD004DC012B16D04FF0FF3314E0042B2D
:1051100016D0082BF8D105230EE0402B14D003DC69
:10512000202BF1D1032307E0802B0FD0B3F5807F34
:10513000EAD1002300E00823336008E00723FBE7FF
:105140000623F9E70423F7E70223F5E73060336825
:1051500001333FF4FCAD2C0144F06C04E4B2214671
:105160002846FFF71AFC33681B0603F0706320F033
:1051700070627DE650B9090141F06C0101F0FC015B
:105180002846FFF70AFCC0F3C130DAE501287FF4B6
:10519000DEAD0C0144F06C04E4B221462846FFF772
:1051A000FCFB3368DB0303F4C03320F4C0325FE65A
:1051B00050B9090141F06C0101F0FC012846FFF7EC
:1051C000ECFBC0F38030BCE501287FF4C0AD0C01DE
:1051D00044F06C04E4B221462846FFF7DEFB336856
:1051E0009B0303F4804320F4804241E601287FF4CE
:1051F000AEAD0C0144F06C04E4B221462846FFF742
:10520000CCFB33681B0303F4805320F480522FE659
:105210000F0147F06C07FFB239462846FFF7BDFB88
:1052200094B910F4804206D039462846FFF7B5FB02
:10523000C0F3C31085E5031103F07003010548BFF7
:1052400043F00803336082E5012C7FF480AD10F455
:105250008044394628460AD0FFF79FFB3368DB01BC
:1052600003F4F06320F4F0621A43394699E5FFF73E
:1052700094FB336813F0080F20F4006218BF4FF45A
:105280000064394628462243FFF70EFB394628467C
:10529000FFF783FB33681B0103F0700320F07002FB
:1052A000E2E70F0147F06C07FFB239462846FFF7E7
:1052B00074FB8046A4B918F480443946284604D0CB
:1052C000FFF76BFBC0F30210C8E6FFF766FB18F4AC
:1052D000006FC0F3C3103FF4C1AE40F0080030E5EA
:1052E000012C7FF434AD39462846FFF756FB10F405
:1052F000804439462846CBD1FFF74FFB3368DB01AA
:1053000003F4F06320F4F0621A43394681E5012882
:105310007FF41DAD0C0144F06C04E4B22146284634
:10532000FFF73BFB20F00F0221463AE550B9090197
:1053300041F06D0101F0FD012846FFF72EFBC0F39F
:10534000C030FEE401287FF402AD0C0144F06D048E
:10535000E4B221462846FFF720FB3368DB039BB20B
:1053600020F4004284E550B9090141F06D0101F0DB
:10537000FD012846FFF711FBC0F34130E1E40128AD
:105380007FF4E5AC0C0144F06D04E4B221462846FC
:10539000FFF703FB33685B0303F4C04320F4C04210
:1053A00066E501287FF4D3AC0C0144F06D04E4B24F
:1053B00021462846FFF7F1FA33681B0203F47063B5
:1053C00020F4706254E550B9090141F06D0101F01B
:1053D000FD012846FFF7E1FAC0F34110B1E40128CE
:1053E0007FF4B5AC0C0144F06D04E4B221462846CC
:1053F000FFF7D3FA33685B0103F0600320F060022B
:1054000036E550B9090141F06D0101F0FD01284672
:10541000FFF7C3FA00F00F0093E401287FF497AC84
:105420000C0144F06D04E4B221462846FFF7B5FABA
:10543000336820F00F0203F00F0319E501287FF411
:1054400086AC0C0144F06D04E4B221462846FFF717
:10545000A4FA33681B0603F0807320F0807207E51E
:1054600080B9090141F06D0101F0FD012846FFF707
:1054700094FA001400F07F0310F0400018BF6FF0A2
:105480007F00A0E401287FF462AC0C0144F06D04BD
:10549000E4B221462846FFF780FA33681B0403F480
:1054A000FE0320F4FE02E3E450B9090141F06C016F
:1054B00001F0FC012846FFF770FAC0F3404040E4D9
:1054C00001287FF444AC0C0144F06C04E4B22146A2
:1054D0002846FFF762FA33685B0403F4003320F4D4
:1054E0000032C5E400283FF4B1AD01287FF42FACB1
:1054F00020248C4064B244F0110144F014041A6872
:10550000C9B22846E4B2FFF7CFF921462846FFF793
:1055100044FA3368002B20F480620CBF00234FF460
:105520008063A5E401287FF412AC0C0144F06C0404
:10553000E4B221462846FFF730FA33685B0303F4F0
:10554000005320F4005293E400287FF43EAC09019C
:1055500041F06F01C9B22846FFF71FFAC0F30900F6
:10556000FFF7EFBB0846FFF718FA00F01800A0F1AC
:1055700010025042504171E501287FF4E8AB79B147
:1055800001297FF4E4AB00212846FFF706FA3368CF
:1055900020F06002A3B142F020020021012001E4CA
:1055A0000846FFF7FAF9336820F018022BB142F0F1
:1055B000100200210846FFF7F5BB42F00802F8E7A9
:1055C00042F04002E9E707B50129019207D80246F7
:1055D00001AB0120FFF749FA03B05DF804FB082096
:1055E000FAE70129134603D802460020FFF73DBA27
:1055F0000820704708B522210020FFF7CEF950B9E6
:1056000042210120FFF7C9F928B9044B1868BDE809
:1056100008400BF0D7BC002008BD00BF8C4BFF1F1B
:1056200070B52D4E2D482E4D0BF04CFCF468636880
:1056300003F5827203F1640003F59273AB60236893
:105640006A60DB6828609847236868681B69984728
:105650002368A8681B699847224B32691A606368FF
:10566000214903F531735360204B5A690A60204980
:10567000C2F804121F49C2F808120121117000215A
:1056800051701D4A1A621D4ADA611D4A9A611D4A0B
:105690005A621D4A9A631D4A5A631D4A9A621D4AFC
:1056A000DA621D4A9A641D4A5A641D4A5A651D4AA7
:1056B0001A651D4ADA641D4A1A661D4ADA653222E5
:1056C000DA6002204FF48C729A601874194A9A6555
:1056D000BDE87040FFF776B8704C0200944BFF1F96
:1056E0005817FF1F904BFF1F8C4BFF1F7431FF1F7C
:1056F000F555010079470100394901009949010038
:105700009549010091490100E3550100C755010089
:10571000CF480100494A0100C5480100394A01004B
:105720004D4701008547010029470100C547010099
:10573000414701000548010001289FBF034B53F872
:1057400020300B60002088BF08207047304EFF1FBC
:10575000014B00225A6070477431FF1F70B5084E2C
:10576000084D336804462A46014600200BF07AFCB7
:1057700033682A4621460120BDE870400BF072BC18
:105780002C4EFF1F304EFF1F014B18680BF0CDBC95
:105790002C4EFF1F012810B5144611D003D3022848
:1057A0001AD0042010BD14680F4A104BD26812683A
:1057B00024B15269D8689047002010BD9269F9E77A
:1057C000094B0A4ADB6850681B681B6A984700301F
:1057D00018BF01202060EFE7034B044ADB689068A4
:1057E0001B681B6AF2E700BF704C02007017FF1FB6
:1057F000022804BF0B4B93F8D00030B90A4BDB688A
:105800001B685B69094A10681847012809D1054BD4
:1058100093F8D030012B04D1034BDB681B689B69E4
:10582000F0E770477431FF1F704C02007017FF1FC4
:1058300070B50020FFF7DCFF104B114CDD682068CD
:105840002B689B6898472B6860689B6898472B6813
:10585000A0689B6898472B68A0699B6898472B684D
:1058600020699B6898472B6860699B6898472B68FC
:10587000E0689B68BDE87040184700BF704C0200AC
:105880007017FF1F38B5244B00F07F04234493F8B2
:105890001432DB0705D4214B1B6803EB84046068DA
:1058A00038BD1F4D2B6800219B68204698472B6808
:1058B00000219B68084698472B6800219B68084692
:1058C00098472B6800219B68084698472B68012160
:1058D0009B68002098472B6800219B6820469847CA
:1058E0002B6800219B68084698472B68002104021A
:1058F0009B68084698472B68002104439B6808462C
:1059000098472B68240204439B6801210020984794
:105910002402204338BD00BF304EFF1F2C4EFF1F16
:10592000C850FF1F08B52220FFF7ACFF48B942203E
:10593000FFF7A8FF28B9044B1868BDE808400BF032
:10594000EBBB002008BD00BF2C4EFF1F10B50C465E
:10595000FFF798FF206010BD2DE9F843184C9DF823
:1059600020609DF82450984623680F469B680021CC
:1059700047F0800091469847236800219B6848467D
:105980009847236800219B68404698472368002178
:105990009B6830469847236828469B6801219847B2
:1059A000084B1B6848EA092807F07F0746EA0826E3
:1059B00003EB870745EA06257D60BDE8F88300BF55
:1059C000C850FF1F2C4EFF1F07B5D3B20193C2F37F
:1059D00007230093C2F30743120EFFF7BDFF03B086
:1059E0005DF804FB0A4601460020FFF7EDBF0128E1
:1059F000F7B505460F4628D8154C044494F8943260
:105A000073B1144B202181401B6841F0070103EB67
:105A10008103C9B25A68FFF7D7FF002384F8943294
:105A20002026AE4046F00D0100243A46C9B2284671
:105A3000FFF7CAFF28460194009423462246F1B29C
:105A4000FFF78AFF204603B0F0BD0820FBE700BF48
:105A5000304EFF1F2C4EFF1F38B504462020A040BB
:105A600040F001000D46C0B2FFF70CFF2B68C118D3
:105A700029602046BDE83840B9E7012873B50546DE
:105A80000C4621D82026864084EAE47246F00701BD
:105A9000A2EBE472C9B2FFF797FF0C4B2B44002C2A
:105AA0004FF0010283F894224FF00004ACBF13467C
:105AB000022301932846009423462246F1B2FFF7C1
:105AC0004BFF204602B070BD0820FBE7304EFF1FA1
:105AD0000021D2E74942D0E7CFE71C2AF8B50446B7
:105AE0000D461E4600F0958300F2A5800C2A00F0BA
:105AF00064824DD8052A00F0EF811ED8022A00F0FA
:105B0000988107D8002A00F06381012A00F07A8189
:105B1000042466E1032A00F0AD81042AF8D10028AC
:105B200040F0BC81C84B20201B68884040F0070033
:105B300003EB80004368336053E1082A00F01F82C2
:105B400012D8062A00F0E081072AE1D1002840F0AF
:105B5000FF812020884040F01000C0B2FFF792FE85
:105B600000F01F0030603CE10A2A00F015820B2A89
:105B7000CED1002840F08E812020884040F01500D2
:105B8000C0B2FFF77FFEC04300F00100306028E1A3
:105B9000122A00F0A58225D80F2A00F0638210D8BF
:105BA0000D2A00F02E820E2AB2D1002840F04C823D
:105BB0002020884040F01400C0B2FFF763FE306040
:105BC0000FE1102A00F06682112AA1D1002840F0CE
:105BD00079822020884040F00800C0B2FFF752FED2
:105BE0003060FEE0152A00F0BD8210D8132A00F0C4
:105BF0008F82142A8CD1002840F0A6822020884071
:105C000040F00B00C0B2FFF73DFE3060E9E0172A1C
:105C100000F0D982C0F0BE82182A7FF479AF002844
:105C200040F0E9822020884040F01300C0B2FFF726
:105C300029FE3060D5E0AC2A00F001855ED8A52AA7
:105C400000F0B6832FD8A22A00F0558317D81D2A5A
:105C500000F002838C2A7FF45BAF002840F00483BD
:105C6000080140F06C0000F0FC00FFF70BFE4FF461
:105C70008073C0F3036043FA00F03060B1E0A32A00
:105C800000F05C83A42A7FF443AF002840F07983BE
:105C9000080140F06C0000F0FC00FFF7F3FDC0F3DA
:105CA000003030609DE0A82A00F0458413D8A62A71
:105CB00000F0DD83A72A7FF42BAF002840F0258475
:105CC000080140F06C0000F0FC00FFF7DBFD00F085
:105CD0000F00306085E0AA2A00F0758440F25084FD
:105CE000002840F09484080140F06D0000F0FD00B1
:105CF000FFF7C8FDC0F34110306072E0B62A00F033
:105D0000498238D8B32A00F0FB841AD8AD2A00F0B3
:105D1000BA84AE2A7FF4FCAE002840F0D984080192
:105D200040F06D0000F0FD00FFF7ACFD001400F046
:105D30007F0310F0400018BF6FF07F001843306001
:105D40004FE0B42A00F00185B52A7FF4E1AE0028C7
:105D500040F009852020884045B245F01400C0B2CB
:105D6000FFF790FD410540D545F01100C0B2FFF7A7
:105D700089FD306035E0CE2A00F0558513D8B82A69
:105D800000F01485B92A7FF4C3AE002840F03385B3
:105D9000080140F06C0000F0FC00FFF773FDC0F359
:105DA000035030601DE0D22A00F05A85D32A00F05B
:105DB0007185D12A7FF4ACAE002840F042852020C6
:105DC000884040F01900C0B2FFF75CFD306008E089
:105DD00048B92020884040F00D00C0B2FFF752FDC6
:105DE00030602046F8BD012801D00024F9E72021C9
:105DF000A94041F00D011A68C9B22846FFF7E4FD39
:105E00000024EEE740B92020884040F00100C0B2F5
:105E1000FFF738FD3060E4E70128E6D12021A940F2
:105E200041F001011A68C9B22846FFF7CDFD0024F0
:105E3000D7E758B92020884040F00700C0B2FFF7EC
:105E400021FD3060CDE700BF2C4EFF1F0128CCD1D3
:105E5000BB4B0B44202183F894023268A940002AEE
:105E600041F00701B8BF5242C9B22846FFF7ACFD66
:105E70000024B6E770B92020884040F00200C0B28C
:105E8000FFF700FD10F4000318BF4FF07F431843E5
:105E90003060A6E7012CA8D10424A2E70128A4D1F0
:105EA000A84B32681B682020884040F0070703EBAE
:105EB0008703002AB8BF52425A60C0B2FFF7E2FC23
:105EC0000446002891D13268002AB8BF5242F9B284
:105ED0002846FFF779FD84E740B92020884040F04C
:105EE0000600C0B2FFF7CEFC30607AE701287FF4ED
:105EF0007CAF2021A94041F006011A68C9B22846AA
:105F0000FFF762FD00246CE750B92020884040F084
:105F10001000C0B2FFF7B6FCC0F30420306060E7A9
:105F200001287FF462AF20248C4044F01004E4B2D6
:105F30002046FFF7A7FC33681B0203F4F85320F454
:105F4000F85221461A432846FFF73EFD002448E751
:105F500001287FF44AAF20248C4044F01004E4B2BE
:105F60002046FFF78FFC336820F01F0203F01F0369
:105F700021461A432846FFF727FD002431E7002871
:105F800088D12020884040F01500C0B2FFF77AFC8D
:105F9000C0F34020306024E700287FF47BAF20204E
:105FA000884040F01500C0B2FFF76CFC10F0020F03
:105FB0000CBF01230023336013E750B92020884031
:105FC00040F01400C0B2FFF75DFCC0F34000306049
:105FD00007E701287FF409AF20248C4044F0140423
:105FE000E4B22046FFF74EFC33685B0003F0020387
:105FF00020F0020221461A432846FFF7E5FC002460
:10600000EFE650B92020884040F01400C0B2FFF7FE
:1060100039FC00F001003060E3E601287FF4E5AED2
:1060200020248C4044F01404E4B22046FFF72AFCFC
:10603000336820F0010203F0010321461A43284689
:10604000FFF7C2FC0024CCE601287FF4CEAE20216D
:10605000A94041F014011A68C9B22846FFF7B4FC00
:106060000024BEE640B92020884040F00400C0B2C1
:10607000FFF708FC3060B4E601287FF4B6AE2021BB
:10608000A94041F004011A68C9B22846FFF79CFCF8
:106090000024A6E640B92020884040F00500C0B2A8
:1060A000FFF7F0FB30609CE601287FF49EAE2021D4
:1060B000A94041F005011A68C9B22846FFF784FCDF
:1060C00000248EE601287FF490AE2021A94041F003
:1060D00008011A68C9B22846FFF776FC002480E65A
:1060E00040B92020884040F00A00C0B2FFF7CAFB48
:1060F000306076E601287FF478AE2021A94041F097
:106100000A011A68C9B22846FFF75EFC002468E657
:1061100040B92020884040F00300C0B2FFF7B2FB36
:1061200030605EE601287FF460AE2021A94041F096
:1061300003011A68C9B22846FFF746FC002450E65E
:10614000304EFF1F2C4EFF1F01287FF44EAE202142
:10615000A94041F00B011A68C9B22846FFF734FC88
:1061600000243EE640B92020884040F00C00C0B238
:10617000FFF788FB306034E601287FF436AE20213B
:10618000A94041F00C011A68C9B22846FFF71CFC6F
:10619000002426E64CB92020A84040F01100C0B2EF
:1061A000FFF770FB002430601BE6012C7FF41DAE6E
:1061B0002021A94041F011013268C9B22846FFF7F9
:1061C00003FC00240DE640B92020884040F0120076
:1061D000C0B2FFF757FB306003E601287FF405AE3D
:1061E0002021A94041F012011A68C9B22846FFF7E0
:1061F000EBFB0024F5E501287FF4F7AD2021A94051
:1062000041F013011A68C9B22846FFF7DDFB0024EC
:10621000E7E550B9080140F06C0000F0FC00FFF722
:1062200031FBC0F380403060DBE501287FF4DDAD59
:106230000C0144F06C04E4B22046FFF723FB336802
:106240009B0403F4802320F4802221461A4328462D
:10625000FFF7BAFB0024C4E500287FF41BAEC74B50
:1062600053F821303360BCE501287FF4BEAD1B68D4
:10627000102B23D00DDC022B1CD004DC012B16D0FC
:106280004FF0FF3314E0042B16D0082BF8D1052370
:106290000EE0402B14D003DC202BF1D1032307E0C8
:1062A000802B0FD0B3F5807FEAD1002300E00823D4
:1062B000336008E00723FBE70623F9E70423F7E749
:1062C0000223F5E73060336801333FF48EAD2C01D3
:1062D00044F06C04E4B22046FFF7D4FA33681B069E
:1062E00003F0706320F0706221461A432846FFF7DE
:1062F0006BFB002475E550B9080140F06C0000F01C
:10630000FC00FFF7BFFAC0F3C130306069E5012837
:106310007FF46BAD0C0144F06C04E4B22046FFF74F
:10632000B1FA3368DB0303F4C03320F4C0322146F2
:106330001A432846FFF748FB002452E550B90801EC
:1063400040F06C0000F0FC00FFF79CFAC0F38030D6
:10635000306046E501287FF448AD0C0144F06C0440
:10636000E4B22046FFF78EFA33689B0303F48043C0
:1063700020F4804221461A432846FFF725FB0024DB
:106380002FE501287FF431AD0C0144F06C04E4B238
:106390002046FFF777FA33681B0303F4805320F499
:1063A000805221461A432846FFF70EFB002418E5C9
:1063B00008BB080140F06C05EDB22846FFF762FA11
:1063C00010F48047284605D0FFF75CFAC0F3C310ED
:1063D000306006E5FFF756FAC0F302103060284639
:1063E000FFF750FA04057FF500AD336843F008036A
:1063F00033603C46F5E401287FF4F7AC0C0144F02F
:106400006C04E4B22046FFF73DFA10F480472046C2
:106410000ED0FFF737FA3368DB0103F4F06320F4A2
:10642000F06221461A432846FFF7CEFA0024D8E44A
:10643000FFF728FA336813F0080F18BF4FF400670E
:1064400020F4006221463A432846FFF7BDFA204671
:10645000FFF718FA33681B0103F0700320F0700295
:1064600021461A432846FFF7AFFA0024B9E408BBD7
:10647000080140F06C05EDB22846FFF703FA10F46E
:106480008044284606D0FFF7FDF9C0F302103060C3
:106490000024A6E4FFF7F6F9C0F3C31030602846E5
:1064A000FFF7F0F900057FF5A0AC336843F008036F
:1064B000336096E401287FF498AC0F0147F06C0735
:1064C000FFB23846FFF7DEF910F4804438460ED0AC
:1064D000FFF7D8F933681B0103F0700320F0700256
:1064E0001A4339462846FFF76FFA002479E4FFF78C
:1064F000C9F93368DB0103F4F06320F4F0621A4356
:1065000039462846FFF760FA6BE401287FF46DAC4A
:106510000C0144F06C04E4B22046FFF7B3F9336891
:1065200020F00F0203F00F0321461A432846FFF71D
:106530004BFA002455E450B9080140F06D0000F01A
:10654000FD00FFF79FF9C0F3C030306049E4012837
:106550007FF44BAC0C0144F06D04E4B22046FFF72D
:1065600091F93368DB039BB220F4004221461A43C1
:106570002846FFF729FA002433E400BF304EFF1FFE
:1065800050B9080140F06D0000F0FD00FFF77AF906
:10659000C0F34130306024E401287FF426AC0C01C4
:1065A00044F06D04E4B22046FFF76CF933685B03F6
:1065B00003F4C04320F4C04221461A432846FFF7A3
:1065C00003FA00240DE450B9080140F06D0000F01A
:1065D000FD00FFF757F9C0F30320306001E4012804
:1065E0007FF403AC0C0144F06D04E4B22046FFF7E5
:1065F00049F933681B0203F4706320F4706221468A
:106600001A432846FFF7E0F90024FFF7EABB012808
:106610007FF4EBAB0C0144F06D04E4B22046FFF7CD
:1066200031F933685B0103F0600320F0600221461A
:106630001A432846FFF7C8F90024FFF7D2BB58B920
:10664000080140F06D0000F0FD00FFF71BF900F0BD
:106650000F003060FFF7C5BB01287FF4C6AB0C010B
:1066600044F06D04E4B22046FFF70CF9336820F0E3
:106670000F0203F00F0321461A432846FFF7A4F93F
:106680000024FFF7AEBB58B9080140F06D0000F0E0
:10669000FD00FFF7F7F8C0F300603060FFF7A1BB23
:1066A00001287FF4A2AB0C0144F06D04E4B2204653
:1066B000FFF7E8F833681B0603F0807320F0807260
:1066C00021461A432846FFF77FF90024FFF789BBCC
:1066D00001287FF48AAB0C0144F06D04E4B220463B
:1066E000FFF7D0F833681B0403F4FE0320F4FE0226
:1066F00021461A432846FFF767F90024FFF771BBCC
:1067000058B9080140F06C0000F0FC00FFF7BAF83F
:10671000C0F340403060FFF764BB01287FF465ABF5
:106720000C0144F06C04E4B22046FFF7ABF8336888
:106730005B0403F4003320F4003221461A43284658
:10674000FFF742F90024FFF74CBB00287FF4A2AB0F
:10675000080140F06F00C0B2FFF794F8C0F30440A6
:106760003060FFF73EBB01287FF43FAB20248C4014
:1067700064B244F0110144F014041A68C9B2E4B2DE
:106780002846FFF721F92046FFF77CF83368002BF5
:1067900020F480620CBF00234FF4806321461A432B
:1067A0002846FFF711F90024FFF71BBB58B9080171
:1067B00040F06C0000F0FC00FFF764F8C0F34030DC
:1067C0003060FFF70EBB01287FF40FAB0C0144F0E3
:1067D0006C04E4B22046FFF755F833685B0303F41A
:1067E000005320F4005221461A432846FFF7ECF8E4
:1067F0000024FFF7F6BA01287FF4F7AA0C0144F051
:106800006C04E4B22046FFF73DF833681B0503F43F
:10681000700320F4700221461A432846FFF7D4F88B
:106820000024FFF7DEBA00287FF434AB080140F003
:106830006F00C0B2FFF726F8C0F309003060FFF721
:10684000D0BA01287FF4D1AA2021A94041F0190132
:106850001A68C9B22846FFF7B7F80024FFF7C1BA93
:1068600048B92020884040F01A00C0B2FFF70AF86B
:106870003060FFF7B6BA01287FF4B7AA2021A940FB
:1068800041F01A011A68C9B22846FFF79DF80024A2
:10689000FFF7A7BAD8B969B101297FF4A2AAFEF718
:1068A000F1FF00F06000A0F1200358425841306031
:1068B000FFF797BA0846FEF7E5FF00F01800A0F1D1
:1068C00010025042504130602C46FFF78ABA01282E
:1068D0007FF48BAA21B1012915D00024FFF781BADA
:1068E0000846FEF7CFFF336820F0180243B142F0AC
:1068F000100200210846FFF767F80024FFF771BA7D
:1069000042F00802F5E70020FEF7BCFF336820F0F4
:10691000600243B142F0200200210120FFF754F849
:106920000024FFF75EBA42F04002F5E707B50129FF
:10693000019207D8024601AB0120FFF7CEF803B061
:106940005DF804FB0820FAE70129134603D8024644
:106950000020FFF7C2B80820704738B5234B01F07C
:106960007F04234493F81432DB0705D4204B1B68C3
:1069700003EB8404606838BD1E4D2B6800219B68C2
:10698000204698472B6800219B68084698472B684B
:1069900000219B68084698472B6800219B680846A1
:1069A00098472B6801219B68002098472B6800219D
:1069B0009B68204698472B6800219B6808469847AB
:1069C0002B68002104029B68084698472B68002129
:1069D00004439B68084698472B68240204439B683D
:1069E0000121002098472402204338BD304EFF1F6C
:1069F0002C4EFF1FC850FF1F70B53D4E3D483E4C0A
:106A00000AF0F2FAF5686B6803F58272626003F5CA
:106A10009272A26003F57172E26003F5797203F17C
:106A20006400226103F2044203F22443A3612B6851
:106A30006261DB68206098472B68E068DB689847F4
:106A40002B68E0689B6998472B6860681B699847CA
:106A50002B68A0681B6998472B68A0691B69984739
:106A60002B6820691B6998472B6860691B699847E8
:106A7000224B32691A606B68214903F53173536008
:106A8000204B5A690A602049C2F804121F49C2F813
:106A9000081201200021107051701D4A1A621D4A0F
:106AA000DA611D4A9A611D4A5A621D4A9A631D4A5B
:106AB0005A631D4A9A621D4ADA621D4A9A641D4A47
:106AC0005A641D4A5A651D4A1A651D4ADA641D4AF0
:106AD0001A661D4ADA6502221A743222DA60DE2250
:106AE0009A601A4A9A65BDE87040FEF781BE00BF01
:106AF000704C0200304EFF1F7017FF1FC850FF1F61
:106B00002C4EFF1F7431FF1F2559010089570100CA
:106B10007B5A0100D95A0100D55A0100D15A01000F
:106B2000496901002D690100EF590100595A01001E
:106B3000E55901004D5901005D57010095570100CD
:106B400039570100F1570100515701003158010038
:106B500001289FBF034B53F820300B60002088BFF3
:106B600008207047D050FF1F014B00225A60704729
:106B70007431FF1F70B5084E084D336804462A462D
:106B8000014600200AF018FB33682A4621460120FE
:106B9000BDE870400AF010BBCC50FF1FD050FF1F63
:106BA000014B18680AF053BBCC50FF1F012810B5E9
:106BB000144611D003D302281AD0042010BD146843
:106BC0000F4A104BD268126824B15269D8689047B6
:106BD000002010BD9269F9E7094B0A4ADB6850684A
:106BE0001B681B6A9847003018BF01202060EFE740
:106BF000034B044ADB6890681B681B6AF2E700BF1E
:106C0000704C02009817FF1F022804BF0B4B93F82B
:106C1000D00030B90A4BDB681B685B69094A106811
:106C20001847012809D1054B93F8D030012B04D126
:106C3000034BDB681B689B69F0E770477431FF1FEB
:106C4000704C02009817FF1F70B50020FFF7DCFFA3
:106C5000104B114CDD6820682B689B6898472B68A7
:106C600060689B6898472B68A0689B6898472B686A
:106C7000A0699B6898472B6820699B6898472B6898
:106C800060699B6898472B68E0689B68BDE8704026
:106C9000184700BF704C02009817FF1F2DE9F843FA
:106CA000184C9DF820609DF82450984623680F46A4
:106CB0009B68002147F08000914698472368002197
:106CC0009B6848469847236800219B684046984740
:106CD000236800219B6830469847236828469B68B4
:106CE00001219847084B1B6848EA092807F07F07ED
:106CF00046EA082603EB870745EA06257D60BDE8DE
:106D0000F88300BF6853FF1FCC50FF1F07B5D3B2F5
:106D10000193C2F307230093C2F30743120EFFF758
:106D2000BDFF03B05DF804FB0A4601460020FFF7F3
:106D3000EDBF0128F7B505460F4628D8154C044489
:106D400094F8943273B1144B202181401B6841F0B8
:106D5000070103EB8103C9B25A68FFF7D7FF00238D
:106D600084F894322026AE4046F00D0100243A46C5
:106D7000C9B22846FFF7CAFF28460194009423466B
:106D80002246F1B2FFF78AFF204603B0F0BD08208B
:106D9000FBE700BFD050FF1FCC50FF1F012873B589
:106DA00005460C4621D82026864084EAE47246F047
:106DB0000701A2EBE472C9B2FFF7A8FF0C4B2B440A
:106DC000002C4FF0010283F894224FF00004ACBF76
:106DD0001346022301932846009423462246F1B22B
:106DE000FFF75CFF204602B070BD0820FBE700BF44
:106DF000D050FF1F0021D1E74942CFE7CEE738B599
:106E0000234B01F07F04234493F81432DB0705D4AD
:106E1000204B1B6803EB8404606838BD1E4D2B6853
:106E200000219B68204698472B6800219B680846F4
:106E300098472B6800219B68084698472B680021DB
:106E40009B68084698472B6801219B68002098475B
:106E50002B6800219B68204698472B6800219B687F
:106E6000084698472B68002104029B68084698470B
:106E70002B68002104439B68084698472B6824022E
:106E800004439B680121002098472402204338BD19
:106E9000D050FF1FCC50FF1F6853FF1F10B50C468A
:106EA00001460020FFF7ABFF206010BD38B50D464E
:106EB0002021814041F00101C9B20446FFF79FFF44
:106EC0002968014429602046BDE8384031E71C2A82
:106ED0002DE9F34104460D461E4600F0F88200F20B
:106EE00092800C2A00F016824BD8052A00F0B78158
:106EF0001ED8022A00F0668107D8002A00F03D81E2
:106F0000012A00F05281042441E1032A00F070813B
:106F1000042AF8D1002840F08381BF4B20201B6851
:106F2000884040F0070003EB8000436833602EE1A7
:106F3000082A00F0D58111D8062A00F09D81072A81
:106F4000E1D1002840F0BB812021A94041F010018F
:106F5000C9B22846FFF753FFC0B217E10A2A00F072
:106F6000CC810B2ACFD1002840F052812021A940AA
:106F700041F01501C9B22846FFF741FF00F00100BA
:106F800004E1122A00F048821DD80F2A00F0208266
:106F90000CD80D2A00F0EB810E2AB4D1002840F065
:106FA0000F822021A94041F01401EBE0102A00F0EB
:106FB0001D82112AA7D1002840F026822021A94055
:106FC00041F00801DEE0152A00F04A820CD8132AAD
:106FD00000F03082142A96D1002840F03982202116
:106FE000A94041F00B01CDE0172A00F05A82C0F011
:106FF0004582182A87D1002840F061822021A940CB
:1070000041F01301BEE0AB2A00F0E5835ED8A52A6B
:1070100000F00A832ED8A22A00F0C48217D81D2AB5
:1070200000F073828C2A7FF46EAF002840F07882E3
:10703000090141F06C0101F0FC012846FFF7DFFE79
:107040004FF4807300F00F0043FA00F09EE0A32A93
:1070500074D0A42A7FF457AF002840F0D3820901EE
:1070600041F06C0101F0FC012846FFF7C8FEC0F3B7
:1070700000308BE0A82A00F0618313D8A62A00F024
:107080001E83A72A7FF43FAF002840F04683090102
:1070900041F06C0101F0FC012846FFF7B0FE00F062
:1070A0000F0073E0A92A00F06683AA2A7FF42BAFB1
:1070B000002840F07E83090141F06D0101F0FD01DF
:1070C0002846FFF79CFEC0F303205FE0B52A00F0DE
:1070D000028429D8AE2A00F0BC8313D8AC2A00F071
:1070E0009883AD2A7FF40FAF002840F0A0830901F8
:1070F00041F06D0101F0FD012846FFF780FEC0F36D
:10710000006043E0B32A00F0C883B42A7FF4FBAEEA
:1071100000287DD1090141F06F01C9B22846FFF76F
:107120006EFEC0F3044031E0CE2A00F0028413D892
:10713000B62A00F0A381B82A7FF4E5AE002C40F017
:107140004F82290141F06C0101F0FC012846FFF754
:1071500056FEC0F340309AE1D22A00F0FF83D32AD2
:1071600000F00A84D12A7FF4CEAE002840F0EE83EE
:107170002021A94041F0190104E060B92021A94073
:1071800041F00D01C9B22846FFF739FE30602046B4
:1071900002B0BDE8F081012801D00024F7E72021EA
:1071A000A94041F00D01326820E020B92021A9401A
:1071B00041F00101E6E70128EFD12021A94041F08B
:1071C0000101F0E720B92021A94041F00701D9E7EA
:1071D0000128E2D1114B0B44202183F8940232683C
:1071E000A940002A41F00701B8BF5242C9B262E289
:1071F00070B92021A94041F00201C9B22846FFF729
:10720000FEFD10F4000318BF4FF07F431843BDE7A5
:10721000012C3FF478AEC0E7CC50FF1FD050FF1FC9
:107220000128BAD1BC4B32681B682021A94041F02B
:10723000070703EB8703002AB8BF52425A60C9B25E
:107240002846FFF7DCFD04460028A6D13268002A54
:10725000B8BF5242F9B22846FFF758FD97E720B968
:107260002021A94041F006018CE7012895D1202179
:10727000A94041F0060196E750B92021A94041F00C
:107280001001C9B22846FFF7BAFDC0F307207DE719
:10729000012882D120248C4044F01004E4B221461D
:1072A0002846FFF7ACFDC3B2019333780093002268
:1072B000C0F3074321462846FFF7F0FC6DE701289D
:1072C0007FF46BAF20248C4044F01004E4B22146DC
:1072D0002846FFF794FD33780193C0F30723E5E7D1
:1072E000002895D12021A94041F01501C9B22846B6
:1072F000FFF785FDC0F3402048E7002888D1202112
:10730000A94041F01501C9B22846FFF778FDC0F346
:1073100040003BE720B92021A94041F01401F2E7E9
:1073200001287FF43AAF20248C4044F01404E4B2E6
:1073300021462846FFF763FD3368002BCCBF0223AC
:10734000002320F002021A4321462846FFF7DEFC04
:1073500021462846FFF753FD3368022B20F0080230
:1073600008BF082318BF00231A432146A3E120B910
:107370002021A94041F01401FCE501287FF40DAF64
:1073800020248C4044F01404E4B221462846FFF740
:1073900036FD326820F00100002AD4BF024640F0DA
:1073A000010221462846FFF7B1FC21462846FFF797
:1073B00026FD3368022B20F0040208BF0423D1E726
:1073C00001287FF4EAAE2021A94041F01401EAE649
:1073D00020B92021A94041F00401D3E601287FF41F
:1073E000DCAE2021A94041F00401DCE620B92021D7
:1073F000A94041F00501C5E601287FF4CEAE202169
:10740000A94041F00501CEE601287FF4C6AE202157
:10741000A94041F00801C6E620B92021A94041F069
:107420000A01AFE601287FF4B8AE2021A94041F05F
:107430000A01B8E620B92021A94041F00301A1E6E4
:1074400001287FF4AAAE2021A94041F00301AAE659
:1074500001287FF4A2AE2021A94041F00B01A2E651
:1074600020B92021A94041F00C018BE601287FF4CE
:1074700094AE2021A94041F00C0194E64CB92021A2
:10748000A94041F01101C9B22846FFF7B8FC3060AD
:1074900083E6012C7FF481AE2021A94041F0110147
:1074A00081E620B92021A94041F012016AE60128B5
:1074B0007FF473AE2021A94041F0120173E6012848
:1074C0007FF46BAE2021A94041F013016BE650B967
:1074D000090141F06C0101F0FC012846FFF78FFC27
:1074E000C0F3804052E601287FF457AE0C0144F00F
:1074F0006C04E4B221462846FFF781FC33689B0404
:1075000003F4802320F480222EE700287FF480AE4D
:10751000024B53F8213009E5CC50FF1FD050FF1F1C
:1075200001287FF43AAE1B68102B23D00DDC022B10
:107530001CD004DC012B16D04FF0FF3314E0042BD9
:1075400016D0082BF8D105230EE0402B14D003DC15
:10755000202BF1D1032307E0802B0FD0B3F5807FE0
:10756000EAD1002300E00823336008E00723FBE7AB
:107570000623F9E70423F7E70223F5E730603368D1
:1075800001333FF40AAE2C0144F06C04E4B221460E
:107590002846FFF734FC33681B0603F0706320F0C5
:1075A0007062E1E650B9090141F06C0101F0FC01A3
:1075B0002846FFF724FCC0F3C130E7E501287FF43B
:1075C000ECAD0C0144F06C04E4B221462846FFF710
:1075D00016FC3368DB0303F4C03320F4C032C3E687
:1075E000012C7FF4DAAD2C0144F06C04E4B22146A6
:1075F0002846FFF704FC33685B0303F4005320F4D0
:107600000052B1E601287FF4C8AD0C0144F06C04CF
:10761000E4B221462846FFF7F2FB33681B0303F46C
:10762000805320F480529FE60F0147F06C07FFB2B1
:1076300039462846FFF7E3FBC0F3803874B9394672
:107640002846B8F1000F04D0FFF7D9FBC0F3C310F0
:107650009CE5FFF7D4FBC0F3021018E7012C7FF480
:107660009CAD39462846B8F1000F08D0FFF7C7FB9C
:107670003368DB0103F4F06320F4F06219E0FFF7F4
:10768000BEFB336813F0080F20F4006218BF4FF4FC
:1076900000683946284642EA0802FFF737FB3946B8
:1076A0002846FFF7ACFB33681B0103F0700320F0A2
:1076B00070021A4339462846FFF728FB6DE50F0193
:1076C00047F06C07FFB239462846FFF798FBC0F336
:1076D0008038CCB939462846B8F1000F04D0FFF7FE
:1076E0008EFBC0F3021051E5FFF789FBC0F3C31016
:1076F000306039462846FFF782FB3368000A00F005
:1077000008000343336048E5012C7FF446AD394659
:107710002846B8F1000FA9D0C3E701287FF43DAD9A
:107720000C0144F06C04E4B221462846FFF767FBE5
:10773000336820F00F0203F00F0315E650B909017A
:1077400041F06D0101F0FD012846FFF758FBC0F341
:10775000C0301BE501287FF420AD0C0144F06D041E
:10776000E4B221462846FFF74AFB3368DB039BB2AD
:1077700020F40042F8E550B9090141F06D0101F033
:10778000FD012846FFF73BFBC0F34130FEE4012832
:107790007FF403AD0C0144F06D04E4B221462846A9
:1077A000FFF72DFB33685B0303F4C04320F4C042B2
:1077B000DAE501287FF4F1AC0C0144F06D04E4B289
:1077C00021462846FFF71BFB33681B0203F4706356
:1077D00020F47062C8E550B9090141F06D0101F073
:1077E000FD012846FFF70BFBC0F34110CEE4012852
:1077F0007FF4D3AC0C0144F06D04E4B2214628467A
:10780000FFF7FDFA33685B0103F0600320F06002CC
:10781000AAE528B9090141F06D0101F0FD013BE441
:1078200001287FF4BAAC0C0144F06D047BE7012819
:107830007FF4B3AC0C0144F06D04E4B22146284659
:10784000FFF7DDFA33681B0603F0807320F08072C7
:107850008AE580B9090141F06D0101F0FD0128467A
:10786000FFF7CDFA001400F07F0310F0400018BFBE
:107870006FF07F00CAE401287FF48FAC0C0144F064
:107880006D04E4B221462846FFF7B9FA33681B04B9
:1078900003F4FE0320F4FE0266E550B9090141F04D
:1078A0006C0101F0FC012846FFF7A9FAC0F3404043
:1078B0006CE401287FF471AC0C0144F06C04E4B278
:1078C00021462846FFF79BFA33685B0403F4003334
:1078D00020F4003248E578B920278F407FB247F086
:1078E0001401C9B22846FFF78AFA10F480603FF409
:1078F000CEAD47F0110145E401287FF44EAC2024C1
:107900008C4064B244F0110144F014041A68C9B206
:107910002846E4B2FFF7FAF921462846FFF76FFA46
:107920003368002B20F4806214BF4FF4806300237F
:107930001AE500287FF46CAC090141F06F01C9B26F
:107940002846FFF75CFAC0F309001FE401287FF422
:1079500024AC2021A94041F0190124E420B92021C0
:10796000A94041F01A010DE401287FF416AC202152
:10797000A94041F01A0116E4C8B971B101297FF498
:1079800006AC01462846FFF73AFA00F06000A0F185
:10799000200358425841FFF7F9BB0846FFF72FFA7A
:1079A00000F01800A0F11002504250416FE501288C
:1079B0007FF4F3ABF1B101297FF4EFAB002128464E
:1079C000FFF71DFA3368002B14BF2023002320F09B
:1079D00020021A4300212846FFF798F90021284683
:1079E000FFF70DFA3368002B20F040020CBF402354
:1079F000002319E00846FFF702FA3368002B0CBF9A
:107A00000823002320F008021A4329462846FFF7DE
:107A10007DF929462846FFF7F2F93368002B20F05C
:107A2000100214BF102300231A43002143E607B5B8
:107A30000129019207D8024601AB0120FFF747FA5E
:107A400003B05DF804FB0820FAE70129134603D8C8
:107A500002460020FFF73BBA0820704708B52221F4
:107A60000020FFF7CCF950B942210120FFF7C7F9F8
:107A700028B9044B1868BDE8084009F0DFBB0020B6
:107A800008BD00BFCC50FF1F70B53D4E3D483E4C79
:107A900009F054FBF5686B6803F58272626003F5C8
:107AA0009272A26003F57172E26003F5797203F1DC
:107AB0006400226103F2044203F22443A3612B68B1
:107AC0006261DB68206098472B68E068DB68984754
:107AD0002B68E0689B6998472B6860681B6998472A
:107AE0002B68A0681B6998472B68A0691B69984799
:107AF0002B6820691B6998472B6860691B69984748
:107B0000224B32691A606B68214903F53173536067
:107B1000204B5A690A602049C2F804121F49C2F872
:107B2000081201211170002151701D4A1A621D4A6C
:107B3000DA611D4A9A611D4A5A621D4A9A631D4ABA
:107B40005A631D4A9A621D4ADA621D4A9A641D4AA6
:107B50005A641D4A5A651D4A1A651D4ADA641D4A4F
:107B60001A661D4ADA653222DA6002204FF48C72FE
:107B70009A601874194A9A65BDE87040FFF744B8D6
:107B8000704C0200D050FF1F9817FF1F6853FF1F53
:107B9000CC50FF1F7431FF1F5D7A0100A16B010003
:107BA0009D6D0100FD6D0100F96D0100F56D010095
:107BB0004B7A01002F7A0100336D0100AD6E010098
:107BC000296D01009D6E0100756B0100AD6B010018
:107BD000516B0100096C0100696B0100496C0100E7
:107BE00018B9034B1B680B6070470820704700BF33
:107BF0007053FF1F014B00225A6070477431FF1F02
:107C00000428F8B5144600F0848009D801284BD028
:107C10001FD3022866D0032862D004242046F8BD72
:107C2000062800F0A580C0F09880072800F0A78003
:107C3000FC28F2D114685B4D5B4B002C00F0AB804C
:107C4000DC6828692368DB689847236828699B6992
:107C500016E0136833F0030240F0A28013F0010F26
:107C6000504D514E0ED0F3681B681B6968689847E9
:107C7000246814F002040DD0F36828681B681B699F
:107C800098472DE0F76868683B68DB6898473B6871
:107C90009B69EBE7F66828683368DB6898473368C8
:107CA00028689B699847B9E7136844F620629342B5
:107CB00076DC42F2107293423B4A3A4BD268586AE1
:107CC0001268CCBF526992699047226842F21173E0
:107CD00092FBF3F003FB1020344B80B29B68984773
:107CE00000249BE71468304B64B1DC68606823684B
:107CF00000F5F270DB6898476068236800F5F27061
:107D00009B69BDE7DB6858681B6800F5F2709B68EB
:107D1000C8E71568234E244B5DB1012D15D0DD68F1
:107D200030692B681B6998472B6830691B6A984734
:107D300009E0DF6830693B68DB6898473B689B690E
:107D40003069984728462060CAE7DF6830693B6899
:107D5000DB6898473B685B69F2E7134B114ADB68C5
:107D6000D0691B681B6A9847003018BF0120EAE7FA
:107D70000D4B0C4ADB68106A1B681B6AF3E713683B
:107D8000094AD268012B1268064B0CBF52699269EE
:107D900098699047A4E7DB6828691B681B6981E73D
:107DA00010243BE7C017FF1F704C02006809FF1F3B
:107DB0001C4B70B5DD681C4C2B68A0689B6998470C
:107DC0002B68A06A9B6898472B68606A9B689847F5
:107DD0002B68E0689B6898472B6820699B689847E8
:107DE0002B6860699B6898472B6820689B68984758
:107DF0002B6860689B6898472B68E0699B68984788
:107E00002B68206A9B6898472B68A0699B689847F5
:107E10002B68A0689B689847044BBDE870405B687E
:107E2000184700BF704C0200C017FF1F6809FF1FF2
:107E3000034B044A1B680146002007F0EABA00BF62
:107E40006C53FF1F7053FF1F014B186807F019BBDD
:107E50006C53FF1F022804BF0B4B93F8D00030B9BE
:107E60000A4BDB681B685B69094A90681847012860
:107E700009D1054B93F8D030012B04D1034BDB68BB
:107E80001B689B69F0E770477431FF1F704C02005C
:107E9000C017FF1F2DE9F0471C4D9DF820709DF87D
:107EA0002460994655F82030044688469B68002196
:107EB00048F080009246984755F8243000219B688E
:107EC0005046984755F8243000219B68484698470B
:107ED00055F8243000219B683846984755F82430DF
:107EE00030469B6801219847094B53F8243049EAF2
:107EF0000A2908F07F0847EA092703EB880846EAC1
:107F00000726C8F80460BDE8F08700BFFC55FF1FD6
:107F10006C53FF1F07B5D3B20193C2F3072300933D
:107F2000C2F30743120EFFF7B5FF03B05DF804FB81
:107F30000A4601460020FFF7EDBF38B50D4604465E
:107F400090B902462021FFF7E5FF084B1B68204649
:107F5000D3F8A0202721FFF7DDFF20462A462D2158
:107F6000FFF7D8FF204638BD082038BD6C53FF1FEF
:107F700037B50D460446A8B981EAE172A2EBE17279
:107F80002721FFF7C7FF002DACBF01230223019378
:107F900020460094234622462021FFF77BFF2046FF
:107FA00003B030BD0820FBE70021E1E74942DFE7ED
:107FB000DEE770B52B4A4FF4237301F07F0403FB17
:107FC00000232344054693F80C32DB0706D4264BE6
:107FD00053F8203003EB8404606870BD234E56F8DC
:107FE000203000219B682046984756F82530002114
:107FF0009B680846984756F8253000219B6808463C
:10800000984756F8253000219B680846984756F84F
:10801000253001219B680020984756F82530002123
:108020009B682046984756F8253000219B680846F3
:10803000984756F82530002104029B680846984767
:1080400056F82530002104439B680846984756F8A7
:108050002530240204439B68012100209847240214
:10806000204370BD7053FF1F6C53FF1FFC55FF1F53
:1080700010B50C4601460020FFF79BFF206010BDA5
:1080800038B50C46054648B92121FFF792FF216813
:10809000014421602846BDE838404EE7082038BD3D
:1080A0008C2A70B504460D461E4600F0728300F21D
:1080B0009B800E2A00F0598241D8062A00F0C58123
:1080C00019D8022A00F0748107D8002A00F04D81E7
:1080D000012A00F05D8104244DE1042A00F0898129
:1080E00040F27681002840F0A78126212846FFF73C
:1080F00060FF30603FE10A2A00F0E6810FD8072ACE
:1081000000F0BF81082AE6D1002840F06E813521B9
:108110002846FFF74EFFC0F3402030602BE10C2AC9
:1081200000F0EA8140F2DD81002840F0068234212F
:108130002846FFF73EFF00F0010030601BE1152AE2
:1081400000F07C821FD8112A00F03B820DD80F2A44
:1081500000F01C82102ABED1002840F02882252180
:108160002846FFF726FF306005E1132A00F04B8216
:1081700040F23882002840F057822B212846FFF732
:1081800018FF3060F7E01C2A00F0AD821AD8182AD8
:1081900000F07B821B2A00F08982172A9BD10028DD
:1081A00040F05D8215212846FFF703FFC34B30B135
:1081B0004FF08072B2FBF0F0834228BF0346336079
:1081C0000024D8E0212A00F0AB82222A00F0C482E9
:1081D0001D2A80D1002840F008814FF423735D43AD
:1081E000B74B5B593360C6E0B32A00F0C58457D85B
:1081F000A82A00F0098424D8A42A00F04C8310D8BF
:10820000A22A00F01783A32A7FF465AF002840F06C
:108210002E836C212846FFF7CCFEC0F380303060FF
:10822000A9E0A62A00F0988340F25283002840F08B
:10823000D8836C212846FFF7BCFE00F00F003060A9
:1082400099E0AB2A00F02D8410D8A92A00F0F88319
:10825000AA2A7FF440AF002840F00F846D21284601
:10826000FFF7A7FEC0F30320306084E0AD2A00F0E2
:108270005184C0F03384AE2A7FF42DAF002840F043
:1082800066846D212846FFF794FE001400F07F03FA
:1082900010F0400018BF6FF07F00184330606AE0B4
:1082A000BB2A00F0448536D8B62A00F0BB841FD81C
:1082B000B42A00F08084B52A7FF40DAF002840F086
:1082C000898434212846FFF774FE430540F17F84FA
:1082D00014212846FFF76DFE784B30B14FF08072C5
:1082E000B2FBF0F0834228BF03463360002442E033
:1082F000B92A00F0D48400F2F184B82A7FF4EBAEFE
:10830000002840F0B7846C212846FFF752FEC0F3E6
:10831000403030602FE0CC2A00F08D8512D8BF2A83
:1083200000F04585C02A00F06485BC2A7FF4D3AEF6
:10833000002840F02A8570212846FFF73AFEC0B297
:10834000306018E0D12A00F09585D22A00F0A5858A
:10835000CE2A7FF4C0AE002847D16F212846FFF710
:1083600028FEC0F30900306005E030B92D21284611
:10837000FFF71FFE3060204670BD012801D00024A9
:10838000F9E71A682D212846FFF7C4FD0024F2E71B
:1083900028B921212846FFF70CFE3060EBE70128C1
:1083A000EDD11A6821212846FFF7B4FD0024E2E749
:1083B00028B927212846FFF7FCFD3060DBE70128BC
:1083C000DDD11A6827212846FFF7A4FD0024D2E753
:1083D00058B922212846FFF7ECFD10F4000318BF1E
:1083E0004FF07F4318433060C5E7012CC7D1042408
:1083F000C1E730B9334B53F82130D3F8A0303360A4
:10840000B9E70128BBD12F4B53F821203368002B4B
:10841000B8BF5B42C2F8A03020212846FFF7C9FD53
:1084200004460028ABD13268002AB8BF5242272147
:108430002846FFF76FFD9EE70128A0D11A68262184
:108440002846FFF767FD002495E738B91021284634
:10845000FFF7AFFDC0F3042030608CE701288ED118
:1084600010212846FFF7A5FD33681B0203F4F853DB
:1084700020F4F8521A4310212846FFF74BFD002440
:1084800079E738B910212846FFF793FD00F01F0067
:10849000306070E701287FF472AF10212846FFF7A3
:1084A00088FD336820F01F0203F01F031A431021D8
:1084B0002846FFF72FFD00245DE700BFFFFF0F00F8
:1084C0007053FF1F6C53FF1F00288ED135212846A3
:1084D000FFF76FFD10F0020F0CBF01230023336084
:1084E00049E7002881D135212846FFF762FDC043C6
:1084F00000F0010030603EE738B934212846FFF72C
:1085000058FDC0F34000306035E701287FF437AFF5
:1085100034212846FFF74DFD346834B940F002029B
:1085200034212846FFF7F6FC25E720F0020234212B
:108530002846FFF7EFFC00241DE701287FF41FAF5A
:1085400034212846FFF735FD346834B940F0010284
:1085500034212846FFF7DEFC0DE720F0010234212C
:108560002846FFF7D7FC002405E728B93421284620
:10857000FFF71FFD3060FEE601287FF400AF1A68A8
:1085800034212846FFF7C6FC0024F4E628B924214C
:108590002846FFF70EFD3060EDE601287FF4EFAED0
:1085A0001A6824212846FFF7B5FC0024E3E60128D9
:1085B0007FF4E5AE1A6825212846FFF7ABFC0024BE
:1085C000D9E628B928212846FFF7F3FC3060D2E627
:1085D00001287FF4D4AE1A6828212846FFF79AFCB8
:1085E0000024C8E628B92A212846FFF7E2FC3060BB
:1085F000C1E601287FF4C3AE1A682A212846FFF796
:1086000089FC0024B7E628B923212846FFF7D1FCCE
:108610003060B0E601287FF4B2AE1A682321284604
:10862000FFF778FC0024A6E601287FF4A8AE1A68BC
:108630002B212846FFF76EFC00249CE628B92C214C
:108640002846FFF7B6FC306095E601287FF497AE28
:108650001A682C212846FFF75DFC00248BE60128D0
:108660007FF48DAE1968BB4B69B14FF0807292FBFD
:10867000F1F29A42A8BF1A46326015212846FFF748
:1086800049FC002477E61A46F6E728B93321284644
:10869000FFF78FFC30606EE601287FF470AE1A6839
:1086A00033212846FFF736FC002464E638B96C21F4
:1086B0002846FFF77EFCC0F3C04030605BE601282F
:1086C0007FF45DAE6C212846FFF773FC3368DB0452
:1086D00003F4002320F400221A436C212846FFF7FC
:1086E00019FC002447E638B96C212846FFF761FCE5
:1086F000C0F3804030603EE601287FF440AE6C213C
:108700002846FFF756FC33689B0403F4802320F4CB
:1087100080221A436C212846FFF7FCFB00242AE63E
:1087200038B900212846FFF744FC00F00100306012
:1087300021E601287FF423AE00212846FFF739FC0B
:10874000336820F0010203F001031A430021284698
:10875000FFF7E0FB00240EE638B901462846FFF794
:1087600028FCC0F34000306005E601287FF407AE26
:1087700000212846FFF71DFC33685B0003F002036D
:1087800020F002021A4300212846FFF7C3FB002411
:10879000F1E558B96C212846FFF70BFC4FF48073C4
:1087A000C0F3036043FA00F03060E4E501287FF491
:1087B000E6AD1B68102B23D00DDC022B1CD004DC93
:1087C000012B16D04FF0FF3314E0042B16D0082BEA
:1087D000F8D105230EE0402B14D003DC202BF1D17F
:1087E000032307E0802B0FD0B3F5807FEAD100236D
:1087F00000E00823336008E00723FBE70623F9E7DE
:108800000423F7E70223F5E730603368013300F013
:1088100057836C212846FFF7CCFB33681B0603F017
:10882000706320F070621A436C212846FFF772FBD8
:108830000024A0E538B96C212846FFF7BAFBC0F345
:10884000C130306097E501287FF499AD6C2128464E
:10885000FFF7AFFB3368DB0303F4C03320F4C0320F
:108860001A436C212846FFF755FB002483E50128B5
:108870007FF485AD6C212846FFF79BFB33689B0393
:1088800003F4804320F480421A436C212846FFF70A
:1088900041FB00246FE538B96C212846FFF789FBBE
:1088A000C0F30030306066E501287FF468AD6C21CC
:1088B0002846FFF77EFB33681B0303F4805320F444
:1088C00080521A436C212846FFF724FB002452E50E
:1088D0006C212846FFF76DFB9CB9430407D56C213A
:1088E0002846FFF766FBC0F3C310306043E5C0F3D2
:1088F000021300F4006003430CBF0023082333601D
:1089000039E5012C7FF43BAD440410D56C21284699
:10891000FFF74FFB3368DB0103F4F06320F4F062F0
:108920001A436C212846FFF7F5FA002423E5326844
:1089300011074CBF40F4006020F40060120120F0E9
:108940007000D2B202436C212846FFF7E3FA0024FC
:1089500011E500BFFFFF0F006C212846FFF729FB40
:10896000ACB910F4804408D06C212846FFF721FBF5
:10897000C0F3021030600024FDE4C0F3C31300F420
:10898000006003430CBF002308233360F3E4012C91
:108990007FF4F5AC6C212846FFF70BFB10F4804404
:1089A0004FF06C0128460ED0FFF703FB33681B0124
:1089B00003F0700320F070021A436C212846FFF781
:1089C000A9FA0024D7E4FFF7F4FA3368DB0103F4D3
:1089D000F06320F4F0621A436C212846FFF79AFAFC
:1089E000C9E401287FF4CBAC6C212846FFF7E1FAFB
:1089F000336820F00F0203F00F031A436C2128465E
:108A0000FFF788FA0024B6E438B96D212846FFF74D
:108A1000D0FAC0F3C0303060ADE401287FF4AFACD1
:108A20006D212846FFF7C5FA3368DB039BB220F4BB
:108A300000421A436D212846FFF76CFA00249AE49D
:108A400038B96D212846FFF7B4FAC0F341303060E1
:108A500091E401287FF493AC6D212846FFF7A9FA31
:108A600033685B0303F4C04320F4C0421A436D2112
:108A70002846FFF74FFA00247DE401287FF47FACFD
:108A80006D212846FFF795FA33681B0203F47063E3
:108A900020F470621A436D212846FFF73BFA002448
:108AA00069E438B96D212846FFF783FAC0F3411015
:108AB000306060E401287FF462AC6D212846FFF746
:108AC00078FA33685B0103F0600320F060021A4318
:108AD0006D212846FFF71EFA00244CE438B96D21B9
:108AE0002846FFF766FA00F00F00306043E40128E3
:108AF0007FF445AC6D212846FFF75BFA336820F020
:108B00000F0203F00F031A436D212846FFF702FA04
:108B1000002430E438B96D212846FFF74AFAC0F343
:108B20000060306027E401287FF429AC6D212846DD
:108B3000FFF73FFA33681B0603F0807320F0807262
:108B40001A436D212846FFF7E5F9002413E40128B4
:108B50007FF415AC6D212846FFF72BFA33681B0410
:108B600003F4FE0320F4FE021A436D212846FFF7AA
:108B7000D1F90024FFF7FFBB40B96C212846FFF76D
:108B800018FAC0F340403060FFF7F5BB01287FF4CE
:108B9000F6AB6C212846FFF70CFA33685B0403F44C
:108BA000003320F400321A436C212846FFF7B2F953
:108BB0000024FFF7E0BB00287FF417AC6F212846A4
:108BC000FFF7F7F9C0F304403060FFF7D4BB34601F
:108BD000FFF7D1BB01287FF4D2AB34212846FFF741
:108BE000E8F93368002B0CBF00234FF4806320F4B6
:108BF00080621A4334212846FFF78CF93168B54B5F
:108C000071B14FF0807292FBF1F29A42A8BF1A46FE
:108C1000326014212846FFF77DF90024FFF7ABBB33
:108C20001A46F5E780B914212846FFF7C2F9A94B87
:108C300030B14FF08072B2FBF0F0834228BF0346A0
:108C400033600024FFF797BB01287FF498AB1B68C3
:108C500073B14FF0807292FBF3F29E4B9A42C8BF01
:108C60001A4614212846FFF755F90024FFF783BB65
:108C7000984AF6E701287FF482AB6C212846FFF77B
:108C800098F933685B0303F4005320F400521A434D
:108C90006C212846FFF73EF90024FFF76CBB40B972
:108CA0006C212846FFF785F9C0F303503060FFF7C9
:108CB00062BB01287FF463AB6C212846FFF779F98A
:108CC00033681B0503F4700320F470021A436C210F
:108CD0002846FFF71FF90024FFF74DBB80B9132189
:108CE0002846FFF766F97B4B30B14FF08072B2FB3C
:108CF000F0F0834228BF034633600024FFF73BBBFC
:108D000001287FF43CAB1968724B71B14FF080724F
:108D100092FBF1F29A42A8BF1A463260132128460C
:108D2000FFF7F8F80024FFF726BB1A46F5E740B92D
:108D300070212846FFF73DF9C0F307203060FFF7A8
:108D40001ABB01287FF41BAB70212846FFF731F9CD
:108D50003268120220F47F4092B20243702128460A
:108D6000FFF7D8F800212846FFF723F93368002BD6
:108D700020F004020CBF002304231A4300212846DC
:108D8000FFF7C8F80024FFF7F6BA01287FF4F7AA26
:108D900070212846FFF70DF9327820F0FF000243DA
:108DA00070212846FFF7B6F80024FFF7E4BA40B96F
:108DB00070212846FFF7FDF8C0F301403060FFF74F
:108DC000DABA01287FF4DBAA1B68032B7BD8702159
:108DD0002846FFF7EEF833681B0403F4403320F411
:108DE00040321A4370212846FFF794F80024FFF719
:108DF000C2BA40B970212846FFF7DBF8C0F38040C3
:108E00003060FFF7B8BA01287FF4B9AA1B68012BBC
:108E10005CD870212846FFF7CCF833689B0403F434
:108E2000802320F480221A4370212846FFF772F82D
:108E30000024FFF7A0BA40B970212846FFF7B9F81F
:108E4000C0F301503060FFF796BA01287FF497AA6B
:108E500070212846FFF7ADF833681B0503F4401373
:108E600020F440121A4370212846FFF753F80024DB
:108E7000FFF781BA30B939212846FFF79AF83060F8
:108E8000FFF779BA01287FF47AAA1A6839212846AF
:108E9000FFF740F80024FFF76EBA30B93A212846B0
:108EA000FFF787F83060FFF766BA01287FF467AAFA
:108EB0001A683A212846FFF72DF80024FFF75BBA1D
:108EC0001024FFF758BA1024FFF755BA1024FFF703
:108ED00052BA00BFFFFF0F0007B5019239B9024631
:108EE00001AB0120FFF7DCF803B05DF804FB0820BC
:108EF000FAE710B413460446084619B9224610BCD6
:108F0000FFF7CEB8082010BC704738B522210020EA
:108F1000FFF74FF818B90A4B186806F0A9FA094B81
:108F2000094CDD68606A2B689B6998472B6820684C
:108F30001B6998472B6860681B699847012038BDFA
:108F40006C53FF1F704C0200C017FF1F70B5534ECB
:108F50005348544C06F026FAF5686B6803F1640236
:108F6000A26003F1A402E26003F1C402226103F5EE
:108F70009272226003F5A272626003F5D27262629D
:108F800003F5E272A26203F5617203F18400A2614B
:108F900003F5697203F57173E3612B6822621B6943
:108FA000606198472B6820691B6998472B68E068C7
:108FB0001B6998472B68E0691B6998472B68206AF2
:108FC0001B6998472B68A069DB6898472B68206865
:108FD0001B6998472B6860681B6998472B68A068D5
:108FE000DB6898472B68606ADB6898472B68A06A43
:108FF000DB6898472B68A0699B6998472A4B3269C0
:109000001A606B68294903F531735360284B5A691C
:109010000A602849C2F804122749C2F8081200263B
:10902000012111705670254A1A62254ADA61254AD3
:109030009A61254A5A62254A9A63254A5A63254A03
:109040009A62254ADA62254A9A64254A5A64254A70
:109050005A65254A1A65254ADA64254A1A66254A58
:10906000DA653222DA604FF4F0729A600220224A06
:1090700019749A65FEF7EEFE2B68A06ADB689847C4
:10908000A06A1E4C042343752B681B68984723680D
:109090009847A3683046BDE870401847704C0200FE
:1090A0007053FF1FC017FF1FFC55FF1F6C53FF1F9E
:1090B0007431FF1F0B8F0100497E0100717F010099
:1090C000B17F0100AD7F0100A97F0100F38E010097
:1090D000D98E01003B7F010081800100317F0100BA
:1090E00071800100317E0100017C0100E17B010003
:1090F000557E0100F57B0100B17D01006809FF1F6D
:1091000018B9034B1B680B6070470820704700BFFD
:109110000856FF1F014B00225A6070477431FF1F31
:109120000428F8B514465ED006D8022844D02FD8BB
:10913000B8B104242046F8BD062800F0838076D319
:10914000FC28F6D11468464D464B002C00F0818077
:10915000DC6828692368DB689847236828699B696D
:1091600015E0136833F0030278D113F0010F3C4D82
:109170003C4E0FD0F3681B681B69686898472468E9
:1091800014F002040ED0F36828681B681B69984726
:109190000024CFE7F76868683B68DB6898473B685E
:1091A0009B69EAE7F66828683368DB6898473368A4
:1091B00028689B699847BDE714682A4B64B1DC684E
:1091C0006068236800F5F270DB6898476068236880
:1091D00000F5F2709B69DAE7DB6858681B6800F5F8
:1091E000F2709B68E6E715681D4E1E4B5DB1012DC0
:1091F00015D0DD6830692B681B6998472B6830698A
:109200001B6A984709E0DF6830693B68DB6898476C
:109210003B689B693069984728462060B8E7DF685B
:1092200030693B68DB6898473B685B69F2E70D4B48
:109230000B4ADB68106A1B681B6A9847003018BF2E
:109240000120EAE7074B064ADB68506A1B681B6A85
:10925000F3E7DB6828691B681B69ABE7102469E743
:10926000F817FF1F704C02001C4B70B5DD681C4CDA
:109270002B68A0689B6998472B68A0699B699847F1
:109280002B68E0699B6998472B68E0689B68984762
:109290002B6820699B6898472B6860699B68984792
:1092A0002B6820689B6898472B6860689B68984784
:1092B0002B68206A9B6898472B68606A9B68984770
:1092C0002B68A0689B6898472B68A0699B689847A3
:1092D0002B68E0699B68BDE870401847704C02003D
:1092E000F817FF1F034B044A1B680146002006F0D5
:1092F00008B900BF0456FF1F0856FF1F014B18682E
:1093000006F037B90456FF1F022804BF0B4B93F831
:10931000D00030B90A4BDB681B685B69094A90686A
:109320001847012809D1054B93F8D030012B04D1FF
:10933000034BDB681B689B69F0E770477431FF1FC4
:10934000704C0200F817FF1F2DE9F0471C4D9DF8E7
:1093500020709DF82460994655F8203004468846D0
:109360009B68002148F080009246984755F82430C9
:1093700000219B685046984755F8243000219B688F
:109380004846984755F8243000219B68384698474E
:1093900055F8243030469B6801219847094B53F813
:1093A000243049EA0A2908F07F0847EA092703EB35
:1093B000880846EA0726C8F80460BDE8F08700BFC1
:1093C0000056FF1F0456FF1F07B5D3B20193C2F327
:1093D00007230093C2F30743120EFFF7B5FF03B054
:1093E0005DF804FB0A4601460020FFF7EDBF73B5A8
:1093F0000D460646E8B9104C94F8283043B10F4B9F
:109400001B682721D3F8A020FFF7DEFF84F828602F
:1094100000242A462D210020FFF7D6FF2046019484
:109420000094234622462021FFF78EFF204602B0FB
:1094300070BD0820FBE700BFF817FF1F0456FF1F91
:1094400037B50D460446C8B90D4B012283F82820D4
:1094500081EAE172A2EBE1722721FFF7B5FF002D4F
:10946000ACBF0123022301932046009423462246E9
:109470002021FFF769FF204603B030BD0820FBE73D
:10948000F817FF1F0021DBE74942D9E7D8E770B59D
:109490002B4A4FF4237301F07F0403FB0023234482
:1094A000054693F80C32DB0706D4264B53F82030E0
:1094B00003EB8404606870BD234E56F82030002111
:1094C0009B682046984756F8253000219B6808463F
:1094D000984756F8253000219B680846984756F86B
:1094E000253000219B680846984756F82530012111
:1094F0009B680020984756F8253000219B6820463D
:10950000984756F8253000219B680846984756F83A
:109510002530002104029B680846984756F82530FC
:10952000002104439B680846984756F825302402DA
:1095300004439B680121002098472402204370BD0A
:109540000856FF1F0456FF1F0056FF1F10B50C469C
:1095500001460020FFF79BFF206010BD38B50C4688
:1095600021210546FFF793FF216801442160284629
:10957000BDE838403BE7222AF8B504460D461E46B2
:1095800000F0468300F28E800E2A00F03C8241D823
:10959000062A00F0B88119D8022A00F0618107D8A4
:1095A000002A00F03A81012A00F04A8104243AE1BD
:1095B000042A00F07C8140F26981002840F09A8101
:1095C00026212846FFF763FF30602CE10A2A00F0CD
:1095D000D2810FD8072A00F0B281082AE6D10028EC
:1095E00040F0618135212846FFF751FFC0F340204C
:1095F000306018E10C2A00F0D68140F2C9810028C1
:1096000040F0EE8134212846FFF741FF00F00100D1
:10961000306008E1152A00F065821FD8112A00F099
:109620001E820DD80F2A00F0FF81102ABED100281B
:1096300040F00B8225212846FFF729FF3060F2E039
:10964000132A00F0348240F22182002840F0408248
:109650002B212846FFF71BFF3060E4E01B2A00F0B7
:1096600083820DD8172A00F04E82182A9ED1002836
:1096700040F0708233212846FFF709FF3060D2E0C6
:109680001D2A00F0AB82C0F08C82212A8ED10028E6
:1096900040F0AB8201462846FFF7F9FE00F00100DA
:1096A0003060C0E0AE2A00F0AE8451D8A72A00F0A6
:1096B000F48328D8A32A00F02D8310D88C2A00F038
:1096C000C482A22A7FF472AF002840F00F836C217D
:1096D0002846FFF7DCFEC0F3C1303060A3E0A52AC6
:1096E00000F0528340F233836C212846FFF7CFFE0F
:1096F000002C40F0AC83410440F19E83000900F04F
:10970000700030608FE0AA2A00F0138410D8A82AD5
:1097100000F0DF83A92A7FF449AF002840F0F583E9
:109720006D212846FFF7B3FEC0F3413030607AE088
:10973000AC2A00F0388440F21984002840F04F84AD
:109740006D212846FFF7A3FEC0F3006030606AE099
:10975000BB2A00F03B8536D8B62A00F0B1841FD86A
:10976000B42A00F07684B52A7FF420AF002840F0B8
:109770007F8434212846FFF78AFE430540F1758433
:1097800014212846FFF783FEBD4B30B14FF08072A5
:10979000B2FBF0F0834228BF03463360002442E06E
:1097A000B92A00F0CB8400F2E884B82A7FF4FEAE38
:1097B000002840F0AE846C212846FFF768FEC0F315
:1097C000403030602FE0CC2A00F0838512D8BF2AC9
:1097D00000F03B85C02A00F05A85BC2A7FF4E6AE33
:1097E000002840F0208570212846FFF750FEC0B2C7
:1097F000306018E0D12A00F08B85D22A00F09B85DA
:10980000CE2A7FF4D3AE00284DD16F212846FFF732
:109810003EFEC0F30900306005E030B92D21284636
:10982000FFF735FE30602046F8BD012801D0002446
:10983000F9E71A682D212846FFF7C6FD0024F2E754
:1098400028B921212846FFF722FE3060EBE70128E6
:10985000EDD11A6821212846FFF7B6FD0024E2E782
:1098600028B927212846FFF712FE3060DBE70128E0
:10987000DDD11A68002AB8BF524227212846FFF7D7
:10988000A3FD804B83F828400024CCE758B922215F
:109890002846FFF7FCFD10F4000318BF4FF07F438C
:1098A00018433060BFE7012CC1D10424BBE730B9B5
:1098B000754B53F82130D3F8A0303360B3E701285B
:1098C000B5D1714B53F821203368002BB8BF5B42F0
:1098D000C2F8A03020212846FFF7D9FD0446002811
:1098E000A5D13268002AB8BF524227212846FFF787
:1098F0006BFD98E701289AD11A6826212846FFF7C0
:1099000063FD00248FE738B910212846FFF7BFFD1B
:10991000C0F30420306086E7012888D11021284652
:10992000FFF7B5FD33681B0203F4F85320F4F85237
:109930001A4310212846FFF747FD002473E738B982
:1099400010212846FFF7A3FD00F01F0030606AE7F2
:1099500001287FF46CAF10212846FFF798FD33688B
:1099600020F01F0203F01F031A4310212846FFF7BF
:109970002BFD002457E7002895D135212846FFF715
:1099800086FD10F0020F0CBF0123002333604AE76D
:10999000002888D135212846FFF779FDC04300F023
:1099A000010030603FE738B934212846FFF76FFDEA
:1099B000C0F34000306036E701287FF438AF34212F
:1099C0002846FFF764FD33685B0003F0020320F0D4
:1099D00002021A4334212846FFF7F6FC002422E74E
:1099E00001287FF424AF34212846FFF750FD336867
:1099F00020F0010203F001031A4334212846FFF747
:109A0000E3FC00240FE728B934212846FFF73FFD87
:109A1000306008E701287FF40AAF1A68342128462D
:109A2000FFF7D2FC0024FEE628B924212846FFF7E0
:109A30002EFD3060F7E601287FF4F9AE1A68242184
:109A40002846FFF7C1FC0024EDE601287FF4EFAEC5
:109A50001A6825212846FFF7B7FC0024E3E628B959
:109A600028212846FFF713FD3060DCE601287FF44B
:109A7000DEAE1A6828212846FFF7A6FC0024D2E6AD
:109A8000FFFF0F00F817FF1F0456FF1F28B92A21F8
:109A90002846FFF7FCFC3060C5E601287FF4C7AE1E
:109AA0001A682A212846FFF78FFC0024BBE628B954
:109AB00023212846FFF7EBFC3060B4E601287FF451
:109AC000B6AE1A6823212846FFF77EFC0024AAE6DA
:109AD00001287FF4ACAE1A682B212846FFF774FCEE
:109AE0000024A0E628B92C212846FFF7D0FC3060DE
:109AF00099E601287FF49BAE1A682C212846FFF7CF
:109B000063FC00248FE678B915212846FFF7BFFCD7
:109B1000BB4B30B14FF08072B2FBF0F0834228BFF4
:109B20000346336000247EE601287FF480AE196886
:109B3000B34B69B14FF0807292FBF1F29A42A8BF29
:109B40001A46326015212846FFF73EFC00246AE6DB
:109B50001A46F6E701287FF46AAE1A6833212846D0
:109B6000FFF732FC00245EE638B96C212846FFF787
:109B70008EFCC0F3C040306055E601287FF457AE3C
:109B80006C212846FFF783FC3368DB0403F40023D1
:109B900020F400221A436C212846FFF715FC00240C
:109BA00041E638B96C212846FFF771FCC0F38040CC
:109BB000306038E601287FF43AAE6C212846FFF782
:109BC00066FC33689B0403F4802320F480221A434C
:109BD0006C212846FFF7F8FB002424E600287FF4D8
:109BE00062AE884B1B6833601DE601287FF41FAE10
:109BF00000212846FFF74BFC336820F0010203F0F8
:109C000001031A4300212846FFF7DEFB00240AE681
:109C100038B901462846FFF73AFCC0F340003060EF
:109C200001E601287FF403AE00212846FFF72FFC50
:109C300033685B0003F0020320F002021A430021A4
:109C40002846FFF7C1FB0024EDE558B96C212846F2
:109C5000FFF71DFC4FF48073C0F3036043FA00F07C
:109C60003060E0E501287FF4E2AD1B68102B23D0C3
:109C70000DDC022B1CD004DC012B16D04FF0FF337F
:109C800014E0042B16D0082BF8D105230EE0402B4E
:109C900014D003DC202BF1D1032307E0802B0FD05D
:109CA000B3F5807FEAD1002300E00823336008E0A9
:109CB0000723FBE70623F9E70423F7E70223F5E789
:109CC00030603368013300F049836C212846FFF788
:109CD000DEFB33681B0603F0706320F070621A43EA
:109CE0006C212846FFF770FB00249CE501287FF4D7
:109CF0009EAD6C212846FFF7CAFB3368DB0303F4F3
:109D0000C03320F4C0321A436C212846FFF75CFBB5
:109D1000002488E538B96C212846FFF7B8FBC0F36A
:109D2000803030607FE501287FF481AD6C212846CA
:109D3000FFF7ADFB33689B0303F4804320F48042BC
:109D40001A436C212846FFF73FFB00246BE538B926
:109D50006C212846FFF79BFBC0F30030306062E5C2
:109D600001287FF464AD6C212846FFF790FB33682F
:109D70001B0303F4805320F480521A436C212846BD
:109D8000FFF722FB00244EE56C212846FFF77FFBFE
:109D90000746CCB910F4804405D0C70907F4F06732
:109DA000376000243FE56C212846FFF770FB17F071
:109DB0000B0F4FEA201000F0700001D1306036E543
:109DC00040F0080030602EE5012C7FF430AD6C21AE
:109DD0002846FFF75CFB10F480444FF06C012846E6
:109DE00012D0FFF754FB3368DB0103F4F06320F477
:109DF000F0621A436C212846FFF7E6FA002412E5C8
:109E0000FFFF0F000856FF1FFFF741FB6C2120F4F6
:109E100000622846FFF7D8FA6C212846FFF737FB87
:109E200033681B0103F0700320F070021A436C21A9
:109E30002846FFF7C9FAF6E4C309020503F4F06304
:109E400001D43360F3E443F008033360EBE4012C06
:109E50007FF4EDAC10F480444FF06C0128460ED036
